:020000040000FA
:10000000000400200108000095040000E107000042
:100010009F040000A9040000B304000000000000D9
:1000200000000000000000000000000025080000A3
:10003000BD04000000000000C7040000D10400005F
:10004000DB040000E5040000EF040000F9040000F8
:10005000030500000D050000170500002105000044
:100060002B050000350500003F0500004905000094
:10007000530500005D0500006705000071050000E4
:100080007B050000850500008F0500009905000034
:10009000A3050000AD050000B7050000C105000084
:1000A000CB050000D5050000DF050000E9050000D4
:1000B000F3050000FD050000070600001106000022
:1000C0001B060000250600002F0600003906000070
:1000D000430600004D0600005706000061060000C0
:1000E0006B060000750600007F0600008906000010
:1000F000930600009D060000A7060000B106000060
:10010000BB0600001FB500F003F88DE80F001FBD0F
:1001100000F06CBBF0B54FF6FF734FF4B4751A46A0
:100120006E1E11E0A94201D3344600E00C46091BC3
:1001300030F8027B641E3B441A44F9D19CB204EBB4
:10014000134394B204EB12420029EBD198B200EBB6
:10015000134002EB124140EA0140F0BDB24992B0B7
:100160000446D1E90001CDE91001FF224021684693
:1001700000F0E2FA94E80F008DE80F00684610A93D
:1001800002E004C841F8042D8842FAD110216846E3
:10019000FFF7C0FF1090AA208DF8440000F0F1F89E
:1001A0004FF01024A06910226946803000F0F2F868
:1001B000A069082210A900F0EDF800F0D6F84FF081
:1001C00080510A69496900684A43824201D8102077
:1001D00070470020704710B5D0E900214FF08050E3
:1001E00002EB8103026944696243934209D84FF0EC
:1001F0001022536903EB81030169406941438B423B
:1002000001D9092010BD5069401C01D0002010BD4B
:100210000F2010BD70B501680446844D4FF01020CA
:10022000072950D2DFE801F0330419293C1E2500CC
:10023000D4E9026564682946304600F0BDF82A46D4
:100240002146304600F0A6F8AA002146304600F0CC
:1002500047FA002800D0032070BD00F0F9FA4FF4EF
:10026000805007E0201DFFF7AAFF0028F4D100F01E
:10027000EFFA60682860002070BD241D94E8070034
:10028000920000F02DFA0028F6D00E2070BD806993
:10029000401C12D0201DFFF79EFF0028F6D109E078
:1002A0008069401C09D0201DFFF789FF0028EDD18F
:1002B000606820B12046FFF751FF042070BD00F0B8
:1002C00060F800F052F8072070BD10B50C461828F1
:1002D00002D00120086010BD2068FFF79BFF20605E
:1002E00010BD4FF01024A069401C05D0A569A66977
:1002F00080353079AA2808D06069401C2DD060690B
:100300000068401C29D060692CE010212846FFF7C6
:1003100001FF316881421CD1A16901F18002C03125
:1003200005E030B108CA51F8040D984201D101200E
:1003300000E000208A42F4D158B1286810B10428A6
:1003400003D0FEE7284600F049F83849686808609D
:1003500008E000F016F800F008F84FF4805001684B
:10036000491C01D000F04EFAFEE7BFF34F8F304832
:100370000168304A01F4E06111430160BFF34F8F1F
:10038000FEE74FF010208169491C02D0806900F01F
:1003900058B870472DE9F04117460D46064600242F
:1003A00006E03046296800F05FF8641C2D1D361DFC
:1003B000BC42F6D3BDE8F08170B50C4605464FF45B
:1003C000806608E0284600F03CF8B44205D3A4F566
:1003D000806405F58055002CF4D170BD4168044659
:1003E00009B1012500E000254FF010267069A268D0
:1003F000920000F075F938B145B17669A568646876
:100400004FF48010844203D3FFF7BBFFFFF7ADFF2B
:100410008542F9D229463046FFF7CEFF2A462146CB
:100420003046FFF7B7FFEFE7740800000000002038
:100430000CED00E00400FA05144801680029FCD026
:100440007047134A0221116010490B68002BFCD041
:100450000F4B1B1D186008680028FCD0002010609E
:1004600008680028FCD07047094B10B501221A60BB
:10047000064A1468002CFCD0016010680028FCD0EB
:100480000020186010680028FCD010BD00E4014076
:1004900004E5014008208F490968095808471020E1
:1004A0008C4909680958084714208A49096809587D
:1004B00008471820874909680958084730208549A6
:1004C00009680958084738208249096809580847C7
:1004D0003C20804909680958084740207D4909683F
:1004E0000958084744207B490968095808474820AB
:1004F00078490968095808474C207649096809581D
:100500000847502073490968095808475420714921
:1005100009680958084758206E490968095808476A
:100520005C206C49096809580847602069490968D6
:10053000095808476420674909680958084768202E
:1005400064490968095808476C20624909680958D4
:10055000084770205F4909680958084774205D49B9
:1005600009680958084778205A490968095808470E
:100570007C2058490968095808478020554909686E
:1005800009580847842053490968095808478820B2
:1005900050490968095808478C204E49096809588C
:1005A000084790204B490968095808479420494951
:1005B00009680958084798204649096809580847B2
:1005C0009C204449096809580847A0204149096806
:1005D00009580847A4203F49096809580847A82036
:1005E0003C49096809580847AC203A490968095844
:1005F0000847B0203749096809580847B4203549E9
:10060000096809580847B820324909680958084755
:10061000BC203049096809580847C0202D4909689D
:1006200009580847C4202B49096809580847C820B9
:100630002849096809580847CC20264909680958FB
:100640000847D0202349096809580847D420214980
:10065000096809580847D8201E49096809580847F9
:10066000DC201C49096809580847E0201949096835
:1006700009580847E4201749096809580847E8203D
:100680001449096809580847EC20124909680958B3
:100690000847F0200F49096809580847F4200D4918
:1006A000096809580847F8200A490968095808479D
:1006B000FC2008490968095808475FF4807005491B
:1006C000096809580847000003480449024A034BD7
:1006D0007047000000000020800800008008000033
:1006E00040EA010310B59B070FD1042A0DD310C8AF
:1006F00008C9121F9C42F8D020BA19BA884201D901
:10070000012010BD4FF0FF3010BD1AB1D30703D048
:10071000521C07E0002010BD10F8013B11F8014BFE
:100720001B1B07D110F8013B11F8014B1B1B01D11A
:10073000921EF1D1184610BD02F0FF0343EA0322D6
:1007400042EA024200F005B87047704770474FF028
:1007500000020429C0F0128010F0030C00F01B808E
:10076000CCF1040CBCF1020F18BF00F8012BA8BF9C
:1007700020F8022BA1EB0C0100F00DB85FEAC17C60
:1007800024BF00F8012B00F8012B48BF00F8012B13
:1007900070474FF0000200B5134694469646203944
:1007A00022BFA0E80C50A0E80C50B1F12001BFF42A
:1007B000F7AF090728BFA0E80C5048BF0CC05DF890
:1007C00004EB890028BF40F8042B08BF704748BFDE
:1007D00020F8022B11F0804F18BF00F8012B704752
:1007E000014B1B68DB6818470000002009480A49D4
:1007F0007047FFF7FBFFFFF785FC00BD20BFFDE75B
:10080000064B1847064A1060016881F30888406863
:10081000004700008008000080080000E30200009C
:10082000000000201EF0040F0CBFEFF30881EFF36F
:100830000981886902380078182803D100E0000097
:10084000074A1047074A12682C3212681047000006
:1008500000B5054B1B68054A9B58984700BD000032
:10086000CB0200000000002070080000040000001F
:10087000001000000000000000FFFFFF0090D00308
:10100000481300201D3B0200CDBB00008F3A0200B8
:10101000CDBB0000CDBB0000CDBB00000000000038
:10102000000000000000000000000000753B02000E
:10103000CDBB000000000000CDBB0000CDBB000018
:10104000DD3B0200E33B0200CDBB0000CDBB000056
:10105000CDBB0000CDBB0000CDBB0000CDBB000070
:10106000E93B0200CDBB0000CDBB0000EF3B02001E
:10107000CDBB0000F53B0200FB3B0200013C02003F
:10108000CDBB0000CDBB0000CDBB0000CDBB000040
:10109000CDBB0000CDBB0000CDBB0000CDBB000030
:1010A000CDBB0000073C0200CDBB0000CDBB000063
:1010B000CDBB0000CDBB0000CDBB0000CDBB000010
:1010C0000D3C0200CDBB0000CDBB0000CDBB00003D
:1010D000CDBB0000CDBB0000CDBB0000CDBB0000F0
:1010E000CDBB0000CDBB0000CDBB0000CDBB0000E0
:1010F000CDBB0000CDBB0000CDBB0000CDBB0000D0
:10110000CDBB0000CDBB000000F002F822F0F3FCE4
:101110000AA090E8000C82448344AAF10107DA4552
:1011200001D122F0E8FCAFF2090EBAE80F0013F08B
:10113000010F18BFFB1A43F001031847802F02006C
:10114000A02F02000A4410F8014B14F00F0508BF4D
:1011500010F8015B240908BF10F8014B6D1E05D083
:1011600010F8013B6D1E01F8013BF9D1641E03D05C
:10117000641E01F8015BFBD19142E4D3704700008B
:101180000023002400250026103A28BF78C1FBD890
:10119000520728BF30C148BF0B6070471FB500F031
:1011A0003DF88DE80F001FBD1EF0040F0CBFEFF3DC
:1011B0000880EFF30980014A104700003B2E000031
:1011C0008269034981614FF00100104470470000BB
:1011D000D511000001B41EB400B512F045FA01B4F7
:1011E0000198864601BC01B01EBD0000F0B4404627
:1011F000494652465B460FB402A0013001B506488D
:10120000004700BF01BC86460FBC80468946924617
:101210009B46F0BC704700000911000022F068BC3A
:1012200070B51A4C054609202070A01C00F05FF82C
:101230005920A08029462046BDE8704007F0AEBF87
:1012400007F0B7BF70B50C461149097829B1A0F174
:101250006001552908D3012013E0602804D06928D3
:1012600002D043F201000CE020CC0A4E94E80E00BC
:1012700006EB8000A0F58050241FD0F8806E284631
:10128000B047206070BD01207047000008000020BA
:101290001C000020603C020010B504460021012023
:1012A00000F03CF800210B2000F038F80421192050
:1012B00000F034F804210D2000F030F804210E2055
:1012C00000F02CF804210F2000F028F80421C84376
:1012D00000F024F80621162000F020F80621152041
:1012E00000F01CF82046FFF79BFF002010BD4FF6D2
:1012F000FE7101807047FFF7A3BF10487047104A86
:1013000010B514680E4B0F4A08331A60FFF79AFFA6
:101310000B48001D046010BD704770474907090E57
:10132000002806DA00F00F0000F1E02080F8141D1C
:10133000704700F1E02080F80014704703F9004284
:101340001005024001000001FE48002101604160DB
:10135000018170472DE9F743044692B091464068F9
:1013600012F048FC40B1606812F04DFC20B9607882
:1013700000F00300022801D0012000E00020F14E1F
:101380004D463072484612F0F1FB18B1102015B0EE
:10139000BDE8F0832946012001F02AFF0028F6D19C
:1013A00001258DF842504FF4C050ADF840000022A6
:1013B00010A9284606F090FB0028E8D18DF842508D
:1013C0004FF428504FF00008ADF8400047461C216C
:1013D0006846CDF81C8022F02EFB9DF81C0008AA60
:1013E00020F00F00401C20F0F00010308DF81C00A1
:1013F00020788DF81D0061789DF81E0061F3420091
:1014000040F001008DF81E009DF800000AA940F090
:1014100002008DF800002089ADF83000ADF8327080
:10142000608907AFADF834000B97606810AC0E9080
:101430000A94684606F045F90028A8D1BDF82000B6
:1014400030808DF8425042F60120ADF840009DF802
:101450001E0008AA20F00600801C20F001008DF874
:101460001E000220ADF83000ADF8340013A80E9035
:101470000AA9684606F025F9002888D1BDF82000A1
:101480007080311D484600F033F9002887D18DF86F
:10149000425042F6A620ADF840001C216846CDF827
:1014A0001C8022F0C8FA9DF81C00ADF8345020F0E2
:1014B0000F00401C20F0F00010308DF81C009DF84B
:1014C0001D0008AA20F0FF008DF81D009DF81E00E9
:1014D0000AA920F0060040F00100801C8DF81E00D3
:1014E0009DF800008DF8445040F002008DF8000097
:1014F000CDE90A4711A80E90ADF83050684606F0C5
:10150000E0F8002899D1BDF82000F08000203EE7E7
:101510003EB504460820ADF80000204612F026FB38
:1015200008B110203EBD2146012001F061FE0028D7
:10153000F8D12088ADF804006088ADF80600A088D6
:10154000ADF80800E088ADF80A007E4801AB6A46B5
:101550008088002106F0BAFCBDF800100829E1D00F
:1015600003203EBD1FB50446002002900820ADF8C0
:101570000800CDF80CD0204612F0F8FA10B1102077
:1015800004B010BD6F4802AA81884FF6FF7006F0C4
:10159000E4FE0028F4D1BDF80810082901D003208A
:1015A000EEE7BDF800102180BDF802106180BDF8A3
:1015B0000410A180BDF80610E180E1E701B582B01A
:1015C0000220ADF800005F4802AB6A464088002167
:1015D00006F07CFCBDF80010022900D003200EBDEF
:1015E0001CB5002100910221ADF80010019012F00D
:1015F000E3FA08B110201CBD52486A4641884FF6F4
:10160000FF7006F0AAFEBDF800100229F3D00320F7
:101610001CBDFEB54B4C06461546207A0F46C0074A
:1016200005D0084612F0A2FA18B11020FEBD0F2016
:10163000FEBDF82D01D90C20FEBD304612F096FA01
:1016400018BB208801A905F082FD0028F4D130786C
:101650008DF80500208801A906F017FC0028EBD1C1
:1016600000909DF800009DF8051040F002008DF8F4
:101670000000090703D040F008008DF80000208822
:10168000694606F09FFB0028D6D1ADF808502088A7
:101690003B4602AA002106F019FCBDF80810A94239
:1016A000CAD00320FEBD7CB5054600200090019005
:1016B0000888ADF800000C462846019512F09AFA09
:1016C00018B9204612F078FA08B110207CBD15B187
:1016D000BDF8000050B11B486A4601884FF6FF7004
:1016E00006F03BFEBDF8001021807CBD0C207CBDC7
:1016F00030B593B0044600200D460090142101A897
:1017000022F099F91C2108A822F095F99DF8000013
:10171000CDF808D020F00F00401C20F0F000103071
:101720008DF800009DF8010020F0FF008DF8010009
:101730009DF8200040F002008DF8200001208DF877
:10174000460001E0E601002042F60420ADF8440026
:1017500011A801902088ADF83C006088ADF83E00EB
:10176000A088ADF84000E088ADF842009DF8020086
:1017700006AA20F00600801C20F001008DF802006F
:101780000820ADF80C00ADF810000FA8059001A9D5
:1017900008A805F096FF002803D1BDF8180028809E
:1017A000002013B030BD0000F0B5007B059F1E4641
:1017B00014460D46012800D0FFDF0C2030803A206F
:1017C0003880002C08D0287A032806D0287B0128EE
:1017D00000D0FFDF17206081F0BDA889FBE72DE96D
:1017E000F04786B0144691F80C900E9A0D46B9F168
:1017F000010F0BD01021007B2E8A8846052807D0C8
:10180000062833D0FFDF06B0BDE8F0870221F2E7FB
:10181000E8890C2100EB400001EB400018803320E8
:101820001080002CEFD0E889608100271AE0009634
:10183000688808F1020301AA696900F085FF06EBD8
:101840000800801C07EB470186B204EB4102BDF89B
:10185000040090810DF1060140460E3210F02CFA82
:101860007F1CBFB26089B842E1D8CCE73420108039
:10187000E889B9F1010F11D0122148430E301880C8
:10188000002CC0D0E88960814846B9F1010F00D032
:101890000220207300270DF1040A1FE00621ECE767
:1018A0000096688808F1020301AA696900F04CFFFC
:1018B00006EB0800801C86B2B9F1010F12D007EBCD
:1018C000C70004EB4000BDF80410C18110220AF1EA
:1018D0000201103022F00EF87F1CBFB26089B842BE
:1018E000DED890E707EB470104EB4102BDF80400A6
:1018F000D0810AF102014046103210F0DDF9EBE729
:101900002DE9F0470E4688B090F80CC096F80C8090
:10191000378AF5890C20109902F10C044FF0000A67
:10192000BCF1030F08D0BCF1040F3ED0BCF1070F8F
:101930007DD0FFDF08B067E705EB850C00EB4C00BE
:10194000188031200880002AF4D0A8F1060000F0A9
:10195000FF09558125E0182101A822F06CF80097B5
:101960007088434601AA716900F0EEFEBDF80400DC
:101970002080BDF80600E080BDF808002081A21C90
:101980000DF10A01484610F097F9B9F1000F00D0A7
:1019900018B184F804A0A4F802A007EB080087B2ED
:1019A0000A346D1EADB2D6D2C4E705EB850C00EB50
:1019B0004C00188032200880002ABBD0A8F1050016
:1019C00000F0FF09558137E000977088434601AA6F
:1019D000716900F0B9FE9DF80600BDF80410E180C1
:1019E0002179420860F3000162F34101820862F349
:1019F0008201C20862F3C301020962F304114209C1
:101A000062F34511820962F386112171C009607188
:101A1000BDF80700208122460DF10901484610F06B
:101A20004BF918B184F802A0A4F800A000E007E088
:101A300007EB080087B20A346D1EADB2C4D279E755
:101A4000A8F1020084B205FB08F000F10E0CA3F827
:101A500000C035230B80002AA6D0558194810097C1
:101A600083B270880E32716900F06EFE62E72DE974
:101A7000F84F1E460A9D0C4681462AB1607A00F551
:101A80008070D080E089108199F80C000C274FF00D
:101A900000084FF00E0A0D2873D2DFE800F09E0711
:101AA0000E1C28303846556A737373002146484629
:101AB0000095FFF779FEBDE8F88F207B9146082856
:101AC00002D0032800D0FFDF378030200AE000BFBB
:101AD000A9F80A80EFE7207B9146042800D0FFDFB9
:101AE000378031202880B9F1000FF1D1E3E7207B66
:101AF0009146042800D0FFDF37803220F2E7207BB8
:101B00009146022800D0FFDF37803320EAE7207BB0
:101B10001746022800D0FFDF3420A6F800A0288056
:101B2000002FC8D0A7F80A80C5E7207B17460428F5
:101B300000D0FFDF3520A6F800A02880002FBAD003
:101B40004046A7F80A8012E0207B1746052802D0FD
:101B5000062800D0FFDF1020308036202880002F9C
:101B6000A9D0E0897881A7F80E80B9F80E00B88175
:101B7000A1E7207B9146072800D0FFDF3780372080
:101B8000B0E72AE04FF0120018804FF0380017003D
:101B9000288090D0E0897881A7F80E80A7F810807F
:101BA00099F80C000A2805D00B2809D00C280DD074
:101BB000FFDF80E7207B0A2800D0FFDF01200AE05A
:101BC000207B0B2800D0FFDF042004E0207B0C28C2
:101BD00000D0FFDF052038736DE7FFDF6BE770B5DE
:101BE0000C46054601F07DFA20B10078222804D287
:101BF000082070BD43F2020070BD052128460EF09A
:101C000067FC206008B1002070BD032070BD30B4B7
:101C10004880087820F00F00C01C20F0F0009030C1
:101C200001F8080B1DCA81E81D0030BC07F037BB66
:101C30002DE9FF4784B00027824602970798904617
:101C4000894612300AF012F8401D20F0030607986A
:101C500028B907A95046FFF7C2FF002853D1B9F1B0
:101C6000000F05D00798017B19BB052504681BE010
:101C700098F80000092803D00D2812D0FFDF45E0B6
:101C8000079903254868B0B3497B42887143914264
:101C900038D98AB2B3B2011D0EF08BFA0446078020
:101CA00002E0079C042508340CB1208810B1032DF4
:101CB00028D02BE00798012112300AF009F8ADF87E
:101CC0000C00024602AB2946504608F02AF90700EC
:101CD00001D1A01C029007983A461230C8F80400BF
:101CE000A8F802A003A94046029B09F0FEFFC0B17C
:101CF000072814D200E005E0DFE800F00608111123
:101D00000F0A0C00132015E6002013E6112011E63F
:101D100008200FE643F203000CE607200AE6032042
:101D200008E6BDF80C002346CDE900702A4650466F
:101D3000079900F019FD57B9032D08D10798B3B2E0
:101D4000417B406871438AB2011D0EF046FAB9F139
:101D5000000FD9D0079981F80C90D5E72DE9FE4FF7
:101D600091461A881C468A468046FAB102AB49461B
:101D700008F0D7F8050019D04046A61C27880EF0B9
:101D8000EBFC3246072629463B4600960EF0F7F854
:101D900020882346CDE900504A465146404600F08F
:101DA000E3FC002020800120BDE8FE8F0020FBE73F
:101DB00010B586B01C46AAB104238DF800301388F4
:101DC000ADF808305288ADF80A208A788DF80E20D8
:101DD0000988ADF80C1000236A462146FFF728FF5A
:101DE00006B010BD1020FBE770B50D4605210EF0C2
:101DF0006FFB040000D1FFDF294604F11200BDE8AB
:101E0000704009F04EBF2DE9F8430D46804600268C
:101E100007F042FA04462878102878D2DFE800F06C
:101E2000773B345331311231313108313131313175
:101E30002879001FC0B2022801D0102810D114BB8D
:101E4000FFDF35E004B9FFDF052140460EF040FB1F
:101E5000007B032806D004280BD0072828D0FFDFFA
:101E6000072655E02879801FC0B2022820D050B143
:101E7000F6E72879401FC0B2022819D0102817D0E1
:101E8000EEE704B9FFDF13E004B9FFDF287901288A
:101E90000ED1172137E0052140460EF019FB07004F
:101EA00000D1FFDF07F11201404609F0D7FE2CB147
:101EB0002A4621464046FFF7AAFE29E01321404664
:101EC00002F038FC24E004B9FFDF052140460EF0A3
:101ED000FFFA060000D1FFDF694606F1120009F0A3
:101EE000C7FE060000D0FFDFA988172901D21722FC
:101EF00000E00A46BDF80000824202D9014602E035
:101F000005E01729C5D3404600F03EFCD0E7FFDFCF
:101F10003046BDE8F883401D20F0030219B102FBF2
:101F200001F0001D00E000201044704713B5009838
:101F300050B100244FEA0D000EF0E5F8002C02D15C
:101F4000F74A009911601CBD01240020F4E72DE937
:101F5000F0470C4615462421204621F06CFD05B9BA
:101F6000FFDFA87860732888DFF8B4A3401D20F055
:101F70000301AF788946DAF800000EF0E2F80600B7
:101F800000D1FFDF4FF000082660A6F8008077B18F
:101F900009FB07F1091D0AD0DAF800000EF0D1F8AC
:101FA000060000D1FFDF6660C6F8008001E0C4F8DB
:101FB0000480298804F11200BDE8F04709F040BE12
:101FC0002DE9F047804601F112000D46814609F0E7
:101FD0004DFE401DD24F20F003026E7B144629684F
:101FE00038680EF0D9F83EB104FB06F2121D03D09A
:101FF000696838680EF0D0F805200EF011FA044632
:1020000005200EF015FA201A012802D138680EF0CA
:102010008DF849464046BDE8F04709F026BE70B548
:10202000054605210EF054FA040000D1FFDF04F14B
:1020300012012846BDE8704009F010BE2DE9F04FAE
:1020400091B04FF0000BADF834B0ADF804B0478854
:102050000C4605469246052138460EF039FA060030
:1020600000D1FFDF24B1A780A4F806B0A4F808B01F
:10207000297809220B20B2EB111F7DD12A7A04F1B5
:10208000100138274FF00C084FF001090391102A76
:1020900073D2DFE802F072F2F1F07F08D2888D9FF0
:1020A0003DDBF3EEB6B6307B022800D0FFDFA88917
:1020B00008EBC001ADF804103021ADF83410002C4D
:1020C00025D06081B5F80E9000271DE004EBC7080D
:1020D000317C88F80E10F189A8F80C10CDF800902A
:1020E0006888042304AA296900F02EFBBDF81010AB
:1020F000A8F8101009F10400BDF812107F1C1FFA97
:1021000080F9A8F81210BFB26089B842DED80DE19C
:10211000307B022800D0FFDFE98908EBC100ADF871
:1021200004003020ADF83400287B0A90001FC0B2B4
:102130000F90002CEBD06181B5F81090002725E0BE
:10214000CDF800906888696903AA0A9B00F0FCFA40
:102150000A9804EBC70848441FFA80F908F10C02FA
:1021600004A90F980FF0A8FD18B188F80EB0A8F8D0
:102170000CB0BDF80C1001E0D4E0CFE0A8F81010CE
:10218000BDF80E107F1CA8F81210BFB26089B842CB
:10219000D6D8CBE00DA8009001AB224629463046A8
:1021A000FFF71DFBC2E0307B082805D0FFDF03E00E
:1021B000307B082800D0FFDFE8891030ADF804003C
:1021C0003620ADF83400002C3FD0A9896181F18917
:1021D000A18127E0307B092800D0FFDFA88900F12A
:1021E0000C01ADF804103721ADF83410002C2CD0C0
:1021F0006081E8890090AB89688804F10C02296944
:1022000056E0E8893921103080B2ADF80400ADF80D
:102210003410002C74D0A9896181287A0E280AD044
:1022200002212173E989E181288A0090EB8968887D
:102230006969039A3CE00121F3E70DA8009001AB26
:10224000224629463046FFF75BFB6FE0307B0A28C9
:1022500000D0FFDF1220ADF80400ADF834704CB3AD
:10226000A9896181A4F810B0A4F80EB084F80C908C
:102270005CE020E002E031E039E042E0307B0B2816
:1022800000D0FFDF288AADF834701230ADF80400BA
:1022900084B104212173A9896181E989E181298AB5
:1022A0002182688A00902B8A688804F11202696989
:1022B00000F04AFA3AE0307B0C2800D0FFDF122011
:1022C000ADF80400ADF834703CB305212173A4F8D7
:1022D0000AB0A4F80EB0A4F810B027E00DA8009042
:1022E00001AB224629463046FFF75EFA1EE00DA8F4
:1022F000009001AB224629463046FFF7B8FB15E0B7
:1023000036E03B21ADF80400ADF8341084B3A4F8F6
:102310000690A4F808B084F80AB007E0FFDF05E0F3
:1023200010000020297A012919D0FFDFBDF8040030
:10233000AAF800007CB1BDF834002080BDF804008C
:102340006080BDF83400392805D03B2803D03C28F4
:1023500001D086F80CB011B00020BDE8F08F3C2110
:10236000ADF80400ADF8341014B1697AA172DDE75C
:10237000FFE7AAF80000EEE72DE9F84356880F467C
:1023800080461546052130460EF0A2F8040000D123
:10239000FFDF123400943B46414630466A6809F03C
:1023A000D6FDB6E570B50D4605210EF091F8040096
:1023B00000D1FFDF294604F11200BDE8704009F0AA
:1023C00062BC70B50D4605210EF082F8040000D104
:1023D000FFDF294604F11200BDE8704009F080BC1F
:1023E00070B5054605210EF073F8040000D1FFDF3B
:1023F00004F1080321462846BDE870400422ADE4FC
:1024000070B5054605210EF063F8040000D1FFDF2A
:10241000214628462368BDE8704005229EE470B539
:10242000064605210EF054F8040000D1FFDF04F148
:10243000120009F01BFC401D20F0030511E0011DF6
:1024400000880322431821463046FFF787FC002806
:102450000BD0607BABB2684382B26068011D0DF0A7
:10246000F2FE606841880029E9D170BD70B50E4662
:10247000054606F011FF040000D1FFDF01202072A5
:1024800066726580207820F00F00C01C20F0F000FC
:1024900030302070BDE8704006F001BF2DE9F043F8
:1024A0008BB00D461446814606A9FFF798FB00281D
:1024B00014D14FF6FF7601274FF420588CB103203A
:1024C0008DF800001020ADF8100007A8059007AAAD
:1024D000204604A90FF00FFC78B107200BB0BDE82F
:1024E000F0830820ADF808508DF80E708DF80000CC
:1024F000ADF80A60ADF80C800CE00698A178017484
:102500002188C1818DF80E70ADF80850ADF80C80AF
:10251000ADF80A606A4602214846069BFFF788FB31
:10252000DCE708B501228DF8022042F60202ADF880
:1025300000200A4603236946FFF73AFC08BD08B5A8
:1025400001228DF8022042F60302ADF800200A466F
:1025500004236946FFF72CFC08BD00B587B079B1AC
:1025600002228DF800200A88ADF808204988ADF8CD
:102570000A1000236A460521FFF75AFB07B000BD89
:102580001020FBE709B1072312E40720704770B55C
:1025900088B00D461446064606A9FFF720FB002822
:1025A0000ED17CB10620ADF808508DF80000ADF8D2
:1025B0000A40069B6A460821DC813046FFF738FB5B
:1025C00008B070BD05208DF80000ADF80850F0E7A8
:1025D00000B587B059B107238DF80030ADF8082059
:1025E000039100236A460921FFF722FBC6E710206A
:1025F000C4E770B588B00C460646002506A9FFF76B
:10260000EEFA0028DCD106980121123009F060FBB7
:102610009CB12178062921D2DFE801F020050516BA
:102620000318801E80B2C01EE28880B20AB1A3687F
:102630001BB1824203D90C20C2E71020C0E7042955
:1026400004D0A08850B901E00620B9E7012913D0D1
:10265000022905D004291CD005292AD00720AFE77C
:1026600009208DF800006088ADF80800E088ADF81A
:102670000A00A068039023E00A208DF8000060881B
:10268000ADF80800E088ADF80A00A0680A250390BC
:1026900016E00B208DF800006088ADF80800A088D7
:1026A000ADF80A00E088ADF80C00A0680B25049096
:1026B00006E00C208DF8000060788DF808000C25ED
:1026C0006A4629463046069BFFF7B2FA78E700B51E
:1026D00087B00D228DF80020ADF8081000236A465F
:1026E0001946FFF7A5FA49E700B587B071B1022294
:1026F0008DF800200A88ADF808204988ADF80A1046
:1027000000236A460621FFF793FA37E7102035E7E2
:1027100070B586B0064601200D46ADF808108DF85C
:102720000000014600236A463046FFF781FA0400A4
:1027300008D12946304605F0E3FB0021304605F07C
:10274000FDFB204606B070BDF8B51C4615460E468A
:10275000069F0DF0EFFF2346FF1DBCB231462A460F
:1027600000940DF0D8FBF8BD30B41146DDE902420B
:102770003CB1032903D0002330BC08F05ABA01232E
:10278000FAE71A8030BC704770B50C460546FFF773
:102790002BFB2146284605F0C2FB2846BDE87040C9
:1027A000012105F0CBBB00004FF0E0224FF40041C7
:1027B0000020C2F88011204908702049900208606A
:1027C000704730B51C4D04462878A04218BF002C35
:1027D00002D0002818BFFFDF2878A04208BF30BD14
:1027E0002C701749154A0020ECB1164DDFF858C07F
:1027F000131F012C0DD0022C1CBFFFDF30BD086061
:1028000003200860CCF800504FF4000010601860FE
:1028100030BD086002200860CCF800504FF04070D6
:102820001060186030BD086008604FF06070106084
:1028300030BD00B5FFDF00BD1800002008F50140E5
:1028400000F500403803002014F5004070B50B205F
:1028500000F0B5F9082000F0B2F900210B2000F0DB
:10286000C4F90021082000F0C0F9EC4C0125656096
:10287000A5600020C4F84001C4F84401C4F8480130
:102880000B2000F0A7F9082000F0A4F90B2000F0BD
:102890008BF9256070BD10B50B2000F090F9082071
:1028A00000F08DF9DD48012141608160DC490A6852
:1028B000002AFCD10021C0F84011C0F84411C0F832
:1028C00048110B2000F086F9BDE81040082000F008
:1028D00081B910B50B2000F07DF9BDE8104008204B
:1028E00000F078B900B530B1012806D0022806D032
:1028F000FFDF002000BDCB4800BDCB4800BDCA486B
:10290000001D00BD70B5C9494FF000400860C84DBA
:10291000C00BC5F80803C74800240460C5F840414F
:102920000820C43500F04BF9C5F83C41C24804709A
:1029300070BD08B5B94A002128B1012811D002287C
:102940001CD0FFDF08BD4FF48030C2F80803C2F886
:102950004803B3483C300160C2F84011BDE808406C
:10296000D0E74FF40030C2F80803C2F84803AC487F
:1029700040300160C2F84411AB480CE04FF48020B5
:10298000C2F80803C2F84803A54844300160C2F801
:102990004811A548001D0068009008BD70B5164696
:1029A0000D460446022800D9FFDF00229B48012380
:1029B00004F110018B4000EB8401C1F8405526B1B1
:1029C000C1F84021C0F8043303E0C0F80833C1F86F
:1029D0004021C0F8443370BD2DE9F0411C46154636
:1029E00030B1012834D0022839D0FFDFBDE8F081B2
:1029F000891E002221F07F411046FFF7CFFF012CF6
:102A000024D000208C4E8A4F012470703C6189498B
:102A100000203C3908600220091D08608549042017
:102A20003039086083483D350560C7F8004208200A
:102A300000F0D0F82004C7F80403082000F0B4F830
:102A40007A49E007091F08603470CFE70120D9E711
:102A5000012B02D00022012005E00122FBE7012B1F
:102A600004D000220220BDE8F04197E70122F9E7F7
:102A70006B480068704770B500F0C7F8674C0546B2
:102A8000D4F840010026012809D1D4F80803C00376
:102A900005D54FF48030C4F80803C4F84061D4F879
:102AA000440101280CD1D4F80803800308D54FF461
:102AB0000030C4F80803C4F84461012010F0E0F8C5
:102AC000D4F8480101280CD1D4F80803400308D5F4
:102AD0004FF48020C4F80803C4F84861022010F0C5
:102AE000CFF85648056070BD70B500F08EF8524DB5
:102AF0000446287858B1FFF705FF687820B1002018
:102B000085F8010010F0BCF84C48046070BD03204B
:102B1000F8E74FF0E0214FF40010C1F800027047D1
:102B2000152000F057B8424901200861082000F044
:102B300051B83F494FF47C10C1F808030020024609
:102B400001EB8003C3F84025C3F84021401CC0B20C
:102B50000628F5D37047410A43F609525143C0F3A2
:102B6000080010FB02F000F5807001EB5020704768
:102B700010B5430B48F2376463431B0C5C020C60D6
:102B80002F4C03FB04002F4B4CF2F72443435B0D07
:102B900013FB04F404EB402000F580704012107029
:102BA00008681844086010BD00F01F020121914020
:102BB0004009800000F1E020C0F80011704700F0EB
:102BC0001F02012191404009800000F1E020C0F87F
:102BD0008011704700F01F020121914040098000E0
:102BE00000F1E020C0F8801270474907090E002864
:102BF00006DA00F00F0000F1E02080F8141D7047A5
:102C000000F1E02080F8001470470C48001F0068B5
:102C10000A4A0D49121D11607047000000B00040C3
:102C200004B500404081004044B1004008F5014037
:102C3000008000404085004038000020140502401C
:102C4000F7C2FFFF6F0C0100010000010A4810B538
:102C50000468094909480831086010F0A5F80648D9
:102C6000001D046010BD0649002008604FF0E021FF
:102C70000220C1F8800270471005024001000001E7
:102C8000FC1F004010B50D2000F06FF8C4B26FF0CB
:102C9000040000F06AF8C0B2844200D0FFDF3A4975
:102CA0000120086010BD70B50D2000F048F8374CC9
:102CB0000020C4F800010125C4F804530D2000F0E1
:102CC00049F825604FF0E0216014C1F8000170BDA3
:102CD00010B50D2000F033F82C480121416000218F
:102CE000C0F80011BDE810400D2000F033B82848AE
:102CF00010B5046826492748083108602349D1F8EF
:102D00000001012804D0FFDF2148001D046010BD30
:102D10001D48001D00680022C0B2C1F8002110F05B
:102D20001BFCF1E710B51948D0F800110029FBD0C1
:102D3000FFF7DDFFBDE810400D2000F00BB800F0FC
:102D40001F02012191404009800000F1E020C0F8FD
:102D50008011704700F01F0201219140400980005E
:102D600000F1E020C0F880127047002806DA00F079
:102D70000F0000F1E02090F8140D03E000F1E020D6
:102D800090F800044009704704D5004000D000408E
:102D9000100502400100000110B5202000F075F878
:102DA000202000F07DF84449202081F800044349A8
:102DB00000060860091D42480860FEF79EFA3F4978
:102DC000C83108603F48D0F8041341F00101C0F851
:102DD0000413D0F8041341F08071C0F8041336498D
:102DE00001201C39C1F8000110BD10B5202000F0F1
:102DF0004CF8324800210160001D01602F4A481E36
:102E0000E83A10602F4AC2F808032C4BC833196007
:102E1000C2F80001C2F860012B490860BDE810400B
:102E2000202000F03DB825492848EC39086070475B
:102E300022492648E8390860704770B51F4A806902
:102E4000E83A224911601F49D1F800610023204D62
:102E50001D4A5C1E1EB1A84206D300210FE0D1F826
:102E6000606186B1A84209D2C1F80031C1F8603171
:102E70001460BDE87040202000F012B81168BDE871
:102E8000704020F003BEFFDF70BD00F01F02012183
:102E900091404009800000F1E020C0F880117047A7
:102EA00000F01F02012191404009800000F1E02064
:102EB000C0F880127047000020E000E000060240E9
:102EC000C413002000000240000402400100000181
:102ED000005002004FF0E0214FF00070C1F8800177
:102EE000C1F88002384B802283F80024C1F8000129
:102EF000704700B502460420344903E001EBC003EB
:102F00001B792BB1401EC0B2F8D2FFDFFF2000BDFD
:102F100041F8302001EBC00100224A718A71012280
:102F20000A7100BD294A002102EBC00001717047FF
:102F300010B50446042800D3FFDF244800EBC40486
:102F40002079012800D0FFDF6079A179401CC0B250
:102F5000814200D060714FF0E0214FF00070C1F865
:102F6000000210BD2DE9F0411948056818491948BB
:102F7000083108601448042690F80004134F4009F3
:102F8000154C042818D0FFDF16E0217807EBC100AC
:102F90000279012A08D1427983799A4204D0427990
:102FA000827157F8310080472078401CC0B22070F1
:102FB000042801D300202070761EF6B2E5D2044822
:102FC000001D0560BDE8F08119E000E074060020F6
:102FD00010050240010000015000002070B50C46B1
:102FE000054609F051F921462846BDE870400AF02F
:102FF00034BA704770477047704770477047000099
:103000002CFFFFFFDBE5B15100500200FEFFFFFF88
:103010008C000000808D5B0086FA71F377B11C5242
:103020008E1A95B8DDF423C04F8DD92A30B5F94DED
:10303000044610280AD0112C06D02846122CC1783C
:1030400006D0132C08D0FFDFEC7030BDFFDFFBE7AC
:103050001129F9D0FFDFF7E71129F5D0FFDFF3E7FA
:1030600070B50EF0B3FF044610F04CF9201AC4B24C
:1030700006200DF0D5F9054606200DF0D9F92E1AD7
:1030800007200DF0CDF9054607200DF0D1F9E149F3
:10309000281A3218C87812280DD000231A44132891
:1030A0000BD0002002440878022808D000201044E9
:1030B000201AC0B270BD0123F0E70120F2E7012021
:1030C000F5E7D44810B5817900F10700490805D02B
:1030D0000BF0AAF9BDE8104005F014BF0BF07DF924
:1030E000F8E702210DF0F4B92DE9FC411D469046A8
:1030F0000E460746FFF7F5FF04000AD02078222885
:1031000004D3A07FC0F34010A84205D10820BDE839
:10311000FC8143F20200FAE7ADF800703DB10120F6
:103120008DF802008DF803608DF8048002E0002025
:103130008DF8020068460CF0A5FAA07F65F34510F3
:10314000A0770020E3E730B50446A1F120000D464A
:103150000A284AD2DFE800F005070C1C2328353A7C
:103160003F44FFDF42E0207820283FD1FFDF3DE0F1
:10317000A8480178032939D0C078132836D02078A0
:10318000242833D0252831D023282FD0FFDF2DE06D
:10319000207822282AD0232828D8FFDF26E020788C
:1031A000222823D0FFDF21E0207822281ED02428E7
:1031B0001CD026281AD0272818D0292816D0FFDF9F
:1031C00014E02078252811D0FFDF0FE02078252893
:1031D0000CD0FFDF0AE02078252807D0FFDF05E0CC
:1031E0002078282802D0FFDF00E0FFDF257030BD07
:1031F00030B50B8840F67B444FF6FF72022801D0B1
:10320000934204D09D1FA54224D2022802D04D88AB
:10321000954203D04D88AD1FA5421BD24C88A342D6
:1032200018D88B88B3F5FA7F14D2022802D0C88848
:10323000904205D0C88840F677450A38A84209D29E
:10324000C888904208D0944206D05B1C6343B3EB1D
:10325000800F01DB072030BD002030BD70B5144663
:103260000D46064610F082FC58B90DB1A54201D9B1
:103270000C2070BD002408E056F8240010F076FC05
:1032800008B1102070BD641CE4B2AC42F4D300203D
:1032900070BD2DE9F0411F4690460E4605004FF0E7
:1032A000000465D010F0AFFC18B9286810F0ABFC32
:1032B00010B11020BDE8F08128680028A88802D04D
:1032C000B84202D84FE00028F4D00920F2E729687C
:1032D000085DB0B1671CCA5D152A2DD03BDC3AD21F
:1032E000DFE802F03912222228282A2A313139391E
:1032F00039393939393939392200085D30BB641C14
:10330000E4B2A242F9D833E00228DED1A01C085C66
:1033100088F80000072801D2400701D40A20C9E735
:10332000307840F0010015E0C143C90707E00128EB
:1033300007D010E00620BDE70107A1F18051002968
:10334000F5D01846B6E73078810701D50B20B1E7F4
:1033500040F0020030702868005D3844C4B2A8888C
:10336000A04202D2B1E74FF4485382B2A242AED893
:1033700000209FE710B50278540809D0012243F2DB
:103380000223012C07D0022C0DD0032C13D10FE007
:103390000020087005E080790324B4EB901F0AD167
:1033A0000A70002010BD8079B2EB901F03D1F7E7BF
:1033B00080798009F4D0184610BD164A117C39B1C5
:1033C000517C022908D0032908D043F2022070471B
:1033D0000146901D01F09ABC032100E0012101701B
:1033E0000020704738B50C460546694601F08EFC52
:1033F00000280DD19DF80010207861F3470020705F
:1034000055F8010FC4F80100A888A4F805000020B1
:1034100038BD0000D001002038B51378C0B10228B3
:1034200016D0FEA46D46246800944C7905EB9414E4
:10343000247864F34703137003280ED003F0FE00D2
:1034400010700868C2F801008888A2F80500DFE75C
:1034500023F0FE0313700228EED1D8B240F0010031
:10346000EEE738B50C460978222901D20820CFE7CB
:10347000ADF800008DF8022068460BF01CF805F04E
:1034800041FD050003D121212046FFF75CFE2846BF
:10349000BEE71FB5ADF800001088ADF802005088F7
:1034A000ADF80400D088ADF808009088ADF80600AB
:1034B0000020ADF80A00ADF80C0068460BF0CCFD1A
:1034C00005F020FD04B010BD1CB500208DF80000F3
:1034D000CDF80100ADF80500D148007C022801D0EC
:1034E000012000E000208DF8070068460BF037F956
:1034F000002800D0FFDF1CBD2DE9FF470220C84E89
:103500008DF804000027B08AADF80600B84643F2F3
:1035100002094DE001A80CF042FF050006D0B08A78
:10352000A8B3A6F81480ADF806803FE0039CA07F06
:1035300001072DD504F124000090A28EBDF80800EB
:10354000214604F1360301F0B6FD050005D04D45D6
:103550002BD0112D3DD0FFDF3BE0A07F20F00800F5
:10356000A077E07F810861F30000C10861F34100AA
:10357000E07794F8210000F01F0084F82000207804
:10358000282827D129212046FFF7DDFD22E015E07C
:1035900040070BD5BDF80800214604F10E02FFF7E5
:1035A00078FF05000DD04D4510D100257F1CFFB2DE
:1035B00002200CF035FF401CB842ABD8052D12D0CC
:1035C00008E0A07F20F00400A07703E0112D00D0D8
:1035D000FFDF0025BDF80600B082052D05D0284686
:1035E00004B0BDE8F087A6F814800020F8E770B5B5
:1035F0000646FFF776FD054605F04EFE040000D1B5
:10360000FFDF6680207820F00F00801C20F0F000A3
:10361000203020700620207295F83E006072BDE8D0
:10362000704005F03CBE2DE9F04786B0040000D1A3
:10363000FFDF20787A4E20F00F00801C20F0F00091
:103640007030207060680178091F1A2932D2DFE8D3
:1036500001F00DEC31313154EB310DEBEB41EC313C
:10366000310D77ECEC313131ECECEAE9868830460B
:10367000FFF737FD0546304607F0D9F9E0B160683D
:10368000807985F83E0021212846FFF75CFD304611
:10369000FEF7C5FC304603F057FF3146022010F01C
:1036A00019FAA87F20F01000A877FFF725FF00285F
:1036B00000D0FFDF06B094E7207820F0F000203043
:1036C000207006202072668060688079607205F044
:1036D000E6FDD8E785882846FFF703FD00B9FFDF40
:1036E00060688078012800D0FFDF6068817906B0CB
:1036F0002846BDE8F04707F077BD86883046FFF7DB
:10370000F0FC050000D1FFDF05F0C9FD606831461F
:10371000C088288160680089688160684089A881C4
:10372000022010F0D7F90020A875A87F00F0030050
:103730000228BFD1FFF7E0FE0028BBD0FFDFB9E7CA
:1037400080783C2803D0002502280AD000E001251B
:10375000002720B13C2802D0022800D0FFDF17B19B
:10376000B7E00127F5E705F09AFD1DB1B07801F04B
:1037700092FAA0E06568B5F804A0A879AD1C01280C
:1037800006D03079814605F02FFB070003D101E018
:10379000B078F7E7FFDF0022022150460CF08FFEE1
:1037A000040000D1FFDF22212046FFF7CCFC28795E
:1037B000012800D00220A17F804668F30101A17793
:1037C000288B2081688B6081A88BA08184F822904F
:1037D0008DF80880B8680090F86801906A46032167
:1037E00050460CF06CFE00B9FFDFB888ADF8100051
:1037F000B8788DF8120004AA052150460CF05FFE3F
:1038000000B9FFDFB888ADF80C00F8788DF80E002D
:1038100003AA042150460CF052FE07E00302FF0108
:10382000D00100206FE068E061E073E000B9FFDFE5
:10383000062105F1120001F094FA00B368798007BF
:1038400000D5FFDF6979E07D61F34700E075D5F8C9
:103850000600A0616889A083062105F10C0001F033
:1038600080FAB0B1B0794108607861F347006070C8
:10387000D6F80700C4F80200B6F80B0012E0E07DAD
:1038800020F0FE00801CE075D5F81200A061E88AE7
:10389000E1E7607820F0FE00801C6070E868C4F802
:1038A0000200288AE080B8F1010F04D0B8F1020FBD
:1038B0000FD0FFDFFEE63078032800D0FFDF0021C5
:1038C000084610F007F906B00120BDE8F04701F006
:1038D000B1B9F078132800D0FFDF0021062010F0E6
:1038E000F9F806B01120BDE8F047FFF79FBB06B01E
:1038F0002046BDE8F04701F089BE05F0D0FCB07C61
:1039000040F0020004E005F0CAFCB07C40F0040086
:10391000B074CFE606B0BDE8F04705F0C0BC2DE9B5
:10392000F04705460078914600270209F7480C4603
:103930003E46012A6CD000234FF6FF71022A68D060
:10394000072A0AD00A2A70D0FFDF00BFA9F800605A
:103950000CB127806680002043E6D5F804C09CF8AF
:103960000020162A7ED00CDC102A21D004DC052A87
:103970005CD0092A59D10DE0142A22D0152AF9D198
:10398000CCE01A2A0BD01B2A6DD01C2A6CD01D2A21
:10399000F0D19DE012271026BCF8040006E11C2798
:1039A0000926A4B3BCF80200A080686800794CE145
:1039B0001B2709265CB30320207268684088A0801A
:1039C000C4E79CF802003C2829D0102718260CF1E7
:1039D000020CE4B1BCF80200A080BCF818006082C0
:1039E000BCF818002082BCF81A00A082BCF81C00A9
:1039F000E0829CF8050004F108020CF10601FFF7D3
:103A00000BFD9CF8040028B10120E0739EE703E061
:103A1000AFE0CFE00220F8E7A9F800609BE71B27A2
:103A20000926002CF8D0237290E710E11D274026CC
:103A3000002CF1D0A180696804F10A02081DCB783E
:103A400001461846FFF7E8FC68681F22C07A6077D5
:103A50006868808920816868807AE07704F12000B6
:103A6000696802E045E021E06CE01C311FF042FF94
:103A7000696804F1110201F115000B7D0146184639
:103A8000FFF7CAFC6868807B01F07AF920766868E5
:103A9000C07B01F075F960766868408A6083686869
:103AA000007CA0776868C07E20774FE7202710262B
:103AB000002CB1D0A180686804F10902807A2072DC
:103AC0006968081DCB7801461846FFF7A5FC3DE75D
:103AD00021270A26002C9FD0BCF80210A18069681B
:103AE00009792172696849796172817C21F0040148
:103AF00057E022270B26002C8ED0BCF80400A080B3
:103B00006868807820726868807901F039F960729D
:103B10006868C07901F034F9A07217E724271026ED
:103B2000002C86D0BCF80200A08068680079208153
:103B30006868007A60816868C088A0816868408988
:103B4000E08103E723271026002CB2D0BCF8021036
:103B5000A1806968898821816968C98861816968EB
:103B60000989A18169684989E181817C21F002018B
:103B700017E0297A012903D0022914D0FFDFE5E6F6
:103B80001F271026002C94D06988A180A989218143
:103B9000E9896181298AA181698AE181817C21F099
:103BA00001018174D2E6122768881026214601F0AF
:103BB000C5F8CBE6287A072850D2DFE800F0373D79
:103BC0003D484848040011270926002C94D0B5F838
:103BD00002804046FFF785FA90F822A0A4F80480FE
:103BE000687A2072042140460CF084FC052140468E
:103BF0000CF080FC002140460CF07CFC012140468A
:103C00000CF078FC032140460CF074FC0221404685
:103C10000CF070FC062140460CF06CFC072140467D
:103C20000CF068FC504601F036F88FE61B27092699
:103C3000002C8AD0A180F6E61B270926002C84D010
:103C4000A180287A012800D0022020727EE64A4610
:103C500021462846BDE8F04701F05EBEFFDF75E66D
:103C600070B52A4DE878132801D0082070BD0BF0FC
:103C7000CAF905F047F9040002D1287901F00BF8E0
:103C8000002106200FF026FF204670BD1CB51F48FE
:103C9000C078122801D008201CBD00208DF800003B
:103CA00068460AF0EDFE05F02DF90028F4D1002158
:103CB00006200FF00FFF1120FFF7B8F900201CBD00
:103CC0001CB5124C2178012916D000218DF8001066
:103CD00001218DF801108DF8020068460BF06DFC93
:103CE00005F010F9002808D1002108460FF0F2FE77
:103CF0002078032802D004E008201CBDA07800F042
:103D0000CAFF012000F096FF00201CBDD00100205A
:103D100070B5002538B1022818D0062837D00728FA
:103D200000D0FFDF70BD0020FFF7CAFF0028F9D1E7
:103D300005F0B2FA0028F5D0017821F00F01891CB6
:103D400021F0F0012031017005723FE08EB2304663
:103D5000FFF7C7F9040000D1FFDF20782128E1D068
:103D600005F09AFA60B1017821F00F01891C21F069
:103D7000F00110310170022101724680A57525E025
:103D800021463046BDE870401322FFF76ABBFE486B
:103D9000C478122C03D0132C04D0FFDF70BDFFF7C2
:103DA00075FF01E0FFF75CFF0028F7D105F074FA1A
:103DB0000028F3D0017821F00F01891C21F0F001D7
:103DC00020310170122C05D002210172BDE8704033
:103DD00005F065BA0121F8E72DE9F04116460C001F
:103DE000804600D1FFDF307820F00F00801C20F0EB
:103DF000F000103030702078012804D0022817D04D
:103E0000FFDFBDE8F0814046FFF76BF9050000D108
:103E1000FFDF0320A87505F042FA94E80F0008368A
:103E200086E80F00D848817C41F001018174E8E701
:103E30004046FFF756F9050000D1FFDFA1884FF695
:103E4000FF700027814202D1E288824203D0814282
:103E500001D1E08840B105F022FA94E80F0008365D
:103E600086E80F00AF75CCE7A87D0128C9D178237B
:103E70000022414602200FF083FD0220A875C0E712
:103E800038B505460C4608460FF070FE20BB203DB5
:103E9000072D51D2DFE805F0041C383D43493100BD
:103EA000002107200FF0ECFD08B1112038BDA01C47
:103EB0000BF03EF905F026F805003ED1002208235C
:103EC000114607200FF05CFD072836D0FFDF34E0F5
:103ED00060680FF08FFE08B1102038BD618820881F
:103EE0006A460BF01DFC05F00DF8050025D1606851
:103EF00018B3BDF8001001801FE0A07800F00101A8
:103F000020880BF043FC14E0206801F0A3FF054675
:103F100013E0207800F001000BF0B4FC09E02078F9
:103F200000F001000AF04CFA03E0618820880BF0F1
:103F300086FB04F0E7FFEAE70725284638BD70B5A1
:103F400005460C4608460FF037FE08B1102070BD3C
:103F5000203D072D1BD2DFE805F0041818181A1AA7
:103F600018002088FFF7BDF820B10078222804D27D
:103F7000082070BD43F2020070BD2088A11C0AF029
:103F800016FBBDE8704004F0BDBF062070BD0720E1
:103F900070BD7D48801D704738B516217A481FF0E6
:103FA00028FD012000F046FE1120FFF73FF8764C77
:103FB0006846E11D05F006F99DF80010A07961F34F
:103FC000470020F00100A071002020744FF46170C0
:103FD000E08102206074FFF774F800B1FFDFFDF7A5
:103FE000B3F901F0D0FA38BD10B50C464021204697
:103FF0001FF0FFFCA07F20F00300A077202020709E
:104000000020A07584F8230010BD70477CB50546DC
:104010000FF0ACFD08B110207CBD5B4CA11DD4F8A5
:1040200006000090D4F80A0001902846FFF7DAF95C
:104030000028F1D1FFF745F80028EDD00099C4F829
:104040000610BDF8041061819DF8061021737CBD37
:1040500010B504460FF0B0FD08B1102010BD4A495C
:1040600022468879C91D4008FFF7D6F9002010BD07
:10407000FEB50D4604004FF0000712D00822FFF7EE
:10408000EDF8002812D1002609E000BF54F8260000
:104090006946FFF76FF9002808D1761CF6B2AE42E8
:1040A000F4D30AF091F810B143F20320FEBD364E6E
:1040B0007771FCB100271AE054F8270002A9FFF736
:1040C00059F900B1FFDF9DF808008DF8000054F8A1
:1040D000270050F8011FCDF801108088ADF80500C9
:1040E00068460AF0BBF800B1FFDF7F1CFFB2AF42A9
:1040F000E2D375710020FEBD2DE9F0478AB0154668
:10410000894604001DD00F4608222946FFF7A6F86D
:10411000002810D1002612E054F82600694610301D
:1041200000F0F4FD002806D13FB157F826000FF04B
:104130001DFD10B110200AB00EE4761CF6B2AE429E
:10414000EAD30026A5F101081CE000BF06F1010A30
:104150000AF0FF0712E000BF54F82600017C4A086D
:1041600054F827100B7CB2EB530F05D10622113007
:1041700011311FF093FB70B17F1CFFB2AF42EBD344
:104180000AF0FF06464501E0D0010020DEDB4E4686
:1041900024B1012003E043F20520CCE700200AF01F
:1041A0008EF810B90AF09FF810B143F20420C2E76C
:1041B00064B300270DF1170826E000BF54F827006C
:1041C0006946103000F0A2FD00B1FFDF54F827006F
:1041D000102250F8111FCDF801108088ADF80500AD
:1041E00054F827100DF107001FF084FB96B156F824
:1041F0002710102240461FF07DFB684609F0FCFFA7
:1042000000B1FFDF7F1CFFB2AF42D7D3FFF75CF9ED
:10421000002090E7404601F011FEEEE730B585B092
:1042200004460FF0A3FC18B960680FF0ECFC10B165
:10423000102005B030BD60884AF2B811884206D817
:104240002078F94D28B1012806D0022804D0072093
:10425000EFE7FEF736FF17E06078022804D0032866
:1042600002D043F20220E4E76874C1B2002000905B
:10427000ADF8040002292BD0032926D0FFDF6846C1
:104280000AF0D2F804F03EFE0028D2D1606801F0B6
:10429000C8FD207858B101208DF800000DF1010013
:1042A00001F0CCFD68460BF0CFFA00B1FFDF2078BB
:1042B0002874FFF709F9608860B1E88180B209F0DD
:1042C000F6FF00B1FFDF0020B3E78DF80500D6E769
:1042D0004020FAE74FF46170EFE710B504460FF0A5
:1042E0006BFC20B9606838B10FF084FC08B1102075
:1042F00010BD606801F0A2FDCB48C1896180417C9E
:104300006170007C2070002010BD30B58FB000209F
:1043100015468DF830008DF82C008DF828008DF8AA
:1043200034000C4651EA050016D01F230AAA0CA936
:104330002046FEF7AEFF00280CD11F230DAA0BA9C3
:104340002846FEF7A6FF002804D19DF82C00C007E0
:1043500004D00A200FB030BD0720FBE7ACB103202A
:104360008DF8010001208DF80200A088ADF804004E
:10437000A2880DF1060021681FF0BCFA68460AF019
:10438000EBFF04F0BFFD0028E4D13DB12879296896
:104390000AF0FDFF04F0B6FD0028DBD1A2499DF82C
:1043A000280048700020D5E72DE9F0478EB0804600
:1043B0004FF000099DA00C468DF81C90D0E900102C
:1043C000CDE90810924620460FF0D0FB88B920793D
:1043D000400703D520680FF0C9FB50B9924D012763
:1043E000287C50B1687C022807D120680FF00BFCB4
:1043F00018B110200EB0BDE8F0872878012801D050
:104400000820F7E707200CF013F820B92079C0073F
:1044100001D01220EEE7FEF723FE18B1A088C109F3
:104420007ED101E01320E5E7A168824BA1F12002D3
:104430009A4206D3020773D5002971D1A1890029B8
:104440006ED169784FEA4070C90709D0002810DBA7
:10445000A089002864D044F25061884260D801E00D
:10446000002806DB287C50B1687C022807D1206830
:1044700028B107A92068FEF77DFF0028BAD1207C6B
:1044800030B1012806D0022806D0032848D105E023
:10449000002604E0012602E0022600E00326A088B0
:1044A000C10701D181071DD5410712D48EB16979A9
:1044B000002935D06978890702D043F2012099E7B5
:1044C000810706D5C00706D1022E29D0032E27D09A
:1044D00008E0C00706D0504600F0C0FB002889D194
:1044E00085F802A08DF80080A088ADF80200A068D1
:1044F0000190A06802900DF10D00FEF75EFF00B183
:10450000FFDF9DF81C008DF80E002079400706D4CF
:10451000287C68B1687C02280AD1206840B100E09C
:1045200059E0206850F8011FCDF80F10808802E094
:104530004846CDF80F90ADF813008DF81560E07B7C
:10454000C0F34002014662F35F01C0F3800041EA1C
:10455000800008A9085C8DF80C00E0B37F208DF87E
:104560001600E07C8DF81800207D032100F07F000C
:104570008DF81A00207DC0098DF81B00627C072091
:10458000012A39D0022A9AD0042A98D18DF817101E
:104590002079C00609D4A27C0720012A2FD0022A44
:1045A00030D0042A8BD18DF819100CA968460AF076
:1045B000BAFE04F0A7FC002891D18DF828708DF880
:1045C00029708DF82A80A089ADF82C00A07B8DF889
:1045D0002E000AA800E00DE00AF0EFFF04F092FCC4
:1045E0000028D2D12079C00710D0A87800F046FB6F
:1045F00003200CE00720FDE68DF81770C8E78DF862
:104600001970D2E702208DF81900CEE7022000F0E1
:1046100011FB2079000719D4A089B8B164280BD305
:104620006421B0FBF1F008E0D0010020070605048A
:1046300003020100E0FFFF00012000228300114679
:1046400010460FF09DF908B10320D3E60020D1E613
:104650002DE9FC4107460D46032608460FF0D3FA24
:10466000002865D13846FEF73CFD040005D02078CF
:10467000222805D20820BDE8FC8143F20200FAE7B7
:10468000A07F00F0030C2DB129466046FEF7B0FD77
:104690000600F0D1BCF1010F05D0BCF1020F18D01B
:1046A000FFDF3046E7E7A07D2946022801D011B19F
:1046B00007E01120DFE76846FCF754FF0028DAD155
:1046C0006946384606F053FD0600EAD10120A07580
:1046D000E7E7A07D032803D1F748807CC00701D01D
:1046E00035B30EE025B1A07F40071FD4002100E0C4
:1046F0000121384606F05BFD0600D2D1A075002DE1
:10470000CFD02A4621463846FEF7C3FE064611287A
:10471000C7D1A07F4107C4D4296844F80E1F696837
:10472000616040F0040020740026BAE71126B8E763
:104730001020A0E770B50C460546FEF7D2FC01003C
:1047400005D022462846BDE87040FEF78ABE43F2F7
:10475000020070BD10B509F0EDFDBDE8104004F099
:10476000D1BB0123FEF7C0BC00231A461946FEF751
:10477000BBBC30B587B004460FF0F8F910B110207B
:1047800007B030BD204600F0B5FA0028F8D1CA4D78
:10479000E878112801D00820F2E7FEF761FC38B173
:1047A0002078C0F34100012804D0032802D003E0A0
:1047B0001320E5E76879E8B36846FEF7FEFD00B12F
:1047C000FFDF20780125C0F341008DF801006178FA
:1047D000072001293AD00229D2D00429D0D10420BF
:1047E0008DF80200207800F001008DF80300608849
:1047F000ADF80600A088ADF80A0068460AF09FF8F8
:1048000004F080FB0028BBD18DF810508DF811000A
:10481000ADF812002089ADF8140004A80AF030F9B0
:1048200004F070FB0028ABD1E088642811D280B17D
:10483000012000E008E000F073FA0400A0D112208B
:10484000FEF7F4FB20469BE7072099E78DF802501E
:10485000C8E76421B0FBF1F0EBE72DE9F047964E95
:10486000074690B0F0789A4615460C46122803D1B8
:10487000FFF70CFA002816D120460FF077F9E8BBB5
:1048800028460FF073F9C8BB204600F033FA002821
:1048900009D129460220FEF7ABFC002803D1F078AD
:1048A000112802D0082010B0A5E506200BF0C0FDAD
:1048B00038B12078C0F34100012804D0032802D089
:1048C00003E01220EFE7707928B1FEF7C9FB022858
:1048D00003D21320E7E70720E5E720784FF001092E
:1048E000C0F341008DF8000061780720012915D040
:1048F0000229D8D00429D6D1042000E015E08DF893
:1049000009006088ADF80A00A088ADF81000207892
:104910004FF000084008C00703D020E08DF8099050
:10492000EFE738460FF022F908B11020BBE73878DE
:10493000400808D0012809D0022807D0032805D054
:1049400043F20220AFE78DF8028001E08DF802907B
:1049500057F8010FCDF80300B888ADF807000DF146
:104960000100FEF72AFD08B103209CE72888ADF876
:1049700016006888ADF81C00A888ADF82200E88809
:10498000ADF82800ADF82E80ADF83480504600F028
:1049900065F9002887D186F804A068460AF030FB44
:1049A00004F0B0FA00288DD1307900F067F9E08882
:1049B00064280AD248B1012000F0B2F9040089D17C
:1049C0001320FEF733FB20466DE76421B0FBF1F0C6
:1049D000F2E770B505460C4608460FF0EDF808B151
:1049E000102070BD2846FEF77CFB38B101782229E3
:1049F00002D3807F800604D4082070BD43F20200F9
:104A000070BD214628460AF072FEBDE8704004F0F1
:104A100079BA38B505460C4608460FF0A7F808B134
:104A2000102038BD2846FEF75CFB20B10078222814
:104A300004D2082038BD43F2020038BD1E48807CF5
:104A4000400701D5112038BD2078C00802D1607818
:104A5000C00801D0072038BDADF8005020788DF88F
:104A6000020060788DF80300684609F05EFF04F0EC
:104A700049FA38BD2DE9F0418EB014460D46064680
:104A8000FEF72FFB070006D03878222806D2082030
:104A90000EB0BDE8F08143F20200F9E728460FF0BE
:104AA000B2F830B94FF0000864B120460FF0A2F818
:104AB00020B11020ECE70000D0010020C4F80080F5
:104AC000A4F80480B648807C800701D51120DFE778
:104AD00097F8220004F088F98088011DFB2901D293
:104AE000001D00E0FB20C0B26A46294600F0DDF858
:104AF000ADF81060BDF80200ADF81200BDF8060078
:104B0000ADF81400BDF80000ADF81600BDF80400C3
:104B1000ADF8180007A904A809F0C9FD00B1FFDF2E
:104B2000BDF81E00ADF80800BDF82000ADF80A0081
:104B3000BDF82200BDF82410BDF800200844ADF8EF
:104B40000C0007201B2AA3D3BDF802101B299FD3FA
:104B5000FB2A9DD8FB299BD806278A4210D1012128
:104B6000104600F056F8BDF80410884208D1BDF890
:104B70000200012100F04DF8BDF80610884201D076
:104B8000384685E7BDF8080028B9BDF80A1011B904
:104B9000BDF80C1029B35DB1298849B1698839B1D4
:104BA00024B102982060BDF80C00A08013206FE7AC
:104BB000BDF80010BDF80A20081A80B2ADF8000058
:104BC000BDF80210891AADF80210012100F021F899
:104BD000ADF80400BDF80200012100F01AF8ADF8AC
:104BE0000600ADF82860BDF80200ADF82A00BDF857
:104BF0000600ADF82C00BDF80000ADF82E00BDF8A1
:104C00000400ADF830000AA809F0F0FC04F07AF9CD
:104C10003EE711F00C0F04D04FF4747101EB8010DB
:104C200006E0022902D0C000703001E080003C3074
:104C300080B2704730B55A4D040008D0012C04D022
:104C4000022C06D0032C04D0FFDF2C7030BDFFDF18
:104C5000FBE728780128F8D0FFDFF6E710B5044617
:104C600004F0C2F830B1407830B1204604F0BBFB0C
:104C7000002010BD072010BD122010BD10B504F09B
:104C8000B3F8040000D1FFDF607800B9FFDF60787F
:104C9000401E607010BD10B504F0A6F8040000D1ED
:104CA000FFDF6078401C607010BD10B5144631B154
:104CB0000A68226049686160218839B107E0208074
:104CC00060800121FFF7A5FFA0800DE020806188B2
:104CD00001B96080A08820B920880121FFF799FFE1
:104CE000A080E088002804D160880121FFF791FFAF
:104CF000E08010BD4188042906D38088042803D3AE
:104D0000884201D800207047072070470278520877
:104D100004D0012A02D043F202207047FEF72ABBDA
:104D200010B548B183000022114606200EF028FE7F
:104D3000062801D0032010BD002010BD70B50C0066
:104D400006460DD0FEF7CDF9050000D1FFDFA680A5
:104D500028892081288960816889A081A889E081CB
:104D600070BD10B500231A4603E0845C2343521C37
:104D7000D2B28A42F9D30BB1002010BD012010BD80
:104D800000B540B1012805D0022803D0032804D083
:104D9000FFDF002000BDFF2000BD042000BD00009B
:104DA000D001002010B504460EF0E0FE08B110203E
:104DB00010BD2078C0F30210042807D860780728B7
:104DC00004D3A178102901D8814201D2072010BD57
:104DD000E078410706D421794A0703D4000701D4BB
:104DE000080701D5062010BD002010BD10B51378AE
:104DF0005C08C37F64F30003C3771478A40864F3EA
:104E00004103C3771078C309487863F341004870C1
:104E100013781C090B7864F347130B701378DB08C5
:104E200063F3000048705078487110BD10B5C47825
:104E30000B7864F300030B70C478640864F34103D7
:104E40000B70C478A40864F382030B70C478E40880
:104E500064F3C3030B700379117863F300011170DD
:104E600003795B0863F34101117003799B0863F3D5
:104E7000820111700079C00860F3C301117010BD88
:104E800070B514460D46064604F006FA80B1017866
:104E9000182221F00F01891C21F0F001A03100F847
:104EA000081B21461EF06BFDBDE8704004F0F7B909
:104EB00029463046BDE870401322FEF7D2BA10B53D
:104EC000FE4C94F8300000280CD104F120014FF67C
:104ED000FF72A1F110000CF075FE00B1FFDF0120A0
:104EE00084F8300010BD2DE9F047064608A8894631
:104EF00090E830041F469046142128461EF09BFD82
:104F00000021CAF80010B8F1000F03D0B9F1000F6A
:104F100003D114E03878C00711D020680EF04CFEA1
:104F2000C8BBB8F1000F07D1206812302860206894
:104F3000143068602068A8602168CAF800103878CA
:104F4000800725D560680EF055FE20BBB9F1000F33
:104F500022D0FFF71EF80168C6F8C8118188A6F8AC
:104F6000CC11807986F8CE01FFF7A9FFD34F203707
:104F7000EF60626862B196F8C80106F2C911400894
:104F80001032FEF749FA1022394660681EF0B2FC72
:104F90000020BDE8F08706E0606820B1E860606846
:104FA000C6F8C401F4E71020F3E730B505460878E9
:104FB0000C4620F00F00401C20F0F0011031217051
:104FC0000020607095F8230030B104280FD0052828
:104FD00011D0062814D0FFDF20780121B1EB101F7B
:104FE00004D295F8200000F01F00607030BD21F061
:104FF000F000203002E021F0F00030302070EBE7CC
:1050000021F0F0004030F9E710B510B190F8BD4044
:1050100044B1AA4890F83540002064B1086010609F
:10502000186010BD00F1BC040C6000F1E40100F553
:1050300086701160F4E7A14C34340C60EFE700B5E2
:105040008BB00723CDE902128DF8013001919B4905
:10505000002364310591099301468DF810306846AC
:105060000CF088FD002800D0FFDF0BB000BD70B54C
:1050700090B015460C4602220646ADF808200921DC
:1050800003AB04F04EFF0490002812D00C208DF8E2
:10509000010004208DF8040004F59A740996059423
:1050A0008DF818500AA968460CF064FD00B1FFDFC6
:1050B000012010B070BD10B588B00C460A99ADF84B
:1050C0000000C3B11868CDF802005868CDF806009A
:1050D000ADF80A20102203A81EF00CFC68460AF066
:1050E00057F803F00FFF002803D1A17F41F0100112
:1050F000A17708B010BD0020CDF80200E6E72DE949
:10510000F0470646808A88B080B20D468246FDF799
:10511000E8FF04463078DFF8A4914FF00008A9F1C9
:105120003807112873D2DFE800F072F735093677B7
:105130007E94A3E7F6F5F4F35BF3F300A07F00F0B1
:105140000300012806D0002150460BF0C1F90500EC
:1051500003D101E00121F7E7FFDF99F85C10C907EF
:1051600002D0D9F860000BE0032105F121000EF018
:10517000D4F9D5F821005249B0FBF1F201FB12003D
:10518000C5F821007068A867B068E867207825280E
:1051900000D0FFDFE6E0A07F00F00300012806D08A
:1051A000002150460BF094F9060003D101E00121E3
:1051B000F7E7FFDF3078810702D52178252904D071
:1051C00040F00100307008B0E3E60220287096F845
:1051D0002000287106F121003136C5E90206F2E708
:1051E000A07F00F00300012806D0002150460BF0FC
:1051F0006FF9040003D101E00121F7E7FFDF207818
:10520000C10605D51320287041346C60DBE7B8E196
:1052100040F008002070D6E72848082138380EF002
:105220007CF9032012E01022684671681EF062FBD0
:10523000102204A8B1681EF05DFB6F60D6E9010181
:105240003A4609F0B6F800B1FFDF042028706F601D
:10525000B9E7E07FC00600D5FFDF307CB28800F000
:10526000010308B05046BDE8F047092105F0E1BC54
:1052700004B9FFDF716821B1102204F124001EF08F
:1052800039FB28212046FDF75EFFA07F00F00300D8
:1052900002280ED104F12400002300901A46214672
:1052A0005046FFF708FF11280CD029212046FDF7B2
:1052B0004AFF307A84F8200085E700002C020020A5
:1052C00040420F00A07F000700D5FFDF14F81E0F3B
:1052D00040F008002070A4F81680C4F81880C4F8C4
:1052E0001C806178084661F38200410861F3C300C5
:1052F0006070307AE07066E7A07F00F0030001285C
:105300000BD0002150460BF0E3F8040008D106E072
:105310001AE032E16DE044E02BE00121F2E7FFDF2B
:10532000022104F189000EF0F8F81020287004F52D
:10533000E4706860B4F88910298204F18000FB49A8
:105340006861C5E902913EE7A07F00F003000128F3
:1053500005D0002150460BF0BBF818B901E001213F
:10536000F8E7FFDF08B0324621465046BDE8F04777
:1053700086E504B9FFDF207821289DD930790128FE
:1053800003D1E07F40F01000E077324621465046DE
:10539000FFF776FD08B02046BDE8F0472321FDF772
:1053A000D2BE3279AA8005F108030921504604F0E3
:1053B000B8FDE86010B11120287004E7A07F00F06C
:1053C0000300012806D0002150460BF081F80400AC
:1053D00003D101E00121F7E7FFDF04F166010223B9
:1053E0001022081F0AF0F9FE80F800803179417020
:1053F000E9E6A07F00F00300012806D00021504616
:105400000BF066F8050003D101E00121F7E7FFDFAB
:1054100095F8880000F00300012879D1A07F00F002
:105420000307E07FC0F3400616B1012F04D02BE044
:1054300095F8A400C0072AD0D5F8C01119B395F883
:105440008720087C62F387000874E27FD5F8C011DA
:1054500062F341000874D5F8C01166F300000874C7
:10546000AEB1D5F8C001102204F124018C351EF034
:1054700041FA287E40F001002876287820F00100CB
:1054800005F88C0900E016B1022F04D02CE095F845
:105490008C00C00726D0D5F8BC1119B395F8872029
:1054A000087C62F387000874E27FD5F8BC1162F3D0
:1054B00041000874D5F8BC1166F3000008748EB181
:1054C000D5F8BC01102204F124018C351EF012FA2B
:1054D000287840F0010005F8180B287820F001002A
:1054E00005F8A409022F44D05FF0000000EB400053
:1054F00005EBC00090F88C00800709D595F8800076
:10550000D5F8C421400805F181011032FDF784FF70
:1055100005208DF8000095F888006A4600F0030029
:105520008DF8010095F88C108DF8021095F8A40004
:105530008DF803002146504601F038FA20782528DE
:1055400005D0212807D0FFDF2078222803D9222187
:105550002046FDF7F8FDA07F00F0030001280AD0E7
:10556000002150460AF0C6FF00283FF438AEFFDFA6
:1055700029E60120BAE70121F3E7716881F801808B
:1055800021E6FFDF1FE670B5684C0025103C04F8EB
:105590005C5F65600CF0BBFA6449A1F1100003F098
:1055A00037FE04F82C5C0620607260487C30206175
:1055B0005030A0611030E06170BD70B50D46FDF750
:1055C00090FD040000D1FFDF4FF4E87128461EF083
:1055D00032FA56485430686104F124002861A07FF3
:1055E00000F00300012809D05FF0020105F59A7070
:1055F0000CF08EFA002800D0FFDF70BD0121F5E726
:105600000A46014602F59A700CF0A2BA70B505463A
:10561000406886B001780A2906D00D2933D00E29BA
:105620002FD0FFDF06B070BD46883046FDF759FD2C
:10563000040000D1FFDF20782128F3D028281BD1D7
:10564000686802210C3001F0A6F9A8B16868082149
:10565000001D01F0A0F978B104F12401304609F0F1
:10566000AEFF03F04FFC00B1FFDF06B02046BDE8FF
:1056700070402921FDF767BD06B0BDE8704003F01A
:105680000EBE01218171686886883046FDF729FDCC
:10569000040000D1FFDFA07F00F00301022902D146
:1056A00020F01000A077207821280AD0686881793E
:1056B00009B1807880B1A07F00F0030002285ED09D
:1056C000FFDFA07F00F003000228ABD1FDF714FF3D
:1056D0000028A7D0FFDFA5E703F0E1FDE07FC107C9
:1056E00028D0800705D594F8200000F01F0010286E
:1056F0001ED0052084F82300207829281CD02428D7
:10570000DFD1314605200EF0E5F922212046FDF7D4
:105710001AFDA07F00F0030001282ED000213046A2
:105720000AF0E8FE0028CCD0FFDFCAE73C020020E8
:105730000620DFE70420DDE7A07F00F0030001285A
:1057400006D0002130460AF0C3FE050003D101E077
:105750000121F7E7FFDF25212046FDF7F4FC0F20AC
:105760008DF80000694605F59A700CF0E8F90228FA
:10577000A7D00028A5D0FFDFA3E70121CFE703F0E2
:105780008EFD9EE72DE9F0438BB09946154688467D
:105790000646FDF7A6FC04004FD0207822284CD303
:1057A00023284AD0E07FC00647D4A07F00F0030042
:1057B000012806D0002130460AF08AFE070002D0F8
:1057C0000CE00121F7E7A07F00F00300012805D1DC
:1057D0000121002230460AF072FE074601AB02AA00
:1057E00003A93846FFF710FC039800B9FFDF4FB15B
:1057F000039807F59A7787612078222806D0242815
:1058000004D007E003990020886103E025212046A9
:10581000FDF799FC03980B21417046628580C0E931
:105820000289029901610199416104A90CF0A2F970
:10583000022802D0002800D0FFDF0BB0BDE8F083C3
:1058400070B586B00546FDF74CFC017822291CD9BD
:10585000807F00F00300012806D0002128460AF0CE
:1058600037FE04002FD101E00121F7E7FFDF2AE036
:10587000B4F8620004F1660630440178427829B138
:1058800021462846FFF7F3FBB0B9CBE6ADF804207C
:105890000921284602AB04F044FB03900028F4D011
:1058A00011208DF80000694604F59A700CF047F954
:1058B000022801D000B1FFDF02231022314604F19B
:1058C00062000AF0C0FCB4F864000028D0D1A9E658
:1058D00010B586B00446FDF704FC0178222919D9D9
:1058E000807F00F00300012806D0002120460AF046
:1058F000EFFD040003D101E00121F7E7FFDF1220F3
:105900008DF80000694604F59A700CF018F900282B
:1059100000D0FFDF06B010BD2DE9F05F05460C4654
:1059200000270078904601093E46BA4604F1080B6C
:1059300002297CD0072902D00A2909D142E06868EF
:1059400001780A2905D00D292CD00E292AD0FFDF95
:10595000B2E114271C26002C6AD04088A080FDF7F5
:10596000C0FB5FEA000900D1FFDF99F817005A4633
:10597000400809F11801FDF74FFD68688089208211
:1059800069684868C4F812008868C4F81600A07EE8
:1059900020F0060040F00100A07699F81E0040F0CB
:1059A00040014DE01A270A26002CD5D08088A0801F
:1059B000FDF797FB050000D1FFDF59462846FFF7AA
:1059C000F4FA79E10CB1A88BA080287A0D287CD05C
:1059D00006DC01287AD0022808D0032804D135E05B
:1059E0000F2874D0102873D0FFDF65E11E27092629
:1059F000002CB1D0A088FDF774FB5FEA000900D14C
:105A0000FFDF287B00F003000128207A1BD020F064
:105A100001002072297B890861F341002072297BF3
:105A2000C90861F382002072297B090901E038E18D
:105A3000EBE061F3C300207299F81E0040F0800192
:105A400089F81E1038E140F00100E2E713270D2627
:105A5000002CAAD0A088FDF744FB8146807F00F08F
:105A60000300012806D00021A0880AF031FD0500BE
:105A700003D101E00121F7E7FFDF99F81E0000F0F4
:105A80000302012A59D0E86F817801F0030101294E
:105A9000217A54D021F00101217283789B0863F3AD
:105AA000410121728378DB0863F3820121728378DC
:105AB0001B0963F3C3012172037863F3061121729A
:105AC000437863F3C711217203E060E0A6E08DE044
:105AD0009EE084F809A0C178A172012A32D04279EF
:105AE000E17A62F30001E1724279520862F3410106
:105AF000E1724279920862F38201E1724279D2083E
:105B000062F3C301E1720279217B62F30001217328
:105B10000279520862F3410121730279920862F31B
:105B2000820121730079C00860F3C301217399F8E1
:105B30000000232859D9262168E0A86FA4E741F086
:105B40000101A9E70279E17A62F30001E1720279C9
:105B5000520862F34101E1720279920862F3820114
:105B6000E1720279D20862F3C301E1724279217BCA
:105B700062F3000121734279520862F341012173FB
:105B80004279920862F3820121734079CBE71827AA
:105B90001026D4B3A088FDF7A4FA8346807F00F0D6
:105BA0000300012807D00021A0880AF091FC5FEAD9
:105BB000000903D101E00121F6E7FFDFE868A060FA
:105BC00099F8000040F0040189F8001099F80100EC
:105BD000800708D5012020739BF8000023286BD98B
:105BE000272158464FE084F80CA065E015270F26C2
:105BF0005CB1A088FDF775FA814606225946E8682F
:105C000008F0E0F80120A0739BE03FE048463AE04E
:105C100016270926D4B3287B20724DE0287B19274C
:105C20000E269CB3C4F808A0A4F80CA0012807D045
:105C3000022805D0032805D0042803D0FFDF0DE09B
:105C4000207207E0697B042801F00F0141F0800118
:105C500021721CD0607A20F003006072A088FDF7EA
:105C600040FA05460078212826D0232800D0FFDFFF
:105C7000A87F00F00300012811D00021A0880AF0BD
:105C800039FC22212846FDF75EFA15E004E0607A2F
:105C900020F00300401CE0E7A8F8006011E00121BB
:105CA000ECE70CB16888A080287A03282BD0042860
:105CB0000AD005284BD0FFDFA8F800600CB1278080
:105CC00066800020BDE8F09F15270F26002CE3D04A
:105CD000A088FDF706FA807F00F00300012806D0B7
:105CE0000021A0880AF0F4FB050003D101E00121A6
:105CF000F7E7FFDFD5F821000622594608F062F8E1
:105D000084F80EA0D8E717270926002CC4D0A08855
:105D1000FDF7E7F98146807F00F00300012806D0F7
:105D20000021A0880AF0D4FB050003D101E0012185
:105D3000F7E7FFDF6878800701D5022000E0012047
:105D4000207299F800002328B6D927215EE7192789
:105D50000E26002CA0D0A088FDF7C3F95FEA000949
:105D600000D1FFDFC4F808A0A4F80CA084F808A0B4
:105D7000A07A40F00300A07299F81F1061F382002E
:105D8000A07299F81F10C1F34002114205D099F892
:105D9000201001F01F0110292CD020F00800A07263
:105DA00099F81F004108607A61F3C3006072697A54
:105DB00001F003010129A5D140F00400607299F8B7
:105DC0001E00E97A00F00300012816D0607B61F321
:105DD00000006073AA7A217B62F300012173EA7AE2
:105DE000520862F341006073A87A400860F34101F1
:105DF000217361E740F00800D1E7207B61F30000E8
:105E00002073AA7A617B62F300016173EA7A520817
:105E100062F341002073A87A400860F34101617386
:105E20004AE710B5FE4C30B10146102204F12000C3
:105E30001DF060FD012084F8300010BD10B504464F
:105E4000FFF73DF8F64920461022BDE8104020310A
:105E50001DF050BD70B5F24D06004FF0000413D098
:105E60000DF084FE08B110240CE00621304607F046
:105E700090FF411C05D028665FF0010085F85C00AA
:105E800000E00724204670BD0020F7E7007810F0FE
:105E90000F0204D0012A05D0022A0CD110E000091B
:105EA00009D10AE00009012807D0022805D00328FB
:105EB00003D0042801D007207047087000207047E5
:105EC0000620704705282AD2DFE800F003070F17E5
:105ED0001F00087820F0FF001EE0087820F00F0077
:105EE000401C20F0F000103016E0087820F00F0081
:105EF000401C20F0F00020300EE0087820F00F0069
:105F0000401C20F0F000303006E0087820F00F0050
:105F1000401C20F0F000403008700020704707203F
:105F200070472DE9F041804688B00D4600270846AD
:105F30000DF069FEA8B94046FDF7D3F8040003D080
:105F40002078222815D104E043F2020008B0BDE811
:105F5000F08145B9A07F010603D500F003000228B7
:105F600001D01020F2E7A07FC10601D4010702D5BD
:105F70000DB10820EAE7E17FC90601D50D20E5E76C
:105F800000F00300022805D125B12846FEF70AFFDC
:105F90000700DBD1A07F00F00300012806D000211C
:105FA00040460AF095FA060002D00DE00121F7E71D
:105FB000A07F00F0030001280CD000210022404601
:105FC0000AF07DFA060007D0A07F00F00300022847
:105FD00004D009E00121F1E70420B7E725B12A4602
:105FE00031462046FEF702FF07AB1A4669463046A7
:105FF000FFF70AF8009800B9FFDF00990C204870FD
:1060000006F59A70C1F82480486100200881A07FBD
:1060100000F00300012828D0EDB302200871301DE4
:1060200088613078400908777078C0F3400048777D
:10603000287800F00102887F62F301008877E27F10
:1060400062F382008877E27F520862F3C3008877A8
:10605000727862F304108877A878C87701F121027A
:1060600028462031FEF7E2FE22E001200871287860
:1060700000F00102087E62F3010008762A785208D7
:1060800062F3820008762A78920862F3C3000876E9
:106090002A78D20800E007E062F304100876242191
:1060A0002046FDF750F80BE0032008710520087624
:1060B00025212046FDF747F8A07F20F08000A0773B
:1060C00001A900980BF056FD022801D000B1FFDFB6
:1060D00038463BE72DE9FF4F524A0D4699B09A46A4
:1060E00007CA14AB002783E807001998FCF7F9FFEB
:1060F000060006D03078262806D008201DB0BDE85E
:10610000F08F43F20200F9E7B07F00F00309B9F124
:10611000010F03D0B9F1020F07D008E03DB91B9879
:10612000FEF740FE0028E9D101E01B9880BBB07F5C
:1061300000F00300012806D0002119980AF0C8F9E0
:10614000040003D101E00121F7E7FFDF852D28D00E
:1061500007DCF5B1812D1ED0822D1ED0832D08D1F4
:106160001DE0862D1FD0882D1FD0892D1FD08A2D90
:106170001FD00F2020710F281DD003F08DF8E0B143
:1061800001208DF83400201D0E902079B8B160E117
:1061900011E00020EEE70120ECE70220EAE703200F
:1061A000E8E70520E6E70620E4E70820E2E7092023
:1061B000E0E70A20DEE70720A0E711209EE7B9F11B
:1061C000010F17D0D4E91E50804602200190012013
:1061D0000090A87898F80210C0F3C000C1F3C00185
:1061E00008405FEA000B63D050460DF0BFFC00286A
:1061F00072D133E0D4E91E85012001900220009085
:10620000214630461B9AFEF7F1FD1B98007800F0FE
:106210000101A87861F30100A870F17F04E000009B
:106220002C020020B43D020061F38200A870F17FCF
:10623000490861F3C300A870617861F30410A87085
:106240002078400928706078C0F3400068701B987F
:106250008078E870002068712871BAE7DAF80C00DD
:106260000DF084FCC0BBDAF81C000DF07FFC98BB7D
:10627000DAF80C00A060DAF81C00E06098F8010081
:10628000617800F0010041EA4000607098F8021067
:10629000C0B2C1F30011891E08406070002084F86C
:1062A0002000009906F1170002290BD001210AE015
:1062B00098F80110607801F00101FD2242EA4101E5
:1062C0000840E2E7002104EB810188610199701C1C
:1062D000022902D0012101E028E0002104EB810124
:1062E0008861A87800F00300012849D198F80200DD
:1062F00000F00300012843D1B9F1010F04D12A1D98
:10630000691D1B98FEF792FD287998F80410084043
:106310008DF82C00697998F8052011408DF830101F
:1063200008432DD050460DF021FC08B11020E5E6C1
:106330000AF1100004F5DE7104F190020490B9F145
:10634000020F3CD00090CDE9012100210BAB5A4651
:106350002046FEF7C8FD0028E9D104F5E07104F1FC
:10636000A802B9F1010F30D004980090CDE90121C5
:1063700000210CAB5A462046FEF7B5FD0028D6D1C9
:106380006078800740D4A87898F80210C0F38000A5
:10639000C1F38001084337D0297898F8000014AA87
:1063A000B9F1010F17D032F810204B00DA4012F08B
:1063B000030718D0012F1ED0022F12D11DE0CDF8F7
:1063C00000A0CDE901210121C0E7CDF800A0CDE971
:1063D00001210121CDE732F811204300DA4002F01B
:1063E0000307032F07D0BBF1000F0DD0012906D002
:1063F000042904D008E00227F5E70127F3E7012884
:1064000001D0042800D10427F07F40F001006BF395
:106410004100F077607881074FF003000CD5A07140
:10642000BBF1000F15D100BF8DF85C0017AA3146F3
:10643000199800F0BBFA0CE00221022F18D0012FAE
:1064400018D0042F22D00020A071F07F20F001008E
:10645000F07725213046FCF776FE0DA904F59A70F9
:106460000BF06DFB10B1022800D0FFDF002045E6E5
:10647000A171D9E7A1710D2104F124001DF0DBFA0F
:10648000207840F0020020700420CDE70120A071A8
:10649000DFE72DE9F04387B09046894604460025A2
:1064A000FCF71FFE060006D03078272806D008200B
:1064B00007B0BDE8F08343F20200F9E7B07F00F0D7
:1064C0000300012806D0002120460AF001F804004C
:1064D00003D101E00121F7E7FFDFA7795FEA0900B7
:1064E00005D0012821D0B9F1020F26D110E0B8F172
:1064F000000F22D1012F05D0022F05D0032F05D088
:10650000FFDF2DE00C252BE0012529E0022527E007
:1065100040460DF02BFBB0B9032F0ED1102241469F
:1065200004F121001DF0E6F91AE0012F02D0022F3C
:1065300003D104E0B8F1000F12D00720B8E74046BD
:106540000DF014FB08B11020B2E7102104F1210076
:106550001DF04FFA0621404607F01BFCC4F821004D
:106560002078252140F0020020703046FCF7EBFD3A
:106570002078C10714D020F00100207002208DF88F
:10658000000004F1210002908DF80450694604F5E2
:106590009A700BF0D4FA022804D018B1FFDF01E0A2
:1065A00084F82050002083E730B587B00D460446BC
:1065B000FCF797FD88B1807F00F0030001280FD021
:1065C0000021204609F084FF04000ED028460DF07B
:1065D000CDFA38B1102007B030BD43F20200FAE71F
:1065E0000121EEE72078400701D40820F3E729468F
:1065F00004F14100202205461DF07CF9207840F08E
:106600001000207001070FD520F008002070132023
:106610008DF80000694604F59A7001950BF08FFA29
:10662000022801D000B1FFDF0020D4E770B50D468D
:106630000646FCF756FD18B1017827291FD102E064
:1066400043F2020070BD807F00F00300012806D0F5
:106650000021304609F03CFF040003D101E0012194
:10666000F7E7FFDFA079022809D16078C00706D0DC
:106670002A4621463046FEF7FAFC10B10FE008200A
:1066800070BDB4F864000E280BD204F16601022339
:106690001022081F09F0A1FD0121017045700020A2
:1066A00070BD112070BD70B5064686B014460D460B
:1066B00008460DF05BFA18B920460DF07DFA10B1CE
:1066C000102006B070BDA6F57F40FF380ED03046D2
:1066D000FCF707FD38B1417822464B08811C18466B
:1066E000FCF79AFE07E043F20200EAE72046FDF7D6
:1066F000AFFC0028E5D11021E01D0CF00EFFE21DDB
:1067000029466846FEF79BFC102204F11700019908
:106710001DF0F0F80020D4E72DE9F041044686B0E2
:1067200015468846002708460DF06DFA18B9284628
:106730000DF069FA10B1102006B008E42046FCF70D
:10674000D0FC060003D03078272818D102E043F2AD
:106750000200F1E7B07F00F00300012806D000211D
:10676000204609F0B5FE040003D101E00121F7E75E
:10677000FFDF2078400702D56078800701D4082029
:10678000DAE7B07F00F00300012818D0D4E91E0139
:10679000407800B1B5B1487810B1B8F1000F11D010
:1067A000C5B1EA1D6846E168FEF749FC102205F113
:1067B000170001991DF072F830B104270AE0D4E9FE
:1067C0001E10E5E70720B7E71022E91D04F13100AC
:1067D0001DF090F8B8F1000F06D0102208F1070163
:1067E00004F121001DF086F82078252140F00200F8
:1067F00020703046FCF7A7FC2078C10716D020F0A7
:106800000100207002208DF8000004F121000290A8
:10681000103003908DF80470694604F59A700BF0FF
:106820008EF9022804D018B1FFDF01E084F820704F
:10683000002081E7F8B515460E460746FCF751FCE7
:10684000040004D02078222804D00820F8BD43F2A8
:106850000200F8BDA07F00F00300022802D043F23E
:106860000500F8BD30460DF081F918B928460DF045
:106870007DF908B11020F8BD00953288B31C21467F
:106880003846FEF718FC112814D00028F3D1297CD3
:106890004A08E17F62F30001E1772A7C62F341015B
:1068A000E177297C890884F82010A17F21F08001FC
:1068B000A177F8BDA17F0907FBD4D6F80200C4F880
:1068C0003600D6F80600C4F83A003088A0861022B8
:1068D000294604F124001DF00DF8287C4108E07FD2
:1068E00061F38200E077297C61F3C300E077287CC4
:1068F000800884F82100A07F40F00800A0770020E5
:10690000D3E770B50D4606460BB1072070BDFCF706
:10691000E8FB040007D02078222802D3A07F40069D
:1069200004D4082070BD43F2020070BDA5B1294611
:10693000304608F044FE02F0E5FA297C4A08E17F7F
:1069400062F30001E1772A7C62F34101E177297C5F
:10695000890884F8201004E0304608F058FE02F060
:10696000D1FAA17F21F04001A17770BD70B50D462D
:10697000FCF7B7FB040005D028460DF01DF920B147
:10698000102070BD43F2020070BD29462046FEF77C
:106990000CFB002070BD04E010F8012B0AB10020B0
:1069A0007047491E89B2F7D20120704770B515466D
:1069B000064602F071FC040000D1FFDF207820F0D1
:1069C0000F00801C20F0F0002030207066802868C6
:1069D000A060BDE8704002F062BC000018B1817890
:1069E000012938D101E010207047018842F60112D8
:1069F000881A914231D018DC42F60102A1EB020064
:106A000091422AD00CDC41B3B1F5C05F25D06FF4C0
:106A1000C050081821D0A0F57060FF381BD11CE0D1
:106A200001281AD002280AD117E0B0F5807F14D0CF
:106A300008DC012811D002280FD003280DD0FF2830
:106A400009D10AE0B0F5817F07D0A0F58070033846
:106A500003D0012801D0002070470F2070470B2879
:106A600026D008DC1BD2DFE800F01C2025251A25E3
:106A7000292325271E0011281CD008DC0C2817D03C
:106A80000D281DD00F2815D0102808D110E082281D
:106A900009D0842810D0852810D0872812D0032050
:106AA0007047002070470520704743F2030070478D
:106AB000072070470F20704704207047062070475A
:106AC0000C20704743F20200704738B50C460500B1
:106AD00041D06946FFF7DAF9002819D19DF8001076
:106AE000607861F3020060706946681CFFF7CEF9B8
:106AF00000280DD19DF80010607861F3C50060702A
:106B0000A978C1F34101012903D0022905D007204A
:106B100038BD217821F0200102E0217841F02001E8
:106B20002170410704D0A978C90861F3861060700C
:106B3000607810F0380F07D0A978090961F3C71001
:106B4000607010F0380F02D16078400603D52078CD
:106B500040F040002070002038BD70B50446002091
:106B6000088015466068FFF7B0FF002816D120891D
:106B7000A189884211D860688078C0070AD0B1F531
:106B8000007F0AD840F20120B1FBF0F200FB1210A6
:106B9000288007E0B1F5FF7F01D90C2070BD01F21C
:106BA00001212980002070BD10B50478137864F3AA
:106BB000000313700478640864F3410313700478CD
:106BC000A40864F3820313700478E40864F3C30335
:106BD00013700478240964F30413137004786409AF
:106BE00064F3451313700078800960F38613137003
:106BF00031B10878C10701D1800701D5012000E03B
:106C0000002060F3C713137010BD4278530702D001
:106C100002F0070306E012F0380F02D0C2F3C203FD
:106C200000E001234A7863F302024A70407810F0D2
:106C3000380F02D0C0F3C20005E0430702D000F0D5
:106C4000070000E0012060F3C5024A7070472DE99B
:106C5000F04F95B00D00804615D0B8F1000F16D05A
:106C6000122128461CF0C5FE4FF6FF7B05AA012124
:106C7000584606F0CEFE0024264637464FF42059EB
:106C80006FF4205A75E0102015B0BDE8F08F072092
:106C9000FAE700BF9DF81E0001280AD1BDF81C00CC
:106CA00048450BD010EB0A000AD001280CD002286E
:106CB0000CD0042C0ED0052C0FD10DE0012400E0E7
:106CC0000224BDF81A6008E0032406E00424BDF89D
:106CD0001A7002E0052400E00624BDF81A104145B0
:106CE00047D12C74BEB34FF0000810AA4FF0070A2A
:106CF000CDE90282CDE900A80DF13C091023CDF8C1
:106D0000109042463146584606F036FF08BBBDF8A3
:106D10003C002A46C0B210A90AF0CEFFC8B9AE8125
:106D2000CFB1CDE900A80DF1080C0AAE40468CE8C1
:106D30004102132300223946584606F01DFF40B990
:106D4000BDF83C00F11CC01EC0B22A1D0AF0B4FF01
:106D500010B1032098E70AE0BDF82900E881062C6D
:106D600005D19DF81E00A872BDF81C0028810020E6
:106D70008AE705A806F059FE00288BD0FFF76FFEC2
:106D800082E72DE9F0471C46DDE90978DDF820901F
:106D900015460E00824600D1FFDF0CB1208818B1E5
:106DA000D5B11120BDE8F087022D01D0012100E00E
:106DB000002106F1140005F01DFDA8F800000246B0
:106DC0003B462946504603F0ACF8C9F8000008B924
:106DD000A41C3C600020E5E71320E3E7F0B4144670
:106DE000DDE904528DB1002314B1022C09D101E078
:106DF000012306E00D7CEE0703D025F001050123F9
:106E00000D742146F0BC03F014BF1A80F0BC70472B
:106E10002DE9FE4F91461A881C468A468046FAB1F3
:106E200002AB494603F07DF8050019D04046A61C88
:106E3000278809F091FC3246072629463B460096F2
:106E400009F09DF820882346CDE900504A46514676
:106E50004046FFF7C3FF002020800120BDE8FE8FE1
:106E60000020FBE72DE9F04786B09146DDE90E46AC
:106E70000F46824603AA05A904A8109D8DE80700C5
:106E80009846324621465046FFF77BFF049909B1E8
:106E9000012200E000222A70002817D1F84A03AB33
:106EA0001060059A009104F11400CDE901204A46D2
:106EB0003946504606F055F890B108280ED2DFE862
:106EC00000F00407040D0D090B0B002006B069E764
:106ED0001120FBE70720F9E70820F7E70320F5E793
:106EE000BDF80C100498CDE9000143463246214616
:106EF0005046FFF773FFE8E72DE9F04389B00D46F0
:106F0000DDE9108781461C461646142103A81CF0B3
:106F100092FD012002218DF810108DF80C008DF8E3
:106F20001170ADF8146064B1A278D20709D08DF861
:106F30001600E088ADF81A00A088ADF81800A06827
:106F4000079008A80095CDE90110424603A94846DC
:106F50006B68FFF787FF09B0BDE8F083F0B58BB031
:106F600000240646069407940727089405A8099468
:106F7000019400970294CDE903400D461023224668
:106F8000304606F0F9FD78B90AA806A901940097E1
:106F90000294CDE90310BDF8143000222946304692
:106FA00006F0C0FB002801D0FFF759FD0BB0F0BD83
:106FB00006F060BA2DE9FC410C468046002602F03E
:106FC0006BF9054620780D287ED2DFE800F0BC077B
:106FD00013B325BD49496383AF959B00A84800685A
:106FE00020B1417841F010014170ADE0404602F01F
:106FF00083F9A9E00421404609F06AFA070000D1AC
:10700000FFDF07F11401404605F088FBA5BB132103
:107010004046FDF78FFB97E00421404609F058FAFF
:10702000070000D1FFDFE088ADF800000020B88144
:107030009DF80000010704D5C00602D5A088B881DC
:1070400005E09DF8010040067ED5A088F88105B9CD
:10705000FFDF22462946404601F068FC022673E025
:10706000E188ADF800109DF8011009060FD507283A
:1070700003D006280AD00AE024E00421404609F0A3
:1070800027FA060000D1FFDFA088F0810226CDB9E3
:10709000FFDF17E00421404609F01AFA070000D18B
:1070A000FFDF07F1140006F01CFA90F0010F02D187
:1070B000E079000648D5387C022640F0020038749A
:1070C00005B9FFDF224600E03DE02946404601F0D9
:1070D0002DFC39E00421404609F0FAF9017C002D2D
:1070E00001F00206C1F340016171017C21F002014F
:1070F0000174E7D1FFDFE5E702260121404602F0F7
:107100002DF921E00421404609F0E2F905466068C6
:1071100000902089ADF8040001226946404602F043
:107120003EF9287C20F0020028740DE0002DC9D122
:10713000FFDFC7E7022600214046FBF742F9002D9A
:10714000C0D1FFDFBEE7FFDF3046BDE8FC813EB5C2
:107150000C0009D001466B4601AA002006F08EFD06
:1071600020B1FFF77CFC3EBD10203EBD00202080FA
:10717000A0709DF8050002A900F00700FEF7A2FE2E
:1071800050B99DF8080020709DF8050002A9C0F3D1
:10719000C200FEF797FE08B103203EBD9DF808002F
:1071A00060709DF80500C109A07861F30410A0701B
:1071B0009DF80510890961F3C300A0709DF80410C3
:1071C000890601D5022100E0012161F342009DF80A
:1071D000001061F30000A07000203EBD70B51446A1
:1071E00006460D4651EA040005D075B108460CF07C
:1071F00001FD78B901E0072070BD2946304606F050
:107200009EFD10B1BDE8704029E454B120460CF059
:10721000F1FC08B1102070BD21463046BDE8704039
:1072200095E7002070BD2DE9FC5F0C4690460546B1
:10723000002701780822007A3E46B2EB111F7DD16B
:1072400004F10A0100910A31821E4FF0020A04F192
:10725000080B0191092A72D2DFE802F0EDE005F592
:1072600028287BAACE006888042109F031F906009D
:1072700000D1FFDFB08928B152270726C3E0000004
:107280002803002051271026002C7DD06888A0807C
:107290000120A071A88900220099FFF79FFF002814
:1072A00073D1A8892081288AE081D1E0B5F81290B5
:1072B000072824D1E87B000621D5512709F11400C5
:1072C00086B2002CE1D0A88900220099FFF786FF42
:1072D00000285AD16888A08084F806A0A889208157
:1072E0000120A073288A2082A4F81290A88A009016
:1072F00068884B46A969019A01F0F5FAA8E0502781
:1073000009F1120086B2002C3ED0A889002259460D
:10731000FFF764FF002838D16888A080A889E08042
:10732000287A072813D002202073288AE081E87B7E
:10733000C0096073A4F81090A88A01E085E082E09B
:10734000009068884B4604F11202A969D4E7012035
:10735000EAE7B5F81290512709F1140086B2002C23
:1073600066D06888042109F0B3F883466888A08055
:10737000A88900220099FFF731FF00286ED184F818
:1073800006A0A889208101E052E067E00420A073F4
:10739000288A2082A4F81290A88A009068884B4618
:1073A000A969019A01F09FFAA989ABF80E104FE084
:1073B0006888FBF796FE07466888042109F088F87C
:1073C000064607B9FFDF06B9FFDF687BC00702D0BA
:1073D0005127142601E0502712264CB36888A0805C
:1073E000502F06D084F806A0287B594601F08BFA6E
:1073F0002EE0287BA11DF9E7FE49A8894989814231
:1074000005D1542706269CB16888A08020E0532728
:107410000BE06888A080A889E08019E068880421D2
:1074200009F056F800B9FFDF55270826002CF0D1E7
:10743000A8F8006011E056270726002CF8D06888CD
:10744000A080002013E0FFDF02E0012808D0FFDF6A
:10745000A8F800600CB1278066800020BDE8FC9F82
:1074600057270726002CE3D06888A080687AA0718F
:10747000EEE7401D20F0030009B14143091D01EB77
:107480004000704713B5DB4A00201071009848B1E6
:107490000024684608F037FE002C02D1D64A009935
:1074A00011601CBD01240020F4E770B50D460646AE
:1074B00086B014465C2128461CF0BDFA04B9FFDFF3
:1074C000A0786874A2782188284601F046FA002046
:1074D000A881E881228805F11401304605F003F9FE
:1074E0006A460121304606F094FA19E09DF803003F
:1074F000000715D5BDF806103046FFF72FFD9DF8A3
:107500000300BDF8061040F010008DF80300BDF830
:107510000300ADF81400FF233046059A06F0DAFBAD
:10752000684606F082FA0028E0D006B070BD10B5BB
:107530000C4601F1140005F00DF90146627C20466D
:10754000BDE8104001F03EBA70B50546042108F0D0
:10755000BFFF040000D1FFDF04F114010C462846F0
:1075600005F0DCF821462846BDE8704005F0DDB89E
:1075700070B58AB00C460646FBF7B3FD050014D083
:107580002878222827D30CB1A08890B101208DF84B
:107590000C0003208DF8100000208DF8110054B16C
:1075A000A088ADF81800206807E043F202000AB096
:1075B00070BD0920FBE7ADF81800059004213046A6
:1075C00008F086FF040000D1FFDF04F1140005F08D
:1075D000D8F8000701D40820E9E701F05DFE60B1AA
:1075E00008A802210094CDE9011095F8232003A9F1
:1075F00030466368FFF736FCD9E71120D7E72DE95D
:10760000F04FB2F802A0834689B01546894650462D
:10761000FBF767FD07460421504608F059FF002696
:10762000044605964FF002080696ADF81C6007B9AF
:10763000FFDF04B9FFDF4146504603F062FE60B948
:1076400007AA06A905A88DE807004246214650462C
:107650006368FFF796FB00B1FFDF664807AB066083
:10766000DDE9051204F11400CDF80090CDE9032006
:10767000CDE9013197F82320594650466B6805F053
:10768000C9F806000AD0022E04D0032E14D0042E0E
:1076900000D0FFDF09B03046BDE8F08FBDF81C0018
:1076A0000028F7D00599CDE9001042462146504602
:1076B0006368FFF793FBEDE7687840F008006870B7
:1076C000E8E72DE9F04F9BB004464FF00008494829
:1076D000ADF85480ADF83080ADF85080A0F8088047
:1076E000ADF81480ADF81880ADF82080ADF81C809E
:1076F000007916460D464746012808D0022806D0D4
:10770000032804D0042802D008201BB0C4E7204678
:107710000CF02CFAD0BB28460CF028FAB0BB6068FD
:107720000CF071FA90BB606848B160892189884289
:1077300002D8B1F5007F01D90C20E6E780460BAAFC
:1077400006A92846FFF709FA0028DED16868807884
:10775000C0F34100022808D19DF8190010F0380F3D
:1077600003D028690CF046FA80B905A92069FFF713
:10777000ACF90028C9D1206950B1607880079DF824
:10778000150000F0380002D5C0B301E011E0A8BB3D
:107790009DF8140080060ED59DF8150010F0380FE6
:1077A00003D060680CF026FA18B960680CF02BFA68
:1077B00008B11020A9E707A96069FFF786F900283A
:1077C000A3D1606940B19DF81D0000F007010129B7
:1077D0003FD110F0380F3CD008A9A069FFF775F928
:1077E000002892D19DF81C00800632D49DF820001C
:1077F000800604E0280300201400002029E028D49B
:10780000A06940B19DF8210000F00701012920D1B5
:1078100010F0380F1DD0E06818B10078C8B11C28EE
:1078200017D20EAA611C2046FFF7BEF90120B94607
:1078300060F30F27BA4607468DF84E0042F6030064
:10784000ADF84C000DF13B0217A928680AF053FA75
:1078500008B1072059E79DF85C0016A9CDF8009003
:10786000C01CCDE9019100F0FF0B00230BF20122B7
:10787000514613A806F010F8F0BBBDF85800099067
:10788000FE482A8929690092CDE901106B89BDF86B
:107890002C202868069905F0FFFF01007ED1207892
:1078A0004FF0020AC10601D480062BD5ADF80C902A
:1078B000606950B907A906A8FFF7A7F99DF81D0050
:1078C00020F00700401C8DF81D009DF81C008DF86D
:1078D0004E7040F0C8008DF81C0042F60210ADF862
:1078E0004C000CA903AACDF800A0CDE9012100238A
:1078F00040F2032213A800E01EE0079905F0CCFF38
:1079000001004BD1DD484D4608385B460089ADF893
:1079100039000EA8CDE90290CDF80490CDF8109072
:107920004FF007090022CDF80090BDF858104FF62F
:10793000FF7005F0F7FE10B1FFF791F8E5E69DF84E
:107940003800000625D52946012060F30F218DF867
:107950004E704FF42450ADF84C00ADF810506278E2
:107960009DF81000002362F300008DF8100062788B
:10797000CDF800A0520862F341008DF8100004AA6F
:10798000CDE9012540F2032213A805F085FF01008F
:1079900004D1606888B32069A8B900E086E005A931
:1079A00006A8FFF732F96078800706D49DF8150025
:1079B00020F038008DF8150005E09DF8140040F027
:1079C00040008DF814008DF84E7042F60110ADF8AD
:1079D0004C00208940F20121B0FBF1F201FB1202C0
:1079E000606814ABCDF80080CDE90103002313A833
:1079F000059905F051FF010058D12078C00729D022
:107A0000ADF80C50A06950B908A906A8FFF7FDF819
:107A10009DF8210020F00700401C8DF821009DF802
:107A200020008DF84E7040F040008DF8200042F6A6
:107A30000310ADF84C0015A903AACDF800A0CDE9BC
:107A40000121002340F2032213A8089905F024FF26
:107A500001002BD1E06868B32946012060F30F21B3
:107A60008DF84E7042F60410ADF84C00E06800232B
:107A700002788DF8602040788DF86100E06818AADF
:107A80004088ADF86200E06800798DF86400E06835
:107A9000C088ADF86500CDF80090CDE901254FF420
:107AA000027213A805F0F8FE010003D0099800F057
:107AB000B5FF2AE6714803210838017156B10089E3
:107AC0003080BDF850007080BDF83000B080BDF847
:107AD0005400F080002018E670B501258AB01646E3
:107AE0000B46012802D0022816D104E08DF80E5072
:107AF0004FF4205003E08DF80E5042F60100ADF82F
:107B00000C005BB10024601C60F30F2404AA08A9D8
:107B100018460AF0F0F818B1072048E5102046E5AD
:107B200004A99DF820205548CDE90021801E02902F
:107B30000023214603A802F2012205F0ADFE10B198
:107B4000FEF78DFF33E54D4808380EB1C18831800E
:107B5000057100202BE5F0B593B0074601268DF89E
:107B60003E6041F60100ADF83C0012AA0FA9304674
:107B7000FFF7B2FF002848D1404C0025083CE7B38E
:107B80001C2102A81BF057FF9DF808008DF83E60ED
:107B900040F020008DF8080042F60520ADF83C00CA
:107BA0000E959DF83A00119520F00600801C8DF886
:107BB0003A009DF838006A4620F0FF008DF8380042
:107BC0009DF8390009A920F0FF008DF83900042044
:107BD000ADF82C00ADF830000EA80A9011A80D9059
:107BE0000FA80990ADF82E5002A8FFF76AFD0028F3
:107BF0000BD1BDF80000608100E008E0BDF8040092
:107C0000A081401CE0812571002013B0F0BD65818A
:107C1000A581BDF84800F4E72DE9F74F1749A0B05A
:107C20000024083917940A79A146012A04D0022AAF
:107C300002D0082023B02FE5CA88824201D0062056
:107C4000F8E721988A46824201D10720F2E7012015
:107C50002146ADF848004FF6FF7860F30F21ADF8EC
:107C60004A808DF86E0042F6020B06918DF8724044
:107C7000ADF86CB0ADF870401CA901E030030020F5
:107C80001391ADF8508012A805F0F3FE00252E46A2
:107C90002F460DAB072212A9404605F0EDFE78B144
:107CA00082285DD195B38EB3ADF86450ADF86660AF
:107CB0009DF85E008DF8144019AC012864D06BE08B
:107CC0009DF83A001FB3012859D1BDF83810594525
:107CD0001FD118A809A901940294CDE90310072027
:107CE0000090BDF8361010230022404605F044FFF6
:107CF000B0BBBDF86000042801D006284AD1BDF809
:107D00002410219881423AD10F2093E73AE00128CC
:107D100035D1BDF83800B0F5205F03D042F601013F
:107D200088422CD1BAF80600BDF83610884201D13D
:107D3000012700E0002705B19EB1219881421ED1A4
:107D400018A809AA01940294CDE903200720009005
:107D50000D4610230022404605F00EFF00B902E058
:107D60002DE04E460BE0BDF86000022801D010283F
:107D700010D1C0B217AA09A909F09EFF50B9BDF8E9
:107D8000369086E7052055E705A917A8221D09F0BA
:107D9000B2FF08B103204DE79DF814000023001D39
:107DA000C2B28DF8142022980092CDE901401BA8A0
:107DB000069905F071FD10B902228AF80420FEF739
:107DC0004EFE37E710B50B46401E88B084B205AAB8
:107DD00000211846FEF7E8FE00200DF1080C06AA67
:107DE00005A901908CE807000720009001230022DC
:107DF00021464FF6FF7005F095FC0446BDF81800CB
:107E0000012800D0FFDF2046FEF729FE08B010BD94
:107E1000F0B5F94F044687B038790E46032804D0F0
:107E2000042802D0082007B0F0BD04AA03A9204608
:107E3000FEF793FE0500F6D160688078C0F341003C
:107E400002280AD19DF80D0010F0380F05D02069E6
:107E50000BF0D0FE08B11020E5E7208905AA2169C2
:107E60008DE807006389BDF810202068039905F0AC
:107E700013FD10B1FEF7F3FDD5E716B1BDF8140000
:107E80003080042038712846CDE7F8B50C0006464E
:107E90000BD001464FF6FF7500236A46284605F0D1
:107EA000EDFE20B1FEF7DBFDF8BD1020F8BD694600
:107EB0002046FEF70AFE0028F8D1A078314600F0EF
:107EC00001032846009A05F005FFEBE730B587B0BF
:107ED000144600220DF1080C05AD01928CE82C002F
:107EE000072200920A46014623884FF6FF7005F0EC
:107EF00019FCBDF814102180FEF7B1FD07B030BDAC
:107F000070B50D46042108F0E3FA040000D1FFDF4C
:107F1000294604F11400BDE8704004F02BBC70B594
:107F20000D46042108F0D4FA040000D1FFDF2946F1
:107F300004F11400BDE8704004F03FBC70B50D467C
:107F4000042108F0C5FA040000D1FFDF294604F13E
:107F50001400BDE8704004F057BC70B5054604211C
:107F600008F0B6FA040000D1FFDF21462846236856
:107F7000BDE870400122FEF74BBF70B506460421F4
:107F800008F0A6FA040000D1FFDF04F1140004F0A9
:107F9000E1FB401D20F0030511E0011D00880022D7
:107FA000431821463046FEF733FF00280BD0607C93
:107FB000ABB2684382B2A068011D08F044F9A06822
:107FC00041880029E9D170BD70B50546042108F04B
:107FD0007FFA040000D1FFDF214628466368BDE830
:107FE00070400222FEF714BF70B50E46054601F040
:107FF00053F9040000D1FFDF012020726672658012
:10800000207820F00F00001D20F0F000403020709C
:10801000BDE8704001F043B910B50446012900D015
:10802000FFDF2046BDE810400121FAF7CAB92DE96B
:10803000F04F97B04FF0000A0C008346ADF818A03F
:10804000D04619D0E06830B1A068A8B10188ADF879
:108050001810A0F800A05846FBF743F8070043F2B9
:10806000020967D03878222862D30421584608F0E4
:108070002FFA050005D103E0102017B0BDE8F08FFE
:10808000FFDF05F1140004F065FB401D20F003063E
:10809000A078012803D0022801D00720EDE720882E
:1080A00078B1401C81B209AA584605F0B2FC09A873
:1080B00005F0BBFC9DF82E204FF45051012A0DD144
:1080C00002E043F20300D8E7BDF82C20A2F52453C8
:1080D000023B03D1822801D0A0B901E00846CCE7D9
:1080E000E068B0B1CDE902A0072006AACDF804A04F
:1080F00000900492A2882188BDF81830584605F0F7
:1081000011FB10B1FEF7ABFCB7E7A168BDF8180092
:1081100008809DF82700C00602D543F20140ACE775
:108120000D9838B1A1780078012905D080071AD4BC
:108130000820A2E74846A0E7C007F9D002208DF842
:108140003C00A8684FF00009A0B1697C42887143E7
:1081500091420FD98AB2B3B2011D08F02AF88046C5
:10816000A0F800A006E003208DF83C00D5F80080C0
:108170004FF001099DF8280010F0380F00D1FFDF03
:108180009DF828001D49C0F3C200084497F8231049
:1081900010F8010C884201D90F206EE72088ADF855
:1081A000400014A90095CDE90191434607220FA98B
:1081B0005846FEF757FE002885D19DF8500050B96B
:1081C000A078012807D1687CB3B2704382B2A86856
:1081D000011D08F002F800204FE770B5064615466D
:1081E0000C460846FEF7FAFB002809D12A4621462C
:1081F0003046BDE870406FE428030020BE3D020019
:1082000070BD09E570B51E4614460D0009D044B195
:10821000616831B138B1F849C988814203D007207B
:1082200070BD102070BD2068FEF7D8FB0028F9D182
:10823000324621462846BDE87040FFF742BA70B585
:1082400015460C0006D038B1EB490989814203D0AC
:10825000072070BD102070BD2068FEF7BFFB00280E
:10826000F9D129462046BDE87040D1E570B50646F3
:1082700086B00D46144610460BF09EFCD0BB6068DD
:108280000BF0C1FCB0BBA6F57F40FF3803D03046F1
:10829000FAF727FF80B128466946FEF7D8FC002888
:1082A0000CD19DF810100F2008293CD2DFE801F016
:1082B00008060606060A0A0843F2020006B070BD68
:1082C0000320FBE79DF80210012908D1BDF800103A
:1082D000B1F5C05FF2D06FF4C052D142EED09DF83C
:1082E000061001290DD1BDF80410A1F52851062969
:1082F00007D200E028E0DFE801F0030304030303F2
:10830000DCE79DF80A1001290ED1BDF80810B1F57F
:10831000245FD3D0A1F524510239CFD00129CDD08B
:10832000022901D1CAE7FFDF606878B9002305AAF6
:108330002946304605F0A2FC10B1FEF790FBBDE7E0
:108340009DF81400800601D41020B7E7618822460A
:1083500028466368FFF7BAFDB0E72DE9F043814690
:1083600087B08846144610460BF026FC18B1102042
:1083700007B0BDE8F083002306AA4146484605F051
:108380007DFC10B1FEF76BFBF2E79DF81800C0060C
:1083900002D543F20140EBE70025072705A8019528
:1083A00000970295CDE9035062884FF6FF7341466E
:1083B000484605F0E1FB060013D160680BF0FCFBBA
:1083C00060B960680195CDE9025000970495238853
:1083D00062884146484605F0CFFB0646BDF81400CA
:1083E00020803046CEE739B1834B0A889B899A4278
:1083F00002D843F20300704719E610B586B07E4CF0
:108400000423ADF81430638943B1A4898C4201D2AE
:10841000914205D943F2030006B010BD0620FBE7E8
:10842000ADF81010002100910191ADF8003002214B
:108430008DF8021005A9029104A90391ADF812204C
:108440006946FFF7F4FDE7E72DE9FC4781460E4654
:1084500008460BF08BFB88BB4846FAF742FE5FEA02
:1084600000080AD098F80000222829D304214846A1
:1084700008F02EF8070005D103E043F20200BDE842
:10848000FC87FFDF07F1140004F07BF90546307824
:10849000012803D0022804D00720F0E7A8070FD551
:1084A00002E015F01C0F0BD0B079341DC00709D0C5
:1084B000E08838B1A0680BF059FB18B11020DEE756
:1084C0000820DCE732782088002628B3A0F20113C8
:1084D0000721112B18D20CD2DFE803F00B090D0B8A
:1084E0001D0B121D100B0B1D1D1D1D0B1D00022A47
:1084F00011D10846C3E7012AFBD00CE02A0700E0AF
:10850000EA06002AF5DA06E0A0F5C0721F2A02D9B1
:108510007D3A022AEDD8C6B200F0BEFE50B198F8FE
:108520002300CDE90006FA89234639464846FEF77E
:10853000E3FCA4E71120A2E72DE9F04F8BB01F4622
:1085400015460C4683460026FAF7CBFD28B1007885
:10855000222805D208200BB090E543F20200FAE78A
:10856000B80801D00720F6E7032F00D100274FF607
:10857000FF79CCB1022D72D320460BF044FB30B909
:1085800004EB0508A8F101000BF03DFB08B1102039
:10859000E1E7AD1EAAB22146484605F024FC38F8B2
:1085A000021C88425BD1ADB21349B80702D5888955
:1085B000401C00E001201FFA80F8F80701D08F89E5
:1085C00000E04F4605AA4146584605F022FA4FF012
:1085D000070A4FF00009D4B3204608E0408810286D
:1085E0003DD8361D304486B2AE4238D2A01902883A
:1085F0004245F3D353E00000280300209DF8170004
:1086000002074CD594B304EB0608361DB8F80230C7
:10861000B6B2102B23D89A19AA4220D8B8F8002055
:1086200091421CD1C0061CD5CDE900A90DF1080C62
:108630000AAAA11948468CE80700B8F800100022E1
:10864000584605F06FF820B1FEF709FA83E726E0F7
:1086500005E0B8F80200BDF82810884201D00B20D0
:1086600079E7B8F80200304486B207E0FFE7C006B9
:1086700004D55846FEF772FC002889D19DF81700F2
:10868000BDF81A1020F010008DF81700BDF8170083
:10869000ADF80000FF235846009A05F01BFB05A823
:1086A00005F0C3F918B9BDF81A10B942A6D90421CA
:1086B000584607F00DFF040000D1FFDFA2895AB130
:1086C000CDE900A94D46002321465846FEF714FC8B
:1086D0000028BBD1A5813EE700203CE72DE9FF4FF4
:1086E0008BB01E4617000D464FF0000412D0B008A4
:1086F00002D007200FB0C1E4032E00D100265DB1E7
:1087000008460BF077FA28B93888691E08440BF040
:1087100071FA08B11020EDE7C64AB00701D5D1893A
:1087200000E00121F0074FF6FF7802D0D089401E0B
:1087300000E0404686B206AA0B9805F06AF94FF0B1
:1087400000094FF0070B0DF1140A38E09DF81B00EB
:10875000000734D5CDF80490CDF800B0CDF80890DE
:10876000CDE9039A434600220B9805F005FA60BB59
:1087700005B3BDF814103A8821442819091D8A420E
:1087800030D3BDF81E2020F8022BBDF8142020F8AD
:10879000022BCDE900B9CDE90290CDF810A0BDF8CB
:1087A0001E10BDF8143000220B9805F0E5F908B151
:1087B00003209FE7BDF814002044001D84B206A8E2
:1087C00005F033F920B1822806D0FEF748F991E789
:1087D000BDF81E10B142B9D934B17DB13888A11CA1
:1087E000884203D20C2085E7052083E722462946EC
:1087F000404605F0F8FA014628190180A41C3C8087
:10880000002077E710B504460BF0D6F908B1102028
:1088100010BD8848C0892080002010BDF0B58BB005
:108820000D460646142103A81BF005F901208DF81A
:108830000C008DF8100000208DF81100ADF81450D8
:108840003046FAF74EFC48B10078222812D30421B2
:10885000304607F03DFE040005D103E043F202007C
:108860000BB0F0BDFFDF04F11400074603F089FFF1
:10887000800601D40820F3E7207C022140F00100AB
:10888000207409A80094CDE90110072203A93046FD
:108890006368FEF7E7FA20B1217C21F00101217421
:1088A000DEE729463046F9F77DFD08A9384603F092
:1088B00057FF00B1FFDFBDF82040172C01D2172071
:1088C00000E02046A84201D92C4602E0172C00D235
:1088D000172421463046FFF722FB21463046F9F7A0
:1088E00083FA0020BCE7F8B51C4615460E46069FE5
:1088F00007F020FF2346FF1DBCB231462A460094F4
:1089000007F009FBF8BD70B50C4605460E21204660
:108910001BF06FF8002020802DB1012D01D0FFDF6A
:1089200070BD062000E00520A07170BD10B5488024
:108930000878134620F00F00001D20F0F000803072
:108940000C4608701422194604F108001BF017F8B1
:1089500000F0A5FC3748046010BD2DE9F047DFF8B2
:10896000D890491D064621F0030117460C46D9F858
:10897000000007F0E6FB050000D1FFDF4FF0000824
:108980003560A5F800802146D9F8000007F0D9FB32
:10899000050000D1FFDF7560A5F800807FB104FB02
:1089A00007F1091D0BD0D9F8000007F0CAFB04003D
:1089B00000D1FFDFB460C4F80080BDE8F087C6F8DE
:1089C0000880FAE72DE9F0411746491D21F003021E
:1089D000194D064601681446286807F0DDFB22465B
:1089E0007168286807F0D8FB3FB104FB07F2121D3D
:1089F00003D0B168286807F0CFFB042007F010FD12
:108A00000446042007F014FD201A012804D1286828
:108A1000BDE8F04107F08ABBBDE8F08110B50C4617
:108A200004F0C3FF00B1FFDF2046BDE81040FEF7B1
:108A300016B80000280300201400002038B50C46AA
:108A4000817B828819B14189914200D90A462280EE
:108A5000C188121D90B26A4606F0CCFEBDF8000037
:108A6000032800D30320C1B2208800F075FF38BD71
:108A700038B50C46817B828819B10189914200D9B1
:108A80000A462280C188121D90B26A4606F0B2FEE4
:108A9000BDF80000022800D30220C1B2208800F0F7
:108AA0005BFF401CC0B238BD2DE9FF5F0C46FF499B
:108AB00081463C22D1E90201CDE9020109F103001E
:108AC00020F00301C91C21F0030100916846114602
:108AD00007F019FBF64E002C02D1F649009A8A6085
:108AE000009901440091357E05F1010504D1E8B2F9
:108AF00009F088F800B1FFDF00984FF0000B00EBA1
:108B00000510C01C20F0030100915CB9707A327A24
:108B100081F800B01044C2B2B08B80B204F0CDFD39
:108B200000B1FFDF0098F1690844009021466846D3
:108B300000F0DCFE0098C01C20F003000090737A67
:108B4000327AB17A04B1002007F0D3FB00990844CF
:108B500000902146684600F00AFF00273D46B246D5
:108B600096F801800CE0284600F0A3FE06468178C6
:108B70008088F9F7D0F971786D1C00FB0177EDB2B0
:108B80004545F0D10098C01C20F00300009004B1CE
:108B900000203946F9F7CAF90099002708440090E7
:108BA0003D469AF801800CE0284600F082FE064619
:108BB000C1788088FEF75DFC71786D1C00FB017741
:108BC000EDB24545F0D10098C01C20F003000090A4
:108BD00004B100203946FEF755FC00994FF000081B
:108BE0000844009045469AF801700EE0284600F0CF
:108BF00060FE0646807B30B106F1080001F0C9FE38
:108C0000727800FB02886D1CEDB2BD42EED1009877
:108C1000C01C20F00300009004B10020414601F088
:108C2000BCFE00990844C01D20F007000090ECBB7A
:108C3000A24AA1491160111D401E086005F09EF86E
:108C40009C484178C06805F073F99A481030C078A4
:108C50008DF8040010B1012804D005E001208DF842
:108C6000040001E08DF804B001A805F0CBFBFBF790
:108C700093F98F4802AA00210C30F8F76BFB00B182
:108C8000FFDF9AF81900FEF766FF00B1FFDF8848A2
:108C90004FF4F67144301AF0CEFE8548042144307A
:108CA00080F8E91180F8EA11062100E003E080F87D
:108CB000EB1103210171009904B0A1EB0900BDE89B
:108CC000F09F70B57A4C06464434207804EB40158A
:108CD000E078083590B9A01990F8E80100280ED086
:108CE000A0780F2800D3FFDF202128461AF0A3FE2A
:108CF000687866F3020068700120E070284670BD55
:108D00002DE9F04105460C460027007805219046E4
:108D10003E46B1EB101F00D0FFDF287A50B101288A
:108D20000ED0FFDFA8F800600CB12780668000201D
:108D3000BDE8F0810127092674B16888A08008E0A9
:108D40000227142644B16888A0802869E060A88AB8
:108D50002082287B2072E5E7A8F80060E7E710B5DD
:108D6000544C6068C11D21F00701814200D0FFDF33
:108D70004F480121002201704270017203234372A7
:108D800081720273052282821F22C28241734CA229
:108D900002610A22027641764FF4B061C1616168D6
:108DA000416010BD30B5434C1568636810339D4277
:108DB00002D20420136030BD3D4B5D785A6802EB4F
:108DC0000512107051700320D08017209080012070
:108DD000D0709070002090735878401C5870606874
:108DE00010306060002030BD70B506463048002469
:108DF000457807E0204600F05CFD0178B14204D0E0
:108E0000641CE4B2AC42F5D1002070BDF7B5064653
:108E100008780C4608B3FFF7E7FF0546202E08D078
:108E2000232E17D0212E31D0222E2FD0242E2BD11D
:108E300014E000F049FD0DB1697800E00021401A0E
:108E400081B2A0780144FF291ED830B1A088022841
:108E50001CD219E06088172818D215E0227AAAB12E
:108E60006188172910D3A08817280DD3A3795BB187
:108E7000E3794BB1402A07D84FF6FB72914201D8F3
:108E8000904203D90420FEBD0720FEBD65B92078BD
:108E900002AA0121FFF786FF0028F6D12078FFF70C
:108EA000A3FF050000D1FFDF203E0DE0C43D02001E
:108EB000440400201C0000200000002000060240A6
:108EC0006E52463578000000052E18D2DFE806F015
:108ED000030B0E081100A0786870A088E8800FE0EE
:108EE0006088A8800CE0A078A87009E0A078E870FD
:108EF00006E054F8020FA8606068E86000E0FFDF59
:108F00000020FEBD1E2829D00EDC0C2822D008DC53
:108F1000092825D2DFE800F013241524241C1C188E
:108F20001A0012281CD119E0302817D018DDA0F142
:108F30003A00032814D2DFE800F00F1309000020E4
:108F4000704743F202007047042070470D207047BD
:108F50000F20704708207047112070470720704786
:108F60000320704710B5007800F0010006F039FCCE
:108F7000BDE81040C6E70EB5017801F001018DF89B
:108F80000010417801F001018DF801100178C1F362
:108F900040018DF802104178C1F340018DF80310B3
:108FA000017889088DF80410417889088DF805103A
:108FB00081788DF80610C1788DF8071000798DF84A
:108FC0000800684605F045FAFFF79CFF0EBD2DE945
:108FD000F84FDFF8F883FE4C00261FE0012000F078
:108FE00009FD0120FFF76DFE05463C214746D8F8F4
:108FF000080007F0A6F8686000B9FFDF686804F0B1
:10900000EAFFA8B12846FAF70EFB284600F0F8FC64
:1090100020B93C226968B86807F0BEF894F9E90104
:109020000428DBDA022007F0FBF907460025A6E05A
:109030003C226968D8F8080007F0AEF8F2E7B8F803
:1090400002104046491C89B2A8F80210B94201D367
:10905000002141800221B8F8020007F039FA002807
:1090600065D0B8F80200694606F02DFBFFF74AFF0D
:1090700000B1FFDF9DF8000078B1B8F8020007F0FA
:109080006BFB5FEA000900D1FFDF484606F0D7FD21
:1090900018B1B8F8020002F023F9B8F8020007F09E
:1090A00049FB5FEA000900D1FFDF484606F0BFFD3B
:1090B000E8BB0321B8F8020007F00AFA5FEA000BE8
:1090C00048D1FFDF46E000BFDBF8100010B10078A8
:1090D000FF2849D0022000F08DFC0220FFF7F1FDAF
:1090E0008246484606F0AFFECAF8040000B9FFDF2A
:1090F000DAF8040006F077FF002100900170B8F85C
:1091000002105046AAF8021001F0F0FD484606F0A1
:109110006CFF00B9FFDF504600F072FC18B99AF8F6
:109120000100000704D50099CBF8101012E024E0EC
:10913000DBF8100038B10178491C11F0FF01017013
:1091400008D1FFDF06E000221146484600F0AFFBE1
:1091500000B9FFDF94F9EA01022805DBB8F8020044
:1091600001F088FD0028AFD194F9E901042804DB5F
:10917000484606F09EFF00B101266D1CEDB2BD42CF
:1091800004D294F9EA010228BFF659AF002E7FF409
:1091900023AFBDE8F84F032000F02CBC10B58B4C7A
:1091A000E06008682061AFF2D910F9F7A2FE6070A4
:1091B00010BD8748002144380170844801708549FA
:1091C0004160704770B505464FF080500C46D0F8AE
:1091D000A410491C05D1D0F8A810C9430904090CF2
:1091E0000BD050F8A01F01F00101297041682160E7
:1091F0008068A080287830B970BD062120460AF02A
:109200008CF901202870607940F0C000607170BD59
:1092100070B54FF080540D46D4F88010491C0BD126
:10922000D4F88410491C07D1D4F88810491C03D104
:10923000D4F88C10491C0CD0D4F880100160D4F8FC
:1092400084104160D4F888108160D4F88C10C1601B
:1092500002E010210AF061F9D4F89000401C0BD113
:10926000D4F89400401C07D1D4F89800401C03D1D6
:10927000D4F89C00401C09D054F8900F2860606816
:109280006860A068A860E068E86070BD2846BDE836
:10929000704010210AF041B94D48007911E570B5D0
:1092A0004B4CE07830B3207804EB4010407A00F06B
:1092B0000700204490F9E801002800DCFFDF207857
:1092C000002504EB4010407A00F00700011991F8E6
:1092D000E801401E81F8E8012078401CC0B22070EF
:1092E0000F2800D12570A078401CA0700AF050F81B
:1092F000E57070BDFFDF70BD3EB50546032107F088
:10930000E7F80446284607F015FA054604B9FFDFDA
:10931000206918B10078FF2800D1FFDF01AA694653
:10932000284600F0C4FA60B9FFDF0AE0002202A973
:10933000284600F0BCFA00B9FFDF9DF8080000B134
:10934000FFDF9DF80000411E8DF80010EED220696D
:109350000199884201D1002020613EBD70B50546CB
:10936000A0F57F400C46FF3800D1FFDF012C01D073
:10937000FFDF70BDFFF790FF040000D1FFDF207812
:1093800020F00F00401D20F0F0005030207065806C
:109390000020207201202073BDE870407FE72DE996
:1093A000F04116460D460746FFF776FF040000D150
:1093B000FFDF207820F00F00401D20F0F00050303B
:1093C0002070678001202072286805E01C000020C2
:1093D00088040020C81300202061A888A08226737A
:1093E000BDE8F0415BE77FB5FFF7FEFC040000D16C
:1093F000FFDF02A92046FFF721FB054603A920460F
:10940000FFF736FB8DF800508DF80100BDF808001D
:10941000001DADF80200BDF80C00001DADF8040001
:10942000E088ADF80600684606F0C4F9002800D0D0
:10943000FFDF7FBD2DE9F047DFF8FC9305460027ED
:1094400099F8000010B10820BDE8F08728460AF01E
:10945000B3FB08B11020F7E7F84C207808B9FFF704
:109460007EFC607A217A0844C6B200F02DFAB04240
:1094700007D2301AC1B22A460020FFF793FC07003A
:10948000E2D1D9F804004E46C01C20F00300C9F810
:10949000040000F01DFB716800EB0108012140464B
:1094A000FFF702FB064629684044884202D8B6F519
:1094B000803F15D328600020FFF796FC05000DD0F3
:1094C00005F11300D9F8041020F003004E4688423D
:1094D00000D0FFDF6078401E607075600420B3E745
:1094E00000214046FFF7E0FA0446A64200D0FFDF25
:1094F00004EB0801C9F8041029604FF6FF71A9F8C0
:109500000210012189F8001038469DE72DE9F0414D
:109510000446C94817460E46007808B1082007E4FB
:1095200008460AF023FB08B11020F8E7C34D28785D
:1095300008B9FFF714FC601E1E2807D8012C22D1A1
:109540003078FE281FD828760020E8E7A4F1200014
:109550001F2805D8E0B23A463146BDE8F04155E44F
:10956000A4F140001F2805D831462046BDE8F0414F
:1095700000F06EBAA4F1A0001F2804D80020A02C8F
:1095800003D0A12C06D00720C9E7317801F00101F2
:109590006976C4E731680922F82901D38B0701D025
:1095A0001046BCE76B7B03F00303012B04D1EB8A6D
:1095B000D7339CB28C42F3D8E961B0E72DE9F0478C
:1095C00081460E4608460AF0F7FA48B948460AF0BE
:1095D00011FB28B909F1030020F00301494501D02E
:1095E000102031E795484FF0000A4430817869B186
:1095F0004178804600EB4114083437883246002118
:10960000204600F00BFA050004D027E0A6F800A0E1
:10961000052019E7B9F1000F24D03088B84201D9EC
:109620000C251FE0607800F00705284600F0E2F9FD
:1096300008EB0507324697F8E8014946401C87F8D1
:10964000E801204607F5F47700F0E8F90546387898
:10965000401E3870032000F0CDF92DB10C2D01D043
:10966000A6F800A02846EFE66078734E00F00701E8
:10967000012923D002290CD0032933D0FFDF98F829
:1096800001104046491CC9B288F801100F2934D096
:1096900035E0616821B1000702D46088FFF72CFE35
:1096A00098F8EA014746012802D17078F9F740FCA2
:1096B00097F9EA010428E2DBFFDFE0E7616819B10E
:1096C0003C22B06806F068FD98F8E9014746032897
:1096D00002D17078F9F72CFC97F9E9010428CEDB68
:1096E000FFDFCCE7C00602D56088FFF705FE98F9DA
:1096F000EB010628C3DBFFDFC1E780F801A081781A
:10970000491E8170617801F0070101EB080090F8B3
:10971000E811491C80F8E811A4E770B50D4604462D
:109720000AF024FA18B928460AF046FA08B11020BF
:1097300070BD29462046BDE8704008F09ABA70B561
:10974000044615460E4608460AF010FA18B928468F
:109750000AF032FA08B1102070BD022C03D0102C90
:1097600001D0092070BD2A463146204608F0A4FAEF
:109770000028F7D0052070BD70B514460D4606468A
:109780000AF0F4F938B928460AF016FA18B9204652
:109790000AF030FA08B1102070BD22462946304642
:1097A00008F0A9FA0028F7D0072070BD3EB504469E
:1097B0000AF002FA08B110203EBD684604F0A9FD87
:1097C000FFF7A0FB0028F7D19DF806002070BDF838
:1097D00008006080BDF80A00A08000203EBD70B582
:1097E00005460C4608460AF005FA20B93CB1206847
:1097F0000AF0E2F908B1102070BDA08828B1214616
:109800002846BDE87040FDF7B3BE092070BD70B5B5
:1098100004460D4608460AF0A9F930B9601E1E2814
:1098200019D828460AF0A2F908B1102070BD022C00
:1098300006D9072070BD00001C0000204404002051
:1098400004B9FFDFF74800EB840050F8041C2846F9
:10985000BDE870400847A4F120001F28E9D8294638
:109860002046BDE87040FAF70BBB70B504460D46C4
:1098700008460AF0A1F930B9601E1E280DD8284606
:109880000AF074F908B11020D4E7012C01D0022CA1
:1098900001D10620CEE70720CCE7A4F120001F2845
:1098A000F9D829462046BDE87040FAF748BB06F0D3
:1098B0008DB930B5DC4D04466878A04200D8FFDF92
:1098C000686800EB041030BD70B5D74800252C4601
:1098D000467807E02046FFF7ECFF4078641C2844F8
:1098E000C5B2E4B2B442F5D12846A3E72DE9F04170
:1098F0000C46064600F024F907463068C01C20F0EC
:10990000030232601CBBC8483B46092120300AF0E4
:1099100007F8002408E0092C11D2DFE804F005075D
:109920000509090B05050700C04804E0C04802E02E
:10993000C04800E0C0480AF013F8054600E0FFDF29
:10994000A54200D0FFDF641CE4B2092CE3D33068E9
:1099500000EB07103060E2E5021D5143452900D2BB
:1099600045210844C01CB0FBF2F0C0B270472DE99D
:10997000FC5F0646AC484FF000088B46474644461D
:1099800090F8019022E02046FFF793FF050000D1F8
:10999000FFDF687869463844C7B22846FFF74EF8BB
:1099A000824601A92846FFF763F80346BDF8040084
:1099B0005246001D81B2BDF80000001D80B206F0C5
:1099C00005FE6A78641C00FB0288E4B24C45DAD1DB
:1099D0003068C01C20F003003060BBF1000F00D0E5
:1099E00000204246394606F0FFFD316808443060E9
:1099F000BDE8FC9F8C49443108710020C870704755
:109A000089494431CA782AB10A7801EB42110831F8
:109A1000814201D001207047002070472DE9F041BC
:109A200006460078154600F00F0400201080601EE6
:109A30000F46052800D3FFDF7A482A46103000EB96
:109A40008400394650F8043C3046BDE8F0411847E0
:109A500070B50C46402804D0412823D0422806D1B6
:109A60001BE0607821784518A178814201D9072050
:109A7000E0E6FF2D08D808F0A9FA064609F042FCF6
:109A8000301A801EA84201DA1220D3E666482188E7
:109A90000181A17881720020CCE6BDE870400846C3
:109AA00000F07FB8062508460AF060F8102618B9BD
:109AB00020680AF05BF808B13046BBE62068017800
:109AC000FF2903D10AF096F80028F5D12846B1E61F
:109AD0002DE9F05F4FF000095348C8464F464E4607
:109AE0004D46CB464C4690F801A011E02046FFF7CA
:109AF000E0FE4178827809F10109884412FB017780
:109B0000C27812FB0166807B10FB0155641CE4B235
:109B10005445EBD10BEB890000EBC80000EB87004C
:109B200000EB860000EBC5013F48027A01EBC20161
:109B3000427A807A01EBC20101EBC000BDE8F09FE0
:109B40002DE9F047DFF8E09000252C4699F8092030
:109B500099F8081099F801700A44D6B299F80A20C9
:109B6000114401F0FF0808E02046FFF7A2FE817BC8
:109B7000407811FB0055641CE4B2BC42F4D199F862
:109B80000800401C304430444044401C0EB10121C8
:109B900000E0002108444419FF2C00D9FFDFE0B2A7
:109BA00052E438B50446407800F00300012803D0A1
:109BB00002280BD0072038BD606858B10AF023F89E
:109BC000D0B960680AF016F820B915E0606809F0AD
:109BD000CDFF88B969462046FCF758F90028EAD13C
:109BE000607800F00300022808D19DF8000028B139
:109BF000606809F0FFFF08B1102038BD6189F829BD
:109C00000DD8208988420AD8607800F003020648FF
:109C1000012A13D1D731C26989B28A420ED20920F2
:109C200038BD0000C43D020044040020113D000086
:109C300065AA0000DD2F0000D319010094E80E0092
:109C400000F10C0585E80E000AB900218182002090
:109C5000E6E700002DE9F04107461446884608462D
:109C600001F020FD064608EB88001C22796802EB13
:109C7000C0000D18688C58B14146384601F01AFDF5
:109C8000014678680078C200082305F120000CE046
:109C9000E88CA8B14146384601F013FD01467868CA
:109CA00008234078C20005F1240006F0CCFA38B150
:109CB000062121726681D0E90010C4E9031009E091
:109CC000287809280BD00520207266816868E0603A
:109CD000002028702046BDE8F04101F0D9BC0720E3
:109CE00020726681F4E72DE9F04116460D460746DD
:109CF000406801EB85011C2202EBC101441820469B
:109D000001F001FD40B10021708865F30F2160F37F
:109D10001F41082009F0DEFE092020703246294646
:109D20003846BDE8F04195E72DE9F0410E4607467B
:109D300000241C21F07816E004EB8403726801EB28
:109D4000C303D25C6AB1FFF7A7FA050000D1FFDFB9
:109D50006F802A4621463046FFF7C5FF0120BDE847
:109D6000F081641CE4B2A042E6D80020F7E770B5A9
:109D7000064600241C21C0780AE000BF04EB8403DF
:109D8000726801EBC303D5182A782AB1641CE4B2C7
:109D9000A042F3D8402070BD2821284619F029FEA2
:109DA000706880892881204670BD70B50346002008
:109DB0001C25DC780DE000BF00EB80065A6805EB3F
:109DC000C6063244167816B1128A8A4204D0401C64
:109DD000C0B28442F0D8402070BDF0B504460020E7
:109DE0001C26E5780EE000BF00EB8007636806EBF9
:109DF000C7073B441F788F4202D15B78934204D05F
:109E0000401CC0B28542EFD84020F0BD0078032846
:109E100001D000207047012070470078022801D04F
:109E200000207047012070470078072801D00020EB
:109E30007047012070472DE9F041064688461078AA
:109E4000F1781546884200D3FFDF2C781C27641C6C
:109E5000F078E4B2A04201D8201AC4B204EB840125
:109E6000706807EBC1010844017821B14146884779
:109E700008B12C7073E72878A042E8D14020287000
:109E80006DE770B514460B880122A240134207D13A
:109E900013430B8001230A22011D06F09EF9047072
:109EA00070BD2DE9FF4F81B00878DDE90E7B9A4641
:109EB00091460E4640072CD4019806F04DFC040054
:109EC00000D1FFDF07F1040820461FFA88F105F0F2
:109ED00088FD050000D1FFDF204629466A4605F0CF
:109EE000D4FF0098A0F80370A0F805A0284606F05B
:109EF0007AF8017869F306016BF3C7110170204607
:109F00001FFA88F105F0B0FD00B9FFDF019803F0FA
:109F100083FF06EB0900017F491C017705B0BDE80E
:109F2000F08F2DE9F84F0E469A46914607460321D9
:109F300006F0CEFA0446008DDFF8B485002518B18E
:109F400098F80000B0421ED1384606F005FC070024
:109F500000D1FFDF09F10401384689B205F041FD67
:109F6000050010D0384629466A4605F08EFF009855
:109F700000210A460180817004F01AF80098C01D83
:109F8000CAF8000021E098F80000B04216D104F1B0
:109F9000260734F8341F012000FA06F911EA090FE8
:109FA00000D0FFDF2088012340EA090020800A2238
:109FB000391D384606F02CF9067006E0324604F1E9
:109FC000340104F12600FFF75CFF0A2188F8001035
:109FD0002846BDE8F88FFEB514460D46064602AB8E
:109FE0000C220621FFF79DFF002826D002996878F1
:109FF00012220A70801C487008224A80A8702088AB
:10A0000088806088C880A0880881E0884881002412
:10A010000C20CDE900040523062229463046FFF72F
:10A0200040FF214666F31F41F0230022012009F082
:10A03000A7FC6878801C68700120FEBDFEB5144640
:10A040000D460622064602AB1146FFF76AFF0028BE
:10A0500012D0029B132000211870A878587002209B
:10A0600058809C800620CDE9000102460523294640
:10A070003046FFF716FF0120FEBD2DE9FE430C46DA
:10A08000804644E002AB0E2207214046FFF749FF1D
:10A09000002841D060681C2267788678BF1C06EBD8
:10A0A000860102EBC1014518029814210170477026
:10A0B0000A214180698A0181E98A4181A9888180D8
:10A0C000A9898181304601F0EDFA02990523072222
:10A0D000C8806F700420287000250E20CDE900058F
:10A0E00021464046FFF7DDFE294666F30F2168F35F
:10A0F0001F41F0230022082009F042FC6078FD494E
:10A10000801C607062682046921CFFF794FE6068B5
:10A1100080784028B6D10120BDE8FE83FEB50D460B
:10A12000064638E002AB0E2207213046FFF7F9FE63
:10A13000002835D068681C23C17801EB810203EB4D
:10A14000C2028418029815220270627842700A22B4
:10A150004280A2894281A2888281084601F0A2FA47
:10A16000014602988180618AC180E18A0181A088CC
:10A17000B8B10020207000210E20CDE90001052398
:10A18000072229463046FFF78CFE6A68DA492846DE
:10A19000D21CFFF750FE6868C0784028C2D1012069
:10A1A000FEBD0620E6E72DE9FE430C46814644E06D
:10A1B000204601F092FAD0B302AB082207214846AC
:10A1C000FFF7AFFE0028A7D060681C2265780679EB
:10A1D000AD1C06EB860102EBC10147180298B7F8E7
:10A1E000108006210170457004214180304601F045
:10A1F00059FA0146029805230722C180A0F804807D
:10A200007D70082038700025CDE9000521464846BC
:10A21000FFF747FE294666F30F2169F31F41F0233C
:10A220000022082009F0ACFB6078801C6070626836
:10A23000B2492046121DFFF7FEFD606801794029F2
:10A24000B6D1012068E72DE9F34F83B00E4680E0D8
:10A25000304601F042FA002875D071681C2091F850
:10A26000068008EB880200EBC2000C18414630461D
:10A2700001F027FA0146A078C30070684078C20058
:10A2800004F1240005F0FBFF07468088E18B401AAB
:10A2900080B2002581B3AA46218B814200D80846AE
:10A2A0008146024602AB07210398FFF73AFE010000
:10A2B00028D0BAF1000F03D0029AB8880225108086
:10A2C0008B46E28B3968A9EB05001FFA80FA0A4435
:10A2D0000398009206F040FAED1D009A5946534645
:10A2E000009505F04CFEE08B504480B2E083B988C5
:10A2F000884209D1012508E0FFE7801C4FF0010AE0
:10A3000080B2C9E7002009E60025CDE90095238A3F
:10A31000072231460398FFF7C4FDE089401EE08123
:10A320008DB1A078401CA0707068F178427811FB64
:10A3300002F1CAB2816901230E3005F04EFF80F8A8
:10A3400000800020E08372686D493046921DFFF75F
:10A3500072FD7068817940297FF47AAF0120DDE5D4
:10A3600070B5064648680D4614468179402910D1DB
:10A3700004EB84011C2202EBC101084401F0E4F962
:10A38000002806D06868294684713046BDE87040D0
:10A3900059E770BDFEB50C460746002645E020464D
:10A3A00001F09BF9D8B360681C22417901EB81016F
:10A3B00002EBC1014518688900B9FFDF02AB082232
:10A3C00007213846FFF7ADFD002833D002996078A9
:10A3D00016220A70801C487004204880606840790A
:10A3E00001F060F9014602980523072281806989FE
:10A3F000C1800820CDE9000621463846FFF751FD0F
:10A400006078801C6070A88969890844B0F5803F35
:10A4100000D3FFDFA88969890844A8816E8162683A
:10A4200038492046521DFFF706FD606841794029F2
:10A43000B5D10120FEBD30B5438C458BC3F3C704B5
:10A44000002345B1838B641EED1AC38A6D1E1D4423
:10A4500095FBF3F3E4B22CB1008918B1A04200D807
:10A46000204603444FF6FF70834200D30346138017
:10A470000C7030BD2DE9FC41074616460D46486874
:10A4800002EB86011C2202EBC10144186A4601A9B5
:10A490002046FFF7D0FFA089618901448AB2BDF848
:10A4A0000010914212D0081A00D50020608168681F
:10A4B000407940280AD1204601F03CF9002805D017
:10A4C0006868294646713846FFF764FFBDE8FC819D
:10A4D0002DE9FE4F8946804615465088032105F038
:10A4E000F7FF8346B8F8020040280DD240200CE068
:10A4F000300000200D9E00001B9E0000299E0000E1
:10A5000049B7000035B70000403880B282460146A6
:10A51000584601F0E2F800287ED00AEB8A001C229F
:10A52000DBF8041002EBC0000C18204601F0EBF839
:10A53000002877D1B8F80000E18A88423CD8A18988
:10A54000D1B348456ED100265146584601F0B2F8C5
:10A55000218C0F18608B48B9B9F1020F62D3B8F89B
:10A5600004006083618A884226D80226A9EB06008F
:10A570001FFA80F9B888A28B801A002814DD49469A
:10A58000814500DA084683B26888696802913968B3
:10A590000A44CDE9003206F0CDF8DDE90121F61DCF
:10A5A000009B009605F0B7FCA18B01EB090080B27F
:10A5B000A083618B884207D9688803B05246594608
:10A5C000BDE8F04F01F0DDB81FD14FF0090028724F
:10A5D000B8F802006881D7E90001C5E90401608B81
:10A5E000A881284601F054F85146584601F062F817
:10A5F0000146DBF8040008230078C20004F12000C3
:10A6000005F021FE0020A0836083A0890AF0FF02EC
:10A61000401EA081688800E004E003B05946BDE810
:10A62000F04F27E7BDE8FE8F2DE9F04106461546BD
:10A630000F461C46184609F099FA18B9206809F027
:10A64000BBFA08B1102015E47168688C0978B0EB8A
:10A65000C10F01D313200DE43946304601F02AF82A
:10A660000146706808230078C20005F1200005F05B
:10A67000B4FDD4E90012C0E900120020E3E710B5F0
:10A680000446032105F024FF0146007800F0030092
:10A69000012804D08A8A2046BDE81040CEE4204636
:10A6A000BDE8104001F1140295E470B504460321A1
:10A6B00005F00EFF054601462046FFF774FD002811
:10A6C00016D029462046FFF765FE002810D02946FF
:10A6D0002046FFF723FD00280AD029462046FFF731
:10A6E000CCFC002804D029462046BDE87040AAE5ED
:10A6F00070BD2DE9F0410C4680461EE0E1784278BD
:10A7000011FB02F1CAB2816901230E3005F09BFDF5
:10A71000077860681C22C179491EC17107EB870167
:10A72000606802EBC10146183946204600F0D5FFAB
:10A7300018B1304600F0E0FF20B16068C17900290F
:10A74000DCD180E7FEF7A8FD050000D1FFDF0A207D
:10A750002872384600F0A6FF68813946204600F08E
:10A76000B0FF0146606808234078C20006F124006B
:10A7700005F069FDD0E90010C5E90310A5F80280D5
:10A78000284600F085FFB07800B9FFDFB078401EA2
:10A79000B07058E770B50C460546032105F098FEE9
:10A7A00001464068C2792244C2712846BDE8704023
:10A7B0009FE72DE9FE4F8246507814460F464FF032
:10A7C000000800284FD0012807D0022822D0FFDF40
:10A7D0002068B8606068F86024E702AB0E220821A8
:10A7E0005046FFF79EFB0028F2D002981521052362
:10A7F0000170217841700A214180C0F80480C0F8BE
:10A800000880A0F80C80628882810E20CDE90008C3
:10A81000082221E0A678304600F044FF054606EB0A
:10A8200086012C22786802EBC1010822465A02AB4D
:10A8300011465046FFF775FB0028C9D00298072142
:10A840000170217841700421418008218580C680F3
:10A85000CDE9001805230A4639465046FFF721FB8B
:10A8600087F80880DEE6A678022516B1022E13D0FE
:10A87000FFDF2A1D914602AB08215046FFF751FB2E
:10A880000028A5D002980121022E01702178417084
:10A890004580868002D005E00625EAE7A188C180D0
:10A8A000E1880181CDE90098052308223946504608
:10A8B000D4E710B50446032105F00AFE014600F175
:10A8C00008022046BDE8104073E72DE9F05F0C4612
:10A8D00001281DD0957992F80480567905EB850101
:10A8E0001F2202EBC10121F0030B08EB060111FB53
:10A8F00005F14FF6FF7202EAC10909F1030115FBE8
:10A900000611F94F21F0031A40B101283DD124E08E
:10A910006168E57891F800804E78DFE759467868FD
:10A9200005F00FFC606000B9FFDF5946606819F060
:10A9300082F8E5705146786805F003FC616848616B
:10A9400000B9FFDF6068426902EB0901816160685C
:10A9500080F800806068467017E060685246416980
:10A96000786805F019FC5A466168786805F014FCAF
:10A97000032005F055FD0446032005F059FD201A7B
:10A98000012802D1786805F0D1FB0BEB0A00BDE885
:10A99000F09F02460021022097E713B5009858B1B6
:10A9A0000024684605F0AFFBCF490A22002C0A704C
:10A9B00001D1009A4A601CBD01240020F2E770B565
:10A9C0000C4615463821204619F035F801266670E8
:10A9D0000A2104F11C0019F02EF805B9FFDF297ACD
:10A9E000207861F301002070A879002817D02A464A
:10A9F00021460020FFF769FF616840208870616888
:10AA0000C8706168087161684871616888716168BF
:10AA1000288808816168688848816068868170BD7F
:10AA2000C878002802D0002201204EE7704770B598
:10AA30000546002165F31F41012009F04BF8032171
:10AA4000284605F045FD040000D1FFDF21462846D9
:10AA5000FFF76AF9002804D0207840F01000207039
:10AA6000012070BD2DE9FF4180460E460F0CFEF718
:10AA700013FC050007D06F800321384605F028FD40
:10AA8000040008D106E004B03846BDE8F0411321C7
:10AA9000F9F750BEFFDFB8F1010F05D0B8F1080F8C
:10AAA00018D0FFDFBDE8FF8120782A4620F008009B
:10AAB00020700020ADF8020002208DF800004FF653
:10AAC000FF70ADF80400ADF8060069463846F9F7A6
:10AAD00083F9E7E7C6F3072101EB81021C236068D5
:10AAE00003EBC202805C042803D008280AD0FFDFF1
:10AAF000D8E7012000904FF440432A46204600F05A
:10AB000009FECFE704B02A462046BDE8F041FFF732
:10AB1000EAB82DE9F05F0027B0F80A9090460C469D
:10AB200005463E46B9F1400F01D2402001E0A9F1AF
:10AB300040001FFA80FA287AC01E08286BD2DFE88E
:10AB400000F00D04192058363C4772271026002CBF
:10AB50006CD0D5E90301C4E902015CE0702712263C
:10AB6000002C63D00A2205F10C0104F1080018F052
:10AB700006FF50E071270C26002C57D0E868A06033
:10AB800049E0742710269CB3D5E90301C4E902010A
:10AB90006888032105F09CFC8346FEF77DFB024696
:10ABA0006888508051465846FFF754F833E07527BF
:10ABB0000A26ECB1A88920812DE076271426BCB1A5
:10ABC00005F10C0004F1080307C883E8070022E040
:10ABD0007727102664B1D5E90301C4E9020168882A
:10ABE000032105F075FC01466888FFF782FD12E03D
:10ABF0001CE073270826CCB16888032105F068FCA7
:10AC000001460078C00606D56888FFF78DF810B9B0
:10AC10006888F8F7ECFCA8F800602CB12780A4F84D
:10AC2000069066806888A0800020B0E6A8F80060E2
:10AC3000FAE72DE9FC410C461E46174680460321E3
:10AC400005F046FC05460A2C0AD2DFE804F00505AB
:10AC50000505050509090907042303E0062301E0AA
:10AC6000FFDF0023CDE90076224629464046FFF764
:10AC700018F92BE438B50546A0F57F40FF3830D0F1
:10AC8000284605F057FD040000D1FFDF204605F0FF
:10AC9000DAF8002815D001466A46204605F0F5F896
:10ACA00000980321B0F80540284605F011FC054640
:10ACB000052C03D0402C05D2402404E0007A80B15A
:10ACC000002038BD403CA4B2214600F006FD40B152
:10ACD000686804EB84013E2202EBC101405A00285F
:10ACE000EFD0012038BD0000300000202DE9F04FEA
:10ACF000044689B0408805F01DFD050000D1FFDF46
:10AD000006AA2846616800F0C1FC069D001F81B2BA
:10AD100035F8032F6B888A4205D1042B0AD0052B06
:10AD20001DD0062B15D022462846FFF7D1FB09B0CF
:10AD3000BDE8F08F16462D1D224629463046F7F70E
:10AD40001BFB0828F3D1224629463046FCF757FC66
:10AD5000EDE76088291D6368FAF714FDE7E71746F9
:10AD60006088032105F0B4FB4FF000088DF80480E3
:10AD70000646ADF80680042FD9D36A79002AD6D0CA
:10AD800028794FF6FF794FF01C0A13282CD008DCE5
:10AD9000012878D0062847D0072875D0122874D10A
:10ADA00006E0142872D0152871D016286DD1ACE1B8
:10ADB0000C2F6AD1307800F00301012965D040F0F2
:10ADC000080030706879B07001208DF8040028897F
:10ADD000ADF808006889ADF80A00A889ADF80C0044
:10ADE000E889ADF80E0019E0B07890429FD1307834
:10ADF00001079CD5062F9AD120F00800307060889A
:10AE0000414660F31F41012008F064FE02208DF8E6
:10AE10000400ADF808902889ADF80A006088224641
:10AE200001A9F8F7D9FF82E7082F80D12F89B5F85B
:10AE30000A90402F01D2402001E0A7F1400080B2EB
:10AE400080460146304600F048FC08B3716808EBC4
:10AE500088002C2202EBC000095A4945E3D1FE4884
:10AE600007AAD0E90210CDE9071068798DF81C0017
:10AE700008F0FF058DF81E5060883146FFF799FCF9
:10AE80002246294639E0B6E014E03CE039E0E6E04D
:10AE9000F148D0E90010CDE907106879ADF82070CD
:10AEA0008DF81C00ADF82290608807AA3146FFF7A4
:10AEB00080FC3CE7082FB6D16889B5F808804028A7
:10AEC00001D2402000E0403887B23946304600F0D9
:10AED00004FC0028A7D007EB870271680AEBC200C8
:10AEE0000844028A42459ED1017808299BD14078C6
:10AEF0006979884297D1F9B222463046FEF7F3FECF
:10AF000015E70E2F07D0CDF81C80CDF8208068798A
:10AF10008DF81C00C8E76989EF898B46B5F80C905D
:10AF20003046FEF742FFABF14001402901D3092032
:10AF30004AE0B9F1170F01D3172F01D20B2043E0DC
:10AF400040280ED000EB800271680AEBC200084472
:10AF50000178012903D1407869798842A9D00A2073
:10AF600032E03046FEF703FF014640282BD001EBCC
:10AF7000810372680AEBC30002EB0008012288F823
:10AF800000206A7988F8012070682A894089B842CF
:10AF900000D938462D8A03232372A282E7812082BA
:10AFA000A4F80C906582084600F07CFB6081A8F84C
:10AFB0001490A8F81870A8F80E50A8F810B0204601
:10AFC00000F066FBB3E6042005212172A4F80A8094
:10AFD000E08101212173A049D1E90421CDE90721B4
:10AFE00069798DF81C10ADF81E00608807AA3146FB
:10AFF000FFF7DFFBE3E7062FE4D3B078904215D1EB
:10B000003078010712D520F0080030706088414682
:10B0100060F31F41012008F05DFD02208DF804005F
:10B020002889ADF80800ADF80A90F7E6042130460B
:10B03000FEF7D3FE05464028C4D0022083030090CB
:10B0400022462946304600F065FB4146608865F39C
:10B050000F2160F31F41082008F03CFD67E60E2F2A
:10B06000B0D104213046FEF7B8FE81464028A9D071
:10B070004146608869F30F2160F31F41082008F002
:10B0800029FD288A0790E88900907068AF89408977
:10B09000B84200D938468346B5F80A802889059019
:10B0A000484600F0FFFA6081079840B10220079BF4
:10B0B000009022464946304600F02CFB37E6B8F1B6
:10B0C000170F1ED3172F1CD3042020720098608204
:10B0D000E781A4F810B0A4F80C8009EB890271682C
:10B0E0000AEBC2000D1800990598A5F81480A5F880
:10B0F00018B0E9812882204600F0CAFA062028709C
:10B1000015E601200B230090D3E7082FA6D129894B
:10B110003046FEF74AFE074640289FD007EB8702DD
:10B1200071680AEBC2000844804600F0ECFA00287F
:10B1300094D16D89B8F80E002844B0F5803F05D34E
:10B1400060883A46314600F01CFBF0E5002D85D0C2
:10B15000A8F80E0060883A463146FFF701F908204A
:10B160002072384600F09EFA6081A58127E770B50D
:10B170000D460646032105F0ABF9040004D0207803
:10B18000000704D5112070BD43F2020070BD2A46AD
:10B1900021463046FEF71FFF18B9286860616868CD
:10B1A000A061207840F008002070002070BD70B5CC
:10B1B0000D460646032105F08BF9040004D02078E3
:10B1C000000704D4082070BD43F2020070BD2A4677
:10B1D00021463046FEF732FF00B9A582207820F0E4
:10B1E00008002070002070BD2DE9F04F0E4691B090
:10B1F0008046032105F06CF90446404605F0ACFAA0
:10B2000007460020079008900990ADF830000A909A
:10B2100002900390049004B9FFDF0DF1080917BBF9
:10B22000FFDF20E038460BA9002204F0CFFC9DF898
:10B230002C0000F07F050A2D00D3FFDF6019017F8D
:10B24000491E01779DF82C0000060CD52A460CA952
:10B2500007A8FEF716FE01E0EC3D020019F8051004
:10B26000491C09F80510761EF6B2DBD204F1340051
:10B27000FC4D04F1260BDFF8F0A304F12A07069039
:10B2800010E05846069900F06EFA064628700A2823
:10B2900000D3FFDF5AF8261040468847E08CC05D97
:10B2A000B04202D0208D0028EBD10A202870EE4D4C
:10B2B0004E4628350EE00CA907A800F054FA0446C3
:10B2C000375D55F8240000B9FFDF55F824203946D2
:10B2D00040469047BDF81E000028ECD111B027E58C
:10B2E00010B5032105F0F4F8040000D1FFDF0A21B6
:10B2F00004F11C0018F09FFB207840F0040020703F
:10B3000010BD10B50C46032105F0E2F801190A7FC3
:10B3100001211AB9808EA140084000D0012010BD43
:10B320002DE9F84F894615468246032105F0D0F8ED
:10B33000070004D0284608F019FC40B903E043F2A6
:10B340000200BDE8F88F484608F036FC08B110202E
:10B35000F7E7786828B169880089814201D9092016
:10B36000EFE7B9F800001C2418B1402809D24020AA
:10B3700008E03846FEF7FBFC8046402819D1132030
:10B38000DFE7403880B280460146384600F0A5F934
:10B3900048B108EB8800796804EBC000085C01281C
:10B3A00003D00820CDE70520CBE7FDF775FF0600A9
:10B3B0000BD008EB8800796804EBC0000C18B9F8D2
:10B3C000000020B1E88910B113E01120B9E7288806
:10B3D000172802D36888172801D20720B1E76868C8
:10B3E00038B12B1D224641463846FFF71DF900288B
:10B3F000A7D104F10C0269462046FFF71CF8288803
:10B4000060826888E082B9F8000030B102202070C4
:10B41000E889A080E889A0B12BE003202070A889EA
:10B42000A08078688178402905D180F8028039466B
:10B430005046FEF722FE404600F034F9A9F800001D
:10B4400021E07868218B4089884200D90846208312
:10B45000A6F802A004203072B9F800007081E089DB
:10B460007082F181208B3082A08AB081304600F05A
:10B470000FF97868C178402905D180F803803946F2
:10B480005046FEF74BFE00205BE770B50D460646C2
:10B49000032105F01DF8040003D0402D04D24025FF
:10B4A00003E043F2020070BD403DADB2294600F01A
:10B4B00014F958B105EB85011C22606802EBC1014B
:10B4C000084400F020F918B1082070BD052070BDB7
:10B4D0002A462146304600F054F9002070BD2DE97F
:10B4E000F0410D4616468046032104F0F1FF044664
:10B4F000402D01D2402500E0403DADB28CB129463F
:10B5000000F0EBF880B105EB85011C22606802EBCE
:10B51000C1014718384600F0F6F838B10820BDE8F8
:10B52000F08143F20200FAE70520F8E733463A4695
:10B5300029462046FFF778F80028F0D1EAB22146E4
:10B540004046FEF797FF0020E9E72DE9F0410D4660
:10B5500016468046032104F0BBFF0446402D01D26D
:10B56000402500E0403DAFB224B1304608F0FEFA7D
:10B5700038B902E043F20200D1E7306808F0F6FA89
:10B5800008B11020CBE73946204600F0A6F860B19C
:10B5900007EB87011C22606802EBC10145182846B1
:10B5A00000F0B1F818B10820B9E70520B7E7B08876
:10B5B000A98A884201D90C20B1E76168E88C4978F2
:10B5C000B0EBC10F01D31320A9E73946204600F0A4
:10B5D00078F80146606808234078C20005F124002D
:10B5E00004F0FBFDD6E90012C0E90012FAB22146D0
:10B5F0004046FEF7B5FE002091E72DE9F0470D46E5
:10B600001F4690468146032104F062FF0446402D08
:10B6100001D2402001E0A5F1400086B23CB14DB11D
:10B62000384608F0E7FA50B11020BDE8F08743F241
:10B630000200FAE76068C8B1A0F80C8024E0314647
:10B64000204600F04AF888B106EB86011C226068AB
:10B6500002EBC1014518284600F055F840B108201A
:10B66000E3E7000030000020043E02000520DCE794
:10B67000A5F80880F2B221464846FEF7FBFE1FB14E
:10B68000A8896989084438800020CEE704F0FDBB12
:10B69000017821F00F01491C21F0F00110310170F7
:10B6A000FDF7FDBD10B50446402800D9FFDF40344A
:10B6B000A0B210BD406842690078484302EBC00068
:10B6C0007047C2784068037812FB03F24378406900
:10B6D00001FB032100EBC1007047C2788A4209D9FF
:10B6E000406801EB81011C2202EBC101405C08B102
:10B6F00001207047002070470078062801D90120FA
:10B700007047002070470078062801D0012070475C
:10B7100000207047F0B401EB81061C27446807EB5A
:10B72000C6063444049D05262670E3802571F0BCCE
:10B73000FEF790BA10B5418911B1FFF7DDFF08B1EE
:10B74000002010BD012010BD10B5C18C8278B1EB76
:10B75000C20F04D9C18911B1FFF7CEFF08B1002093
:10B7600010BD012010BD10B50C4601230A22011D99
:10B7700004F069FD007821880122824091432180F4
:10B7800010BDF0B402EB82051C264C6806EBC50523
:10B79000072363554B681C79402C03D11A71F0BC08
:10B7A000FEF701BDF0BC704710B5EFF3108000F05C
:10B7B000010472B6F9484178491C4170407801286B
:10B7C00001D107F005FE002C00D162B610BD70B5A6
:10B7D000F24CE07848B90125E570FFF7E5FF07F086
:10B7E000FFFD20B1002007F0DAFD002070BD4FF012
:10B7F00080406571C0F80453F7E770B5EFF310802F
:10B8000000F0010572B6E54C607800B9FFDF6078A2
:10B81000401E6070607808B907F0DEFD002D00D191
:10B8200062B670BDDD4810B5C17821B1002141710B
:10B83000C170FFF7E2FF002010BD10B5044607F00D
:10B84000CFFDD649C978084000D0012020600020F3
:10B8500010BD2DE9F05FDFF844934278817889F8D4
:10B860000620002689F80710074689F80860007846
:10B87000354620B101280FD002280FD0FFDF07F096
:10B88000BCFD98B107F0C0FDB0420FD1304607F0C3
:10B89000BFFD0028FAD047E00126F0E7FFF784FF5C
:10B8A00007F09EFD0028FBD00226E8E70120840770
:10B8B000E060C4F80451BA490E600107D1F844129F
:10B8C000B74AC1F3423124321160B54934310860BE
:10B8D0004FF0020BC4F804B3A060DFF8C8A2DAF896
:10B8E0000010C94341F3001101F10108DAF800101A
:10B8F00041F01001CAF8001000E020BFD4F80401A4
:10B900000028FAD0304607F083FD0028FAD0B8F1BD
:10B91000000F05D1DAF8001021F01001CAF800106C
:10B92000C4F808B3C4F8045199F807004C4670B144
:10B93000387860B907F054FD074607F0B9FE6FF09C
:10B94000004117B1C4E9031001E0C4E9030116B1D5
:10B950002571BDE8F09F0127BE0727714FF0190838
:10B96000C6F80883B761C6F80051C6F80C51C6F88E
:10B97000105107F035FD10B1A770376100E0277056
:10B98000FFF712FF8649A07920310860C6F80483CA
:10B99000DFE770B5050000D1FFDF4FF080424FF0C8
:10B9A000FF30C2F808030021C2F80011C2F80411E8
:10B9B000C2F80C11C2F81011784C617007F016FD36
:10B9C00010B10120E07060702846BDE8704040E78B
:10B9D0002DE9FE4F74480068734A744908321160BB
:10B9E0008C070290D4F8080108B1012500E0002579
:10B9F000D4F8240100B101208246D4F81C0100B122
:10BA000001208346D4F8200100B101200190D4F830
:10BA1000000110B14FF0010801E04FF00008D4F828
:10BA2000040108B1012700E00027D4F80C0100B19F
:10BA300001208146D4F8100108B1012100E0002165
:10BA4000009145EA080127EA0100009920EA09006F
:10BA5000884320EA0A0030EA0B0000D0FFDF00260E
:10BA600025B1C4F80861012007F099FCBAF1000F74
:10BA700004D0C4F82461092007F091FCBBF1000F49
:10BA800004D0C4F81C610A2007F089FC019820B199
:10BA9000C4F820610B2007F082FC404D4FF0010AF2
:10BAA000B8F1000F10D0C4F80061687918B16E7158
:10BAB000002007F074FC287830B107F091FC18B131
:10BAC00085F802A0C4F810A00FB1C4F80461B9F160
:10BAD000000F0AD0C4F80C61A87800B9FFDFAE707F
:10BAE0002E70C4F814A0FFF788FE009828B1C4F89F
:10BAF0001061287908B100F021F82B490298091D3E
:10BB00000860BDE8FE8F70B5244DE87808B907F0ED
:10BB100063FC01208407A061A87850B1D4F80C011F
:10BB200020B9002007F074FC0028F7D10020C4F8E9
:10BB30000C014FF0FF30C4F8080370BD2DE9F0414F
:10BB4000164C4FF080470125E079F0B1012803D071
:10BB5000217A401E814218DA07F042FC064607F0BF
:10BB6000A7FDE179012902D9217A491C21720EB180
:10BB7000216900E0E168411A022902DA11F1020F9D
:10BB800016DC0EB1206100E0E060FFF70DFE07F06B
:10BB900027FC80B13D61A5700EE000003C00002054
:10BBA0001805004010ED00E0100502400100000102
:10BBB0007D61BDE8F081257000202072F9E700006A
:10BBC0000F4A12680D498A420CD118470C4A126874
:10BBD0000A4B9A4206D101B507F038FDF7F723F971
:10BBE000BDE8014007490968095808470648074960
:10BBF000054A064B7047000000000000BEBAFECAAE
:10BC0000B00000200400002048130020481300204A
:10BC1000F8B51D46DDE906470E000AD004F09CFD8C
:10BC20002346FF1DBCB231462A46009404F0A7F912
:10BC3000F8BDD0192246194617F05CFE2046F8BD23
:10BC400070B50D460446102117F0D3FE258117204C
:10BC50006081A07B40F00A00A07370BD4FF6FF72B8
:10BC60000A800146032007F035BF704700897047FE
:10BC7000827BD30701D1920703D4808908800020FA
:10BC8000704705207047827B920700D581817047FD
:10BC900001460020098841F6FE52114200D00120E1
:10BCA000704700B50346807BC00701D0052000BD6A
:10BCB00059811846FFF7ECFFC00703D0987B40F08E
:10BCC00004009873987B40F001009873002000BD39
:10BCD000827B520700D509B1408970471720704711
:10BCE000827B61F3C302827370472DE9FC5F0E46CD
:10BCF000044601789646012000FA01F14DF6FF5204
:10BD000001EA020962684FF6FF7B1188594506D0A7
:10BD1000B9F1000F06D041F6FE55294202D00120AC
:10BD2000BDE8FC9F41EA090111801D0014D04FF0CD
:10BD3000000C85F800C023780521032267464FF0E8
:10BD4000020A0E2B74D2DFE803F0F809252F4762B0
:10BD50006974479092B3D0D70420E1E761682089E5
:10BD60008B7B9B077DD5172848D30B89834245D30E
:10BD70008989172901D3814240D185F800A0A5F80F
:10BD800001003280616888816068817B21F0020156
:10BD90008173C5E0042028702089A5F8010060891E
:10BDA000A5F803003180BBE0208A3188C01D1FFA4E
:10BDB00080F8414522D3062028702089A5F801008B
:10BDC0006089A5F80300A089A5F805000721208A4D
:10BDD000CDE9000163693EE0082B10D008202870EF
:10BDE0002089A5F801006089A5F8030031806A1D4B
:10BDF000694604F10C0005F07EFF10B15FE01020F1
:10BE0000EDE730889DF800100844308088E00A2073
:10BE100028702089A5F80100328045E00C202870A8
:10BE20002089A5F801006089A5F8030031803BE076
:10BE300083E02189338800EB41021FFA82F84345F1
:10BE40003DD3B8F1050F3AD30E222A700BEA410117
:10BE5000CDE90010E36860882A467146FFF7D8FEF6
:10BE600000E04DE0A6F800805AE04020287060898C
:10BE70003188C01C1FFA80F8414520D328787146CC
:10BE800020F03F00123028702089A5F80100608959
:10BE9000CDE9000260882A46E368FFF7B9FEA6F8FC
:10BEA0000080287840063BD461682089888037E08C
:10BEB000A0893288401D1FFA80F8424501D204272C
:10BEC0003EE0162028702089A5F801006089A5F8B9
:10BED0000300A089CDE9000160882A4671462369E4
:10BEE000FFF796FEA6F80080DEE718202870207A7B
:10BEF0006870A6F800A013E061680A88920401D473
:10BF000005271DE0C9882289914201D0062717E044
:10BF10001E21297030806068018821F40051018061
:10BF2000B9F1000F0CD0618878230022032007F0BC
:10BF300027FD61682078887007E0A6F800C0032715
:10BF40006068018821EA090101803846E8E62DE9A8
:10BF5000FF4F85B01746129C0D001E461CD030784E
:10BF6000C10703D000F03F00192801D9012100E0EA
:10BF700000212046FFF7ACFEA8420DD32088A0F593
:10BF80007F41FF3908D03078410601D4000605D53D
:10BF9000082009B0BDE8F08F0720FAE700208DF8EF
:10BFA00000008DF8010030786B1E00F03F0C01217D
:10BFB000A81E4FF0050A4FF002094FF0030B9AB28A
:10BFC000BCF1200F75D2DFE80CF08B10745E746842
:10BFD000748C749C74B674BB74C974D574E2747434
:10BFE00074F274F074EF74EE748B052D78D18DF8C3
:10BFF0000090A0788DF804007088ADF806003079C4
:10C000008DF80100707800F03F000C2829D00ADC80
:10C01000A0F10200092863D2DFE800F01262156285
:10C020001A621D622000122824D004DC0E281BD0C6
:10C030001028DBD11BE016281FD01828D6D11FE00E
:10C040002078800701E020784007002848DAEFE0F8
:10C0500020780007F9E72078C006F6E72078800608
:10C06000F3E720784006F0E720780006EDE7208827
:10C07000C005EAE720884005E7E720880005E4E7F7
:10C080002088C004E1E72078800729D5032D27D137
:10C090008DF800B0B6F8010082E0217849071FD57D
:10C0A000062D1DD381B27078012803D0022817D144
:10C0B00002E0CAE0022000E0102004228DF80020F7
:10C0C00072788DF80420801CB1FBF0F2ADF80620E8
:10C0D00092B242438A4203D10397ADF80890A7E099
:10C0E0007AE02078000777D598B282088DF800A012
:10C0F000ADF80420B0EB820F6ED10297ADF80610B8
:10C1000096E02178C90667D5022D65D381B2062055
:10C110008DF80000707802285ED300BFB1FBF0F20A
:10C120008DF80400ADF8062092B242438A4253D102
:10C13000ADF808907BE0207880064DD5072003E01D
:10C14000207840067FD508208DF80000A088ADF843
:10C150000400ADF80620ADF8081068E0207800066D
:10C1600071D50920ADF804208DF80000ADF8061057
:10C1700002975DE02188C90565D5022D63D381B2A0
:10C180000A208DF80000707804285CD3C6E7208868
:10C19000400558D5012D56D10B208DF80000A08800
:10C1A000ADF8040044E021E026E016E0FFE7208837
:10C1B000000548D5052D46D30C208DF80000A08839
:10C1C000ADF80400B6F803006D1FADF80850ADF8E7
:10C1D0000600ADF80AA02AE035E02088C00432D578
:10C1E000012D30D10D208DF8000021E02088800441
:10C1F00029D4B6F80100E080A07B000723D5032DE9
:10C2000021D3307800F03F001B2818D00F208DF884
:10C210000000208840F40050A4F80000B6F80100A7
:10C22000ADF80400ED1EADF80650ADF808B0039768
:10C2300069460598F5F7E7FD050008D016E00E20E1
:10C240008DF80000EAE7072510E008250EE03078B9
:10C2500000F03F001B2809D01D2807D003200599B6
:10C2600007F038FC208800F400502080A07B4007B5
:10C2700008D52046FFF70CFDC00703D1A07B20F0B6
:10C280000400A073284684E61FB5032806D10120C8
:10C290008DF8000088B26946F5F7B5FD1FBD0000B6
:10C2A000F8B51D46DDE906470E000AD004F054FA41
:10C2B0002346FF1DBCB231462A46009403F05FFEC0
:10C2C000F8BDD0192246194617F014FB2046F8BDD8
:10C2D0002DE9FF4F8DB09B46DDE91B57DDF87CA0B3
:10C2E0000C46082B05D0E06901F000F950B1102090
:10C2F000D2E02888092140F0100028808AF8001038
:10C30000022617E0E16901208871E2694FF42051AB
:10C310009180E1698872E06942F601010181E0697A
:10C32000002181732888112140F0200028808AF89C
:10C330000010042638780A900A2038704FF002095D
:10C3400004F118004D460C9001F093FBB04681E0DB
:10C35000BBF1100F0ED1022D0CD0A9EB0800801CF0
:10C3600080B20221CDE9001005AB52461E990D980E
:10C37000FFF796FFBDF816101A98814203D9F748C7
:10C3800000790F9004E003D10A9808B138702FE0CB
:10C390004FF00201CDE900190DF1160352461E9926
:10C3A0000D98FFF77DFF1D980088401B801B83B20E
:10C3B000C6F1FF00984200D203461E990BA8D9B1DE
:10C3C0005FF00002DDF878C0CDE9032009EB06013B
:10C3D00089B2CDE901C10F980090BDF81610002276
:10C3E0000D9801F0C9FB387070B1C0B2832807D036
:10C3F000BDF8160020833AE00AEB09018A19E1E74B
:10C40000022011B0BDE8F08FBDF82C00811901F0B9
:10C41000FF08022D0DD09AF80120424506D1BDF843
:10C420002010814207D0B8F1FF0F04D09AF80180A4
:10C430001FE08AF80180C94800680178052902D107
:10C44000BDF81610818009EB08001FFA80F905EB92
:10C45000080085B2DDE90C1005AB0F9A01F00CFB6A
:10C4600028B91D980088411B4145BFF671AF022DC8
:10C4700013D0BBF1100F0CD1A9EB0800801C81B2C6
:10C480000220CDE9000105AB52461E990D98FFF739
:10C4900007FF1D980580002038700020B1E72DE9C6
:10C4A000F8439C46089E13460027B26B9AB3491F77
:10C4B0008CB2F18FA1F57F45FF3D05D05518AD88B1
:10C4C0002944891D8DB200E000252919B6F83C8069
:10C4D0000831414520D82A44BCF8011022F8021B3B
:10C4E000BCF8031022F8021B984622F8024B914632
:10C4F00004F020F94FF00C0C41464A462346CDF893
:10C5000000C003F008FDF587B16B00202944A41D8D
:10C510002144088003E001E0092700E08327384632
:10C52000BDE8F88310B50B88848F9C420CD9846BCE
:10C53000E018048844B1848824F40044A41D2344F2
:10C540000B801060002010BD822010BD2DE9F04747
:10C550008AB00025904689468246ADF818500727D4
:10C560004BE0059806888088000446D4A8F800604F
:10C5700007A8019500970295CDE903504FF4007389
:10C5800000223146504601F0F7FA04003CD1BDF8D4
:10C590001800ADF82000059804888188B44216D1AF
:10C5A0000A0414D401950295039521F400410097E3
:10C5B000049541F4804342882146504601F0B2F888
:10C5C00004000BD10598818841F40041818005AABF
:10C5D00008A94846FFF7A6FF0400DCD0009705989D
:10C5E00002950195039504950188BDF81C30002241
:10C5F000504601F097F8822C06D105AA06A94846B4
:10C60000FFF790FF0400ACD0ADF8185004E0059897
:10C61000818821F40041818005AA06A94846FFF7D8
:10C6200081FF0028F3D0822C03D020460AB0BDE859
:10C63000F0870020FAE710B50C46896B86B051B13F
:10C640000C218DF80010A18FADF80810A16B01919D
:10C650006946FAF7AFFC00204FF6FF71A063E1874F
:10C66000A08706B010BD2DE9F0410D460746896B45
:10C670000020069E1446002911D0012B0FD132460E
:10C6800029463846FFF762FF002808D1002C06D063
:10C69000324629463846BDE8F04100F036BFBDE8D5
:10C6A000F0812DE9FC411446DDE9087C0E46DDE908
:10C6B0000A15521DBCF800E092B2964502D207203E
:10C6C000BDE8FC81ACF8002017222A70A5F80160B3
:10C6D000A5F803300522CDE900423B462A46FFF784
:10C6E000DFFD0020ECE770B50C46154648212046DA
:10C6F00017F0A1F904F1080044F81C0F00204FF6D0
:10C70000FF71E06161842084A5841720E08494F89F
:10C710002A0040F00A0084F82A0070BD4FF6FF722C
:10C720000A800146042007F0D5B930B585B00C4623
:10C730000546FFF780FFA18E284629B101218DF81B
:10C7400000106946FAF736FC0020E062206360635F
:10C7500005B030BDB0F84000704700005400002024
:10C7600090F84620920703D4408808800020F3E721
:10C770000620F1E790F846209207EDD5A0F8441086
:10C78000EAE70146002009880A0700D5012011F0D8
:10C79000F00F01D040F00200CA0501D540F00400BE
:10C7A0008A0501D540F008004A0501D540F0100087
:10C7B0000905D1D540F02000CEE700B5034690F83A
:10C7C0004600C00701D0062000BDA3F8421018465D
:10C7D000FFF7D7FF10F03E0F05D093F8460040F06A
:10C7E000040083F8460013F8460F40F0010018706B
:10C7F000002000BD90F84620520700D511B1B0F8D6
:10C800004200A9E71720A7E710F8462F61F3C302FB
:10C810000270A1E72DE9FF4F9BB00E00DDE92B343C
:10C82000DDE92978289D24D02878C10703D000F0BD
:10C830003F00192801D9012100E000212046FFF71F
:10C84000D9FFB04215D32878410600F03F010CD43F
:10C850001E290CD0218811F47F6F0AD13A8842B189
:10C86000A1F57F42FF3A04D001E0122901D1000670
:10C8700002D504201FB0C5E5F9491D984FF0000A04
:10C8800008718DF818A08DF83CA00FAA0A60ADF8C9
:10C890001CA0ADF850A02978994601F03F02701F06
:10C8A0005B1C04F1180C4FF0060E4FF0040BCDF892
:10C8B00058C01F2A7ED2DFE802F07D7D107D267DE4
:10C8C000AC7DF47DF37DF27DF17DF47DF07D7D7DA9
:10C8D000EF7DEE7D7D7D7D7DED0094F84610B5F811
:10C8E0000100890701D5032E02D08DF818B022E38C
:10C8F0004FF40061ADF85010608003218DF83C10BA
:10C90000ADF84000D8E2052EEFD1B5F80100208344
:10C91000ADF81C00B5F80310618308B1884201D955
:10C9200001207FE10020A07220814FF6FF7020845B
:10C93000169801F09EF8052089F800000220029068
:10C9400083460AAB1D9A16991B9801F095F890BB87
:10C950009DF82E00012804D0022089F80100102043
:10C9600003E0012089F8010002200590002203A9BC
:10C970000BA805F0C0F9E8BB9DF80C0005998142B1
:10C980003DD13A88801CA2EB0B01814237DB029932
:10C990000220CDE900010DF12A034A4641461B98C9
:10C9A000FFF77EFC02980BF1020B801C80B217AAE5
:10C9B00003A901E0A0E228E002900BA805F09BF992
:10C9C00002999DF80C00CDE9000117AB4A4641469B
:10C9D0001B98FFF765FC9DF80C100AAB0BEB0100F0
:10C9E0001FFA80FB02981D9A084480B202901699A3
:10C9F0001B9800E003E001F03FF80028B6D0BBF13F
:10CA0000020F02D0A7F800B053E20A208DF81800F8
:10CA10004FE200210391072EFFF467AFB5F8010044
:10CA20002083ADF81C00B5F80320628300283FF492
:10CA300077AF90423FF674AF0120A072B5F80500C1
:10CA400020810020A073E06900F050FD78B9E16911
:10CA500001208871E2694FF420519180E169887268
:10CA6000E06942F601010181E06900218173F01F54
:10CA700020841E98606207206084169800F0F9FFF9
:10CA8000072089F800000120049002900020ADF8F2
:10CA90002A0028E01DE2A3E13AE1EAE016E2AEE076
:10CAA00086E049E00298012814D0E06980790128E5
:10CAB00003D1BDF82800ADF80E00049803ABCDE912
:10CAC00000B04A4641461B98FFF7EAFB0498001D58
:10CAD00080B20490BDF82A00ADF80C00ADF80E004D
:10CAE000059880B202900AAB1D9A16991B9800F027
:10CAF000C3FF28B902983988001D05908142D1D220
:10CB00000298012881D0E0698079012805D0BDF81C
:10CB10002810A1F57F40FF3803D1BDF82800ADF8FB
:10CB20000E00049803ABCDE900B04A4641461B987D
:10CB3000FFF7B6FB0298BBE1072E02D0152E7FF45B
:10CB4000D4AEB5F801102183ADF81C10B5F8032060
:10CB5000628300293FF4E4AE91423FF6E1AE012149
:10CB6000A1724FF0000BA4F808B084F80EB0052EA7
:10CB700007D0C0B2691DE26905F09EF800287FF475
:10CB800044AF4FF6FF70208401A906AA14A8CDF87F
:10CB900000B081E885032878214600F03F031D9A04
:10CBA0001B98FFF795FB8246208BADF81C0080E1B7
:10CBB0000120032EC3D14021ADF85010B5F801106B
:10CBC0002183ADF81C100AAAB8F1000F00D0002391
:10CBD000CDE9020304921D98CDF8048000903888B6
:10CBE0000022401E83B21B9800F0C6FF8DF818008B
:10CBF00090BB0B2089F80000BDF8280037E04FF00B
:10CC0000010C052E9BD18020ADF85000B5F8011025
:10CC10002183B5F803002084ADF81C10B0F5007F27
:10CC200003D907208DF8180085E140F47C42228466
:10CC30000CA8B8F1000F00D00023CDE90330CDE9F6
:10CC4000018C1D9800903888401E83B21B9800F01C
:10CC500093FF8DF8180028B18328A8D10220BDE0E9
:10CC6000540000200D2189F80010BDF83000401C50
:10CC70001EE1032E04D248067FF537AE002017E1EF
:10CC8000B5F80110ADF81C102878400602D58DF8D3
:10CC90003CE002E007208DF83C004FF00008032044
:10CCA000CDE902081E9BCDF810801D980193A6F1D6
:10CCB000030B00901FFA8BF342461B9800F032FDE5
:10CCC0008DF818008DF83C80297849060DD520880C
:10CCD000C00506D5208BBDF81C10884201D1C4F8D0
:10CCE000248040468DF81880E2E0832801D14FF07F
:10CCF000020A4FF48070ADF85000BDF81C0020838C
:10CD0000A4F820B01E986062032060841321CCE058
:10CD1000052EFFF4EAADB5F80110ADF81C10A28F96
:10CD200062B3A2F57F43FE3B28D008228DF83C2059
:10CD30004FF0000B0523CDE9023BDDF878C0CDF8BC
:10CD400010B01D9A80B2CDF804C040F400430092A8
:10CD5000B5F803201B9800F0E5FC8DF83CB04FF4CB
:10CD600000718DF81800ADF85010832810D0F8B17C
:10CD7000A18FA1F57F40FE3807D0DCE00B228DF8B3
:10CD80003C204FF6FE72A287D2E7A4F83CB0D2E076
:10CD900000942B4631461E9A1B98FFF780FB8DF8B6
:10CDA000180008B183284BD1BDF81C00208355E73B
:10CDB00000942B4631461E9A1B98FFF770FB8DF8A6
:10CDC0001800E8BBE18FA06B0844811D8DE8820349
:10CDD0004388828801881B98FFF763FC824668E0DD
:10CDE00095F80180022E70D15FEA080002D0B8F1F8
:10CDF000010F6AD109208DF83C0007A800908DF83A
:10CE000040804346002221461B98FFF72CFC8DF8FA
:10CE100042004FF0000B8DF843B050B9B8F1010F4C
:10CE200012D0B8F1000F04D1A18FA1F57F40FF38D7
:10CE30000AD0A08F40B18DF83CB04FF4806000E084
:10CE400037E0ADF850000DE00FA91B98FAF7B2F8E3
:10CE500082468DF83CB04FF48060ADF85000BAF1D6
:10CE6000020F06D0FB480068C07928B18DF8180081
:10CE700027E0A4F8188044E0BAF1000F03D0812025
:10CE80008DF818003DE007A8009043460122214696
:10CE90001B98FFF7E8FB8DF8180021461B98FFF759
:10CEA000CAFB9DF8180020B9192189F8001001204B
:10CEB00038809DF83C0020B10FA91B98FAF77AF84A
:10CEC0008246BAF1000F33D01BE018E08DF818E06D
:10CED00031E02078000712D5012E10D10A208DF8FC
:10CEE0003C00E088ADF8400004201B9906F0F2FDFC
:10CEF0000820ADF85000C1E648067FF5F6AC4FF0CB
:10CF0000040A2088BDF8501008432080BDF8500066
:10CF100080050BD5A18FA1F57F40FE3806D11E9864
:10CF2000E06228982063A6864FF0030A5046A1E4E9
:10CF30009DF8180078B1012089F80000297889F857
:10CF40000110BDF81C10A9F802109DF8181089F8FE
:10CF50000410052038802088BDF8501088432080B8
:10CF6000E4E72DE9FF4F8846087895B0012181401C
:10CF70004FF20900249C0140ADF820102088DDF814
:10CF80008890A0F57F424FF0000AFF3A02D029B105
:10CF9000000703D5012019B0BDE8F08F239E4FF0A4
:10CFA000000B0EA886F800B018995D460988ADF808
:10CFB0003410A8498DF81CB0179A0A718DF838B052
:10CFC000086098F8000001283BD0022809D0032807
:10CFD0006FD1307820F03F001D303070B8F8040079
:10CFE000E08098F800100320022904D1317821F064
:10CFF0003F011B31317094F84610090759D505AB34
:10D00000B9F1000F13D0002102AA82E80B0007201B
:10D01000CDE90009BDF83400B8F80410C01E83B291
:10D020000022159800F0A8FD0028D1D101E0F11CE4
:10D03000EAE7B8F80400A6F80100BDF81400C01C27
:10D0400004E198F805108DF81C1098F804000128E8
:10D0500006D04FF4007A02282CD00328B8D16CE116
:10D060002188B8F8080011F40061ADF8201020D034
:10D0700017281CD3B4F84010814218D3B4F84410D8
:10D08000172901D3814212D1317821F03F01C91C07
:10D090003170A6F801000321ADF83410A4F8440063
:10D0A00094F8460020F0020084F8460065E105256A
:10D0B0007EE177E1208808F1080700F4FE60ADF812
:10D0C000200010F0F00F1BD010F0C00F03D03888F4
:10D0D000228B9042EBD199B9B878C00710D0B968CB
:10D0E0000720CDE902B1CDF804B00090CDF810B022
:10D0F000FB88BA883988159800F014FB0028D6D12F
:10D100002398BDF82010401C80294ED006DC102941
:10D110000DD020290BD0402987D124E0B1F5807FA4
:10D120006ED051457ED0B1F5806F97D1DEE0C80654
:10D1300001D5082000E0102082460DA907AA05208D
:10D14000CDE902218DF83800ADF83CB0CDE9049668
:10D1500008A93888CDE900015346072221461598D1
:10D16000FFF7B6F8A8E09DF81C2001214FF00A0A4D
:10D17000002A9BD105ABB9F1000F00D00020CDE90A
:10D1800002100720CDE90009BDF834000493401EC9
:10D1900083B2218B0022159800F0EEFC8DF81C0064
:10D1A0000B203070BDF8140020E09DF81C200121F8
:10D1B0004FF00C0A002A22D113ABB9F1000F00D0B6
:10D1C0000020CDE902100720CDE900090493BDF845
:10D1D0003400228C401E83B2218B159800F0CCFCC9
:10D1E0008DF81C000D203070BDF84C00401CADF8CF
:10D1F000340005208DF83800208BADF83C00BCE0F1
:10D200003888218B88427FF452AF9DF81C004FF084
:10D21000120A00281CD1606AA8B1B878C0073FF490
:10D2200046AF00E018E0BA680720CDE902B2CDF8B9
:10D2300004B00090CDF810B0FB88BA88159800F0C3
:10D2400071FA8DF81C00132030700120ADF8340005
:10D2500093E00000540000203988208B8142D2D115
:10D260009DF81C004FF0160A0028A06B08D0E0B310
:10D270004FF6FF7000215F46ADF808B0019027E03F
:10D2800068B1B978C907BED1E18F0DAB0844821DE2
:10D2900003968DE80C0243888288018809E0B878FB
:10D2A000C007BCD0BA680DAB03968DE80C02BB88F2
:10D2B000FA881598FFF7F5F905005ED0072D72D0B2
:10D2C00076E0019005AA02A92046FFF72BF9014656
:10D2D000E28FBDF80800824201D00029F1D0E08F32
:10D2E000A16B084407800198E08746E09DF81C0088
:10D2F0004FF0180A40B1208BC8B1388820832146EE
:10D300001598FFF798F938E004F118000090237E93
:10D31000012221461598FFF7A6F98DF81C00002878
:10D32000EDD1192030700120ADF83400E7E7052574
:10D3300021461598FFF77FF93AE0208800F4007045
:10D34000ADF8200050452DD1A08FA0F57F41FE39CA
:10D3500001D006252CE0D8F808004FF0160A48B195
:10D36000A063B8F80C10A1874FF6FF71E187A0F811
:10D3700000B002E04FF6FF70A087BDF8200030F447
:10D380007F611AD0782300220420159906F0F8FA5C
:10D3900098F8000020712088BDF8201008432080F4
:10D3A0000EE000E007252088BDF82010884320808B
:10D3B000208810F47F6F1CD03AE0218881432180BF
:10D3C0009DF8380020B10EA91598F9F7F3FD054630
:10D3D0009DF81C000028EBD086F801A001203070D9
:10D3E000208B70809DF81C0030710520ADF8340052
:10D3F000DEE7A18EE1B118980DAB0088ADF83400DE
:10D400002398CDE90304CDE90139206B0090E36A4C
:10D41000179A1598FFF7FEF9054601208DF8380098
:10D420000EA91598F9F7C6FD00B10546A4F834B069
:10D4300094F8460040070AD52046FFF7A2F910F0FD
:10D440003E0F04D114F8460F20F004002070189805
:10D45000BDF83410018028469DE500B585B004284C
:10D4600006D102208DF8000088B26946F9F7A2FDC6
:10D4700005B000BD10B5384C0B782268012B02D0E6
:10D48000022B2AD111E013780BB1052B01D1042313
:10D49000137023688A889A802268CB88D380226898
:10D4A0000B891381498951810DE08B889380226813
:10D4B000CB88D38022680B8913814B8953818B8958
:10D4C0009381096911612168F9F774FD22680021CF
:10D4D0000228117003D0002800D0812010BD8320C5
:10D4E00010BD806B002800D0012070478178012991
:10D4F00009D10088B0F5205F03D042F601018842CF
:10D5000001D10020704707207047F0B587B0002494
:10D5100015460E460746ADF8144010E006980188FF
:10D520002980811DCDE902410721019404940091D5
:10D53000838842880188384600F0F4F830B906AA9A
:10D5400005A93046FEF7EEFF0028E7D0822800D17B
:10D55000002007B0F0BD00005400002010B58B780B
:10D5600083B102789A4205D10B885BB102E08B79D6
:10D57000091D4BB18B789A42F9D1B0F801300C8873
:10D58000A342F4D1002010BD812010BD072826D071
:10D5900012B1012A27D103E0497801F0070102E026
:10D5A0004978C1F3C20105291DD2DFE801F0031853
:10D5B000080C12000AB103207047022070470428AB
:10D5C0000DD250B10DE0052809D2801E022808D3E3
:10D5D00003E0062803D0032803D00520704700206D
:10D5E00070470F20704781207047C0B282060BD46D
:10D5F000000607D5FE48807A4143C01D01EBD000EC
:10D6000080B27047084670470020704770B5138895
:10D610000B800B781C0625D5F54CA47A844204D8DF
:10D6200043F010000870002070BD956800F00706F8
:10D6300005EBD0052D78F54065F304130B701378D6
:10D64000D17803F0030341EA032140F20123B1FB47
:10D65000F3F503FB15119268E41D00FB012000EBBC
:10D66000D40070BD906870BD37B51446BDF8041085
:10D6700011809DF804100A061ED5C1F30013DC4981
:10D68000A568897A814208D8FE2811D1C91DC90828
:10D690005A42284616F0A5F90AE005EBD00100F041
:10D6A0000702012508789540A84393401843087065
:10D6B000207820F0100020703EBD2DE9F041074693
:10D6C000C81C0E4620F00300B04202D08620BDE800
:10D6D000F081C74D002034462E60AF802881AA72A9
:10D6E000E8801AE0E988491CE980810614D4E178D1
:10D6F00000F0030041EA002040F20121B0FBF1F20A
:10D7000001FB12012068FFF770FF2989084480B2ED
:10D710002881381A3044A0600C3420784107E1D4C5
:10D720000020D4E72DE9FF4F89B01646DDE9168ABF
:10D730000F46994623F44045084600F00DFB0400CF
:10D740000FD0099802F08AFE0290207800060AD5D0
:10D75000A748817A0298814205D887200DB0BDE89C
:10D76000F08F0120FAE7224601A90298FFF74EFF49
:10D77000834600208DF80C004046B8F1070F1AD000
:10D7800001222146FFF702FF0028E7D1207840065A
:10D7900011D502208DF80C00ADF81070BDF8040012
:10D7A000ADF81200ADF814601898ADF81650CDF829
:10D7B0001CA0ADF818005FEA094004D500252E46EC
:10D7C000A84601270CE02178E07801F0030140EA47
:10D7D000012040F20121B0FBF1F2804601FB1287EB
:10D7E0005FEA494009D5B84507D1A178207901F011
:10D7F000030140EA0120B04201D3BE4201D9072013
:10D80000ACE7A8191FFA80F9B94501D90D20A5E7A1
:10D810009DF80C0028B103A90998F9F7C9FB002865
:10D820009CD1B84507D1A0784FEA192161F30100D6
:10D83000A07084F804901A9800B10580199850EAF5
:10D840000A0027D0199830B10BEB06002A46199927
:10D8500016F050F80EE00BEB06085746189E099894
:10D8600002F068FF2B46F61DB5B2394642460095D8
:10D8700002F051FB224601A90298FFF7C7FE9DF86E
:10D880000400224620F010008DF80400DDE90110AC
:10D89000FFF7EAFE002061E72DE9FF4FDFF8509126
:10D8A00082461746B9F80610D9F8000001EB41018D
:10D8B00000EB810440F20120B2FBF0F185B000FBE7
:10D8C00011764D46DDF84C8031460698FFF78DFE07
:10D8D00029682A898B46611A0C3101441144AB88AE
:10D8E00089B28B4202D8842009B038E70699CDB2BC
:10D8F000290603D5A90601D58520F5E7B9F806C0A4
:10D900000CF1010C1FFA8CFCA9F806C0149909B19E
:10D91000A1F800C0A90602D5C4F8088007E01044A9
:10D9200080B2A9F80800191A01EB0B00A06022468A
:10D93000FE200699FFF798FEE77026712078390AD5
:10D9400061F30100320AA17840F0040062F30101A2
:10D95000A17020709AF802006071BAF80000E080AF
:10D9600000262673280602D599F80A7000E00127E0
:10D97000A80601D54FF000084D4600244FF00709D6
:10D980000FE0CDE902680196CDF800900496E98891
:10D990002046129B089AFFF7C5FE0028A4D1641CFC
:10D9A000E4B2BC42EDD300209EE72DE9F04780466B
:10D9B00000F0D2F9070005D0002644460C4D40F295
:10D9C000012919E00120BDE8F087204600F0C4F9E4
:10D9D0000278C17802F0030241EA0222B2FBF9F3B5
:10D9E00009FB13210068FFF700FE304486B201E016
:10D9F00094060020641CA4B2E988601E8142E4DC25
:10DA0000A8F10100E8802889801B28810020387057
:10DA1000D9E710B5144631B1491E218002F01EFD30
:10DA2000A070002010BD012010BD10B5D2490446E1
:10DA30000088CA88904201D3822010BD096800EB9B
:10DA4000400001EB80025079A072D088208191784B
:10DA5000107901F0030140EA0120A081A078E11CC7
:10DA6000FFF7D4FD20612088401C2080E08000204A
:10DA700010BD0121018270472DE9FF4F85B04FF69F
:10DA8000FF788246A3F8008048681F460D468078DC
:10DA90008DF8060048680088ADF8040000208DF875
:10DAA0000A00088A0C88A04200D304462C8241E078
:10DAB000288A401C2882701D6968FFF74FFDB8BB9B
:10DAC0003988414501D1601E38806888A04236D32C
:10DAD000B178307901F0030140EA012901A9701DF4
:10DAE000FFF73CFD20BB298941452CD0002231465F
:10DAF0000798FFF74BFDD8B92989494518D1E9683E
:10DB00000391B5F80AC0D6F808B05046CDF800C069
:10DB100002F010FEDDF800C05A460CF1070C1FFAA7
:10DB20008CFC4B460399CDF800C002F0BEF950B111
:10DB3000641CA4B2204600F00FF90600B8D1641EA0
:10DB40002C828220D0E67C807079B871F088B88011
:10DB50003178F07801F0030140EA01207881A7F8DC
:10DB60000C90504602F07AFC324607F10801FFF7AC
:10DB70004DFD38610020B7E62DE9FF4F87B08146A3
:10DB80001C469246DDF860B0DDF85480089800F03D
:10DB9000E3F805000CD0484602F060FC297809063D
:10DBA00008D57549897A814204D887200BB0D6E51B
:10DBB0000120FBE7CAF309062A4601A9FFF726FD63
:10DBC0000746149807281CD000222946FFF7DEFCE0
:10DBD0000028EBD12878400613D501208DF80800E5
:10DBE0000898ADF80C00BDF80400ADF80E00ADF8D3
:10DBF0001060ADF8124002A94846F9F7D9F900289B
:10DC0000D4D12978E87801F0030140EA0121AA780B
:10DC1000287902F0030240EA0220564507D0B1F508
:10DC2000007F04D9611E814201DD0B20BEE78642E0
:10DC300001D90720BAE7801B85B2A54200D9254645
:10DC4000BBF1000F01D0ABF80050179818B1B9190B
:10DC50002A4615F04FFEB8F1000F0DD03E4448465D
:10DC60004446169F02F078FD2146FF1DBCB23246A5
:10DC70002B46009402F083F9002097E72DE9F0414C
:10DC800007461D461646084600F066F804000BD00D
:10DC9000384602F0E3FB2178090607D53649897A30
:10DCA000814203D8872012E5012010E52246314643
:10DCB000FFF7ACFC65B12178E07801F0030140EAA0
:10DCC0000120B0F5007F01D8012000E0002028707D
:10DCD0000020FCE42DE9F04107461D4616460846A3
:10DCE00000F03AF804000BD0384602F0B7FB217878
:10DCF000090607D52049897A814203D88720E6E4BE
:10DD00000120E4E422463146FFF7AEFCFF2D14D09B
:10DD10002178E07801F0030240EA022040F201227B
:10DD2000B0FBF2F302FB130015B900F2012080B240
:10DD3000E070000A60F3010121700020C7E410B513
:10DD40000C4600F009F828B1C18821804079A07004
:10DD5000002010BD012010BD0749CA88824209D3A6
:10DD600040B1096800EB40006FF00B0202EB80004D
:10DD700008447047002070479406002010B506F054
:10DD8000D7F8F4F711FD05F06FFFBDE8104006F07D
:10DD900021B870B50346002002466FF02F050EE053
:10DDA0009C5CA4F130060A2E02D34FF0FF3070BD08
:10DDB00000EB800005EB4000521C2044D2B28A42A6
:10DDC000EED370BD30B50A240AE0B0FBF4F304FBD7
:10DDD00013008D18303005F8010C521E1846D2B2CF
:10DDE000002AF2D130BD30B500234FF6FF7510E0A8
:10DDF000040A44EA002084B2C85C6040C0F3031403
:10DE0000604005EA00344440E0B25B1C84EA401004
:10DE10009BB29342ECD330BD10B582B0694601F09D
:10DE20003EFD002818BFFFDF9DF8000000240128F8
:10DE300009D1019890F8D50028B1019880F8D54013
:10DE400001980CF06DFFFE488068A0F8CA4002B04F
:10DE500010BD2DE9F04704460D46062002F0E0FA19
:10DE60000646072002F0DCFA304400F0FF080027E5
:10DE700018EB050618BF4FF000091DD02088401C84
:10DE800080B22080B04228BFA4F800902588454584
:10DE900001D3B54209D30621284602F019FB20B967
:10DEA0000721284602F014FB10B10020BDE8F087DE
:10DEB000781CC7B2BE42E1D84FF6FF702080122016
:10DEC000BDE8F08770B5DFA182B0D1E90001CDE9EE
:10DED000000106F0A3FF11F079FFDC4C4FF6FF764E
:10DEE00000256683A683257065706946A01C15F021
:10DEF000B2FEA11C601C0EF033FC25721B20608159
:10DF00004FF4A471A181E08121820321A174042234
:10DF1000E274A082E082A4F13E0021830570468075
:10DF2000CB480570A4F110000570468002B070BDAA
:10DF3000F8B5C34D0E466860297006F0E9FE4FF64D
:10DF4000FF70ADF8000000216846FFF782FFA0B91E
:10DF50000621BDF8000002F0CDFA04460721BDF805
:10DF6000000002F0C7FA002C1CBF0028FFDF0021D0
:10DF70006846FFF76EFF0028EAD0FFF7A3FF287876
:10DF80000BF099F909F0F5F8297868680EF0FCFAB9
:10DF9000287811F0ABF830460CF0D3FD07F04AF8C2
:10DFA0002978686810F006F8BDE8F84011F00EBF57
:10DFB00010B50124002A1CBF002010BD002908BF95
:10DFC000022105D0012918BF002401D0204610BD30
:10DFD00013F0DAFCFAE72DE9F04F8BB0040008BF2C
:10DFE000FFDF0221994E06F11C00FFF732FF0028E7
:10DFF00018BFFFDFB6F81CA0062002F011FA054694
:10E00000072002F00DFA284400F0FF0808F1010093
:10E0100000F0FF094FF0000BB78B474519D12046A0
:10E0200008F03EFB002840F0BD803078002800F06A
:10E03000BD8084F801B0142020702021A01C15F0B0
:10E04000D8FC0220A07086F800B00BB00120BDE81B
:10E05000F08F4F451CD1204606F092FF00287AD061
:10E060002078142804BFA0783C2853D1A088072129
:10E0700002F02EFA050008BFFFDF288806F061FED7
:10E08000A088072102F036FA002818BFFFDF89E0D8
:10E0900004A9384601F003FC00285CD19DF810006B
:10E0A00048B106F0BCFFB84255D0214638460FF0C3
:10E0B00081FE80B376E008F08BFBB84276D0214633
:10E0C00038460EF073F900286CD1059800F1580518
:10E0D00090F8C80018B9A87E08B1012000E000201F
:10E0E000079095F8350000281CBF95F8360010F011
:10E0F000020F1CD084F801B00120207084F802B017
:10E10000A78095F83700A071288F2081688F6081E3
:10E1100085F835B046E0FFE7059800F1580590F81E
:10E1200004010028DBD1A87E0028D8D0D5E73846E6
:10E1300002F012FB0290002808BFFFDF029801F0F6
:10E140001EFD48B184F801B00F212170A780E08046
:10E150000120A07026E029E0384602F0EBFA029098
:10E16000002808BFFFDF079800B3029801F05FFDA9
:10E17000E0B19DF8100038B90598D0F8F00041885A
:10E18000B94208BF80F800B0384606F0DAFD84F8DE
:10E1900001B00C20207084F802B0A780E87EA07146
:10E1A00085F81AB00BB00120BDE8F08F022106F10E
:10E1B0001C00FFF74EFE18B9B08B50457FF42CAF12
:10E1C0000BB00020BDE8F08F10B50BF0F1FD042876
:10E1D00003D00BF0EDFD052802D109F0CBF928B9E9
:10E1E0000CF087FF20B107F036F808B10C2010BD05
:10E1F00011F037FE002010BD10B50446007800284D
:10E200001EBF0128122010BD0BF0D2FD042806D03D
:10E210000BF0CEFD052802D00CF06BFF28B111F0F9
:10E220006AFF00281CBF0C2010BD2078002816BFF4
:10E2300002280020012004F11703E21D611C09E0FF
:10E240005C000020FFFFFFFF1F000000DE06002033
:10E2500068000020BDE8104011F05ABE10B5044619
:10E26000007800281EBF0128122010BD0BF0A0FD71
:10E27000042803D00BF09CFD052802D109F07AF99F
:10E2800028B90CF036FF20B106F0E5FF08B10C20EC
:10E2900010BD2078002816BF022800200120611C34
:10E2A00011F0A6FD002814BF0020072010BD10B5F6
:10E2B00011F024FF002814BF0020302010BD10B53D
:10E2C00004460BF075FD042806D00BF071FD0528FF
:10E2D00002D00CF00EFF08B10C2010BD204611F04A
:10E2E00007FF002010BD10B50BF062FD042806D01A
:10E2F0000BF05EFD052802D00CF0FBFE28B111F0FA
:10E30000FAFE00281CBF0C2010BD11F055FE0020A5
:10E3100010BDFF2181704FF6FF718180FE49496871
:10E320000A7882718A88028149884181012141707D
:10E330000020704710B5002482B0022A18D014DCE7
:10E3400012F10C0F14D008DC12F1280F1CBF12F1CF
:10E35000140F12F1100F10D10AE012F1080F1CBFB8
:10E3600012F1040F002A08D102E0D31E062B04D8B4
:10E3700038B1012809D002280BD0122402B020465F
:10E3800010BD104607F01EF9F8E7104608F0B0FE81
:10E39000F4E708461446694601F081FA002818BFE0
:10E3A0000224EBD19DF80000019880F8544000242D
:10E3B000E4E710B51346012212F029FD002010BD3C
:10E3C00010B504460BF0F4FC052804BF0C2010BD6A
:10E3D00020460AF05EFF002010BD10B504460BF089
:10E3E000E7FC042806D00BF0E3FC052802D00CF073
:10E3F00080FE08B10C2010BD2146002006F00FFD64
:10E40000002010BD10B504460AF0EDFF50B10CF02D
:10E4100063FE38B120780CF0B8FB207809F0E3F8FF
:10E42000002010BD0C2010BD10B504460BF0C0FC40
:10E43000042806D00BF0BCFC052802D00CF059FED5
:10E4400008B10C2010BD2146012006F0E8FC002098
:10E4500010BD38B504464FF6FF70ADF80000A07946
:10E46000E179884213D021791F299CBF61791F2946
:10E470000DD80022114614F0A7FB40B90022E07924
:10E48000114614F0A1FB10B9207A072801D91220F7
:10E4900038BD0CF02EFE60B90BF08AFC48B90021A3
:10E4A0006846FFF7D6FC20B1204605F06FFD00203E
:10E4B00038BD0C2038BD70B504468078002582B088
:10E4C0001A2825D00EDC162841D2DFE800F04040A3
:10E4D000404040214040404040404040404040405B
:10E4E000402121212A2832D00BDCA0F11E000C286B
:10E4F0002DD2DFE800F02C2C2C2C2C2C2C2C2C2CAE
:10E500002C0D3A38042822D2DFE800F02102210243
:10E510002088B0F5706F1AD20126694601F0BFF964
:10E5200000281EBF022002B070BD9DF80000002828
:10E5300001980BBF00F1EC0100F5B37100F1ED02A1
:10E5400000F2671290F8723012D173B903E002B092
:10E550004FF0120070BD90F8C830002B1CBF90F82F
:10E56000C800042801D0087868B102B00C2070BD42
:10E57000002BFAD190F80431002B1CBF90F8040155
:10E580000428F0D1F1E70E70A07810709DF800001B
:10E59000012809D1019890F8D50028B1019880F898
:10E5A000D55001980CF0BCFB02B0002070BDF0B556
:10E5B00083B00C46694601F072F928B1204615F087
:10E5C0003DFB03B00220F0BD0198002700F1580583
:10E5D00000F1080685F83E703146204615F03BFBF9
:10E5E00095F83E000028F5D103B0F0BD2DE9F041CB
:10E5F00082B004460088694601F051F900281CBF2A
:10E6000002B0BDE8F0812289E1880123684601F06B
:10E610005EF900281CBF02B0BDE8F081A2886188C5
:10E620000023684601F053F906001CBF02B0BDE8A4
:10E63000F0819DF800000127002801984FF00008A4
:10E6400008D000F5C47580F88971019890F8C80168
:10E65000C8B107E000F1FC0580F8FD70019890F862
:10E66000200108B13A261CE0E08868802089A88053
:10E670006088E880A088288101222846019912F04C
:10E68000E1FD2F700DE0E08868802089A880608817
:10E69000E880A088288100222846019912F0D2FD46
:10E6A0002F7085F8018002B03046BDE8F08130B5AA
:10E6B00087B00D460446008804A901F0F0F8002850
:10E6C0001CBF07B030BD9DF81000002814BF002209
:10E6D0000122E0880599B1F8483098428CBFC01AF1
:10E6E000002068806388B1F84A0083428CBF181A02
:10E6F0000020A8800020009001900290E088ADF8F2
:10E7000002002089ADF804006088ADF80600A088FA
:10E71000ADF80800684601E05C00002012F092FDB0
:10E720002089BDF80410401AE880A088BDF80810C0
:10E73000401A2881E088BDF80210411A6888814299
:10E74000C8BF084668806088BDF80610411AA888CE
:10E750008142C8BF0846A88007B0002030BD10B570
:10E7600004460BF025FB042806D00BF021FB0528FE
:10E7700002D00CF0BEFC28B111F0BDFC00281CBF7B
:10E780000C2010BD2078002816BF02280020012090
:10E79000E279611C11F032FE002814BF0020022033
:10E7A00010BD2DE9F04182B004460088694601F0B1
:10E7B00076F806001CBF02B0BDE8F081E846A078FC
:10E7C000002814BF05460725E17800290CBF07245F
:10E7D0000C4615F0040F16BF00280020012014F08D
:10E7E000040F16BF00290021012108424FF009073C
:10E7F0000AD001221146404601F081F8002838D0A5
:10E8000002B03846BDE8F08180B1002201214046C7
:10E8100001F075F80028F3D114F0040F29D001227B
:10E820001146404601F06BF818B343E081B1012274
:10E830000021404601F063F80028E1D115F0040FF3
:10E8400017D001221146404601F059F888B125E061
:10E8500015F0040F04F0040023D0C0B101221146CA
:10E86000404601F04CF800281CBF25F0040524F0B8
:10E87000040400219DF800200120002A019A1CD0E8
:10E8800082F89301019A92F8DC219AB33BE00022CE
:10E890000121404601F033F80028EAD025F00405B4
:10E8A000E7E70028E5D001220021404601F027F8E3
:10E8B0000028DED024F00404DBE782F80701019A87
:10E8C00092F82C213AB9019A92F806211AB9019AC4
:10E8D00092F87B200AB13A2608E0019A82F80601F4
:10E8E000019880F80851019880F80941019880F852
:10E8F000071116E0FFE7019A92F892211AB9019ADE
:10E9000092F87B200AB13A2608E0019A82F8920137
:10E91000019880F89451019880F89541019880F809
:10E92000931102B03046BDE8F081817831F00701E3
:10E9300007BFC17831F007011220704731E710B5E9
:10E9400004460178122086B0012918BF002904D09E
:10E9500002291EBF032906B010BD6178002918BF27
:10E96000012904D002291EBF032906B010BDA278D8
:10E9700032F005011CBF06B010BD12F0050F04BF38
:10E9800006B010BDE178B4F806C0638900291EBF47
:10E99000012906B010BDBCF1040F2EBF042B06B038
:10E9A00010BD052A3DD000BF0BF002FA042846D066
:10E9B0000BF0FEF9052842D0A0788DF80000A07871
:10E9C0008DF80C0060788DF8100020788DF80F001D
:10E9D000A07810F0010F35D0E078012808BF0220A0
:10E9E00003D000280CBF012000208DF80D00E08826
:10E9F000ADF802006089ADF80400A07810F0040FB3
:10EA000034D02079012808BF022003D000280CBF91
:10EA1000012000208DF80E002089ADF80600A089A5
:10EA200022E021792389A28900291EBF012906B08D
:10EA300010BD042B2EBF042A06B010BDB4E706B0EB
:10EA40000C2010BD10F0040F10D0E078012808BF92
:10EA5000022003D000280CBF012000208DF80E00FA
:10EA6000E088ADF806006089ADF8080068460AF055
:10EA7000C7FC002804BF03A808F0BAFD06B010BD0B
:10EA800010B5044602781220012A0FD0002A18BFC0
:10EA900010BD012A26D00BF08BF9052804D00AF00E
:10EAA00030FB002808BF10BD0C2010BD6178002984
:10EAB00018BF012906D0022918BF10BDA18800295E
:10EAC00008BF10BD6388002B1CBFA1880029E0D0BF
:10EAD00003EB83035B0001EB8101B3EB012F28BF44
:10EAE00010BDD6E708F072FC002804BF122010BD4C
:10EAF00008F081FC002008F02BFD002818BF10BD95
:10EB0000607808F017FD002818BF10BDA188608844
:10EB1000BDE810400AF0B6BC2DE9F04F91B00C46AC
:10EB2000AFF6E002D2E90012CDE90D120546607A97
:10EB300010F007034FF0120004BF11B0BDE8F08FD2
:10EB4000012B18BF022B05D0042B1EBF112011B0C2
:10EB5000BDE8F08F4FF0000C13F0010F4FF03001C3
:10EB600040F67B4238D075B1B4F80AC0278AACF1C0
:10EB7000040843F6FD76B0453CBFA7F10408B04554
:10EB800026D2BC4524D3E78AB4F81CC0B4F822A02E
:10EB9000268DB4F82E90B4F83480A7F1060B934577
:10EBA0003CBFACF1060B934512D2674598BFBAF54E
:10EBB000FA7F3EBFA6F10A0AFE4F17EB0A0707D2FB
:10EBC000B6EBDC0F04D9C14598BF4FF0010C03D957
:10EBD00011B00846BDE8F08F13F0020F29D004EB06
:10EBE0004C09B9F81680B9F81C60B9F822E0B9F8F8
:10EBF0002870B9F82EA0B9F83490A8F1060B5A4540
:10EC000084BFA6F1060B5A45E2D9B04598BFBEF5C0
:10EC1000FA7F3EBFA7F10A0BDFF8988318EB0B08C9
:10EC2000D6D2B7EBD60FD3D9CA4598BF0CF1010C99
:10EC3000CED813F0040F22D004EB4C03DE8AB3F8D5
:10EC40001CC0B3F822901F8DB3F82E809B8EA6F1C6
:10EC5000060A524584BFACF1060A5245B8D966454A
:10EC600098BFB9F5FA7F3EBFA7F10A06D14A12EB69
:10EC70000602ADD2B7EBDC0FAAD99845A8D8217807
:10EC800021B1012915D011B0BDE8F08FA17855B19F
:10EC9000002918BF01290CD0022918BF032908D068
:10ECA00011B0BDE8F08F00291EBF012911B0BDE8E9
:10ECB000F08F6178002918BF012905D002291EBFF5
:10ECC000032911B0BDE8F08F0BF072F804280CD0C6
:10ECD0000BF06EF8052808D0B74E307828B907F049
:10ECE00077FDA0F57F41FF3903D011B00C20BDE8BE
:10ECF000F08FB2480A90B2480B90B2480C900AAA22
:10ED000006210FA801F0B2FB050002BF092011B0D7
:10ED1000BDE8F08F032111F0EDFDB18AA5F8481090
:10ED2000F28AA5F84A20F07C0090B37C288801F094
:10ED30008AFC002818BFFFDF288806F001F82F881A
:10ED400005F10E094FF0000B4FF00A0A0421484666
:10ED500004F0E3FB484611F096FF062001F060FB4B
:10ED600080461CE003A9062001F03BFB03A801F04C
:10ED700016FB5FEA000B10D1BDF81000B84206D0B8
:10ED80000598042249460E3014F088FD70B103A89E
:10ED900001F005FB5FEA000BEED0A8F10108B8F125
:10EDA000000F07DDBBF1000FDCD007E0484611F093
:10EDB00073FFF2E7BBF1000F08BFFFDFD9F80000D7
:10EDC00011F085FFBAF1010A01D00028BED07EA063
:10EDD00005F1120700680290032102A804F074FBF9
:10EDE000002002A90A5C3A54401CC0B20328F9D39F
:10EDF000A08B6880608CA880208DE88095F85220D8
:10EE000095F85110308B0AF0A6FB0146A8622846FF
:10EE10000AF0E4FB4FF0000885F85E8085F85F801B
:10EE2000A07800281ABF0228012000206876D4F8B4
:10EE30000300C5F81A00B4F80700E8830DA905F12E
:10EE4000080014F008FF4FF0010985F8F890708968
:10EE5000B5F84A1005F1FC074A46884228BF084623
:10EE600095F852304FF4747B13F00C0F1CBF0BEB72
:10EE7000811189B25AD0B3898B4238BF1946B6F88E
:10EE80000EC0B5F848309C4528BF9C4695F851A067
:10EE90001AF00C0F1CBF0BEB83139BB24ED0368ABB
:10EEA0009E4238BF3346BCF11B0F18BFB3F5A47F99
:10EEB0004DD0F8803981A7F802C0BB80294638467A
:10EEC00012F0C0F987F800908DF8008001216846A3
:10EED00004F0FAFA9DF8000000F00701C0F3C10247
:10EEE0001144C0F3401008448DF80000401D2876FE
:10EEF00009283CBF083028760021284611F0FAFC8A
:10EF0000607808F06EFAA1782078E21C08F03CFAEC
:10EF1000002808BF122665D008F06DFAA178207885
:10EF2000E21C08F0E1FA060017D05BE0022B07BFF5
:10EF300089003C31C900703189B29CE7BAF1020FF7
:10EF400007BF9B003C33DB0070339BB2A7E71B2855
:10EF500018BFB1F5A47FACD1B6E7607A10F0040F0A
:10EF600014BF0820012008F009FA06003AD129460A
:10EF7000032008F0E3FA060034D1617A8DF8081016
:10EF8000617A11F0010F06D06089ADF80A00208A7D
:10EF9000ADF80C000120617A11F0020F18BF401C7F
:10EFA00011F0040F14D004EB40004189ADF80E10AD
:10EFB000008A0BE089F3FFFFDE060020A006002098
:10EFC00068000020CE06002011223300ADF81000AA
:10EFD00002A80AF015FA060004D128460AF0AAF998
:10EFE000060009D0288805F0ACFE2888062101F02B
:10EFF00081FA002818BFFFDF304611B0BDE8F08F5E
:10F000000146002088E538B5F74C207870B90AF041
:10F01000CFFE052805D007F0DBFBA0F57F41FF39C7
:10F0200004D068460AF069FA10B113E00C2038BD2C
:10F030000098008805F085FE00980621008801F000
:10F0400059FA002818BFFFDF01202070E748007838
:10F05000F3F76EFF002038BD70B542880446911F5B
:10F0600040F67B433020994228BF70BDA188A1F1B2
:10F07000060C9C4528BF70BD8A429CBFE288B2F551
:10F08000FA7F28BF70BD2289DFF864C3A2F10A03AA
:10F090001CEB030C28BF70BDB2EBD10F98BF70BD45
:10F0A0006189A289914288BF70BD00252088062110
:10F0B00001F00EFA78B190F8721061B990F8C810AA
:10F0C00000291CBF90F8C810042904D0D0F8F01013
:10F0D0000A7812B105E0022070BDD0F83C21127808
:10F0E0000AB13A2070BD05228A71D0F8F0100D8166
:10F0F000D0F8F020A1885181D0F8F020E1889181EA
:10F10000D0F8F0202189D181D0F8F0100A894B89FC
:10F110009A429EBF8A79082A9A4224BF122070BD63
:10F1200022884A80D0F8F00002210170002070BDD2
:10F13000F0B583B0054611F005FE002802BF12208D
:10F1400003B0F0BD0026A84F012429467C70B81CEE
:10F1500014F081FD7E706946062001F042F9002816
:10F1600018BFFFDF684601F01AF9002808BFBDF894
:10F1700004500AD1029880F8F840684601F00FF96F
:10F1800018B9BDF80400A842F4D103B00020F0BDC6
:10F1900010B504460088062101F09AF978B190F87C
:10F1A000721061B990F8C81000291CBF90F8C810FF
:10F1B000042904D0D0F8F0100A7812B105E002203A
:10F1C00010BDD0F83C2112780AB13A2010BD90F859
:10F1D000942012F0010F04BF0C2010BDD4F80220BF
:10F1E000D4F806304A608B60D0F8F01062898A81CA
:10F1F000D0F8F010E268C1F80E202269C1F81220A0
:10F200006269C1F81620A269C1F81A20D0F8F0206E
:10F2100003211170D0F8F00021884180002010BD3A
:10F22000017881B0EF296CD8D0E901C3634503D2DE
:10F23000817811F0080F64D04188ADF8001011F00A
:10F24000100F0CD011F0010F01F0020215D082B1A5
:10F2500011F0080F08BF11F0040F18D014E011F0DE
:10F26000080F4ED111F0010F18BF11F0020F48D155
:10F270000DE011F0040F0AD106E02AB111F0080FD9
:10F2800008BF11F0040F02D011F00F0F39D14188DF
:10F29000C27D11F0100F02D0012A0DD031E0012AF9
:10F2A00018BF032A2DD111F0100F05D1427E012A7B
:10F2B0001CBF022A032A24D1027B12B3072A20D8BA
:10F2C000427B002A18BF012A03D0022A18BF032A52
:10F2D00017D111F0040F1EBF827B002A012A10D122
:10F2E000427D002A18BF012A03D0022A18BF032A30
:10F2F00007D1C27E002A18BF012A02D1807E0F28C2
:10F3000002D9122001B07047B3F1807F02D2BCF164
:10F31000200F05D211F0080F02BF112001B0704775
:10F32000002001B0704770B50D4604460BF0E1FEB9
:10F3300000281CBF0C2070BD2046FFF771FF00287D
:10F3400018BF70BD00202870607B05F0A6FF204626
:10F35000BDE8704006F07AB810B5014682881220E8
:10F360001F2A88BF10BD4B78042B06D0032B08D072
:10F37000002A08BF10BD112010BD002A18BF10BD03
:10F38000F9E71046891D06F004F9002010BD1F287A
:10F3900084BF1220704770B50D46044606F0DBF8B6
:10F3A000002804BF122070BD2946204606F0DCF874
:10F3B000002070BD2DE9F0434278122183B0012A6C
:10F3C00003D903B00846BDE8F0830078012811D0C6
:10F3D0000028F6D10AF0FAFC04460BF011FB0028D5
:10F3E00040F0E78000F0D6B8DE0600205C00002088
:10F3F00089F3FFFF002AE4D005F04EFE58B105F076
:10F4000032FF10B906F0EAF828B10BF072FE0028BE
:10F4100040F0CF8003E003B01220BDE8F08305F098
:10F42000FEFDA0F57F41FF3940F0C38005F03DFFB0
:10F4300006F0CDF800287DD00022072101A801F0B8
:10F4400015F8040002BF092003B0BDE8F083FB48B3
:10F4500003218460204611F05BF9204606F00AFC87
:10F46000F74D0121A88AA4F84800E88AA4F84A00C8
:10F47000288B0BF032FCA062288B01210BF02DFCB5
:10F480000146002220460AF0A4FC06F0AEF810F077
:10F490000C0F08D001231A462146184611F009FE28
:10F4A000616A88426FD8E87C0090AB7CEA8AA98ABE
:10F4B000208801F0C8F8002818BFFFDF208805F079
:10F4C0003FFC20460BF064FB002818BFFFDF2146FD
:10F4D0006889B4F84A30002204F5C476984228BFFF
:10F4E0001846044691F852004FF4747710F00C0F50
:10F4F0001CBF07EB831083B233D0A889984238BF72
:10F500000346E889B1F848C0604528BF6046804698
:10F5100091F8510010F00C0F1CBF07EB8C1080B25B
:10F5200027D000BFB5F810C0844538BF6046B8F199
:10F530001B0F00E00EE018BFB0F5A47F24D0F480CC
:10F540003381A6F80280B080304611F07BFE0120A6
:10F5500030702AE000200BF01BFB002818BFFFDFF3
:10F5600023E0022807BF98003C30D800703083B2F7
:10F57000C3E7022807BF4FEA8C003C304FEACC00BB
:10F58000703080B2CEE714E01B2C18BFB3F5A47F17
:10F59000D5D10AE04CB1208805F0D3FB20880721A3
:10F5A00000F0A8FF002818BFFFDF002003B0BDE86F
:10F5B000F08303B00C20BDE8F0830121FAE610B51A
:10F5C0000C46072100F084FF002804BF022010BD74
:10F5D00090F8691109B10C2010BD90F8641014293D
:10F5E00012BF152990F8AA110029F4D12168C0F89A
:10F5F0006A116168C0F86E11A168C0F87211E16803
:10F60000C0F87611012180F86911002010BD10B5F5
:10F61000072100F05DFF002804BF022010BD90F814
:10F62000691109B10C2010BD90F86410142918BF9D
:10F630001529F7D1022180F86911002010BDF0B51D
:10F640000E464BF68032122183B0964217D8B6B1DF
:10F65000694600F024F900281CBF03B0F0BD0198F2
:10F6600000F15807841C258832462946384611F097
:10F6700045F82088A842F6D103B00020F0BD03B0C1
:10F680000846F0BD10B582B004460088694600F017
:10F6900006F900281CBF02B010BD01987F22014668
:10F6A00080F8602080F86120002280F86220A07835
:10F6B00081F82C00E07881F82D00207981F82E0067
:10F6C00002B0104610BD10B582B00C46694600F07D
:10F6D000E6F800281CBF02B010BD019890F8720037
:10F6E000002818BF0120207002B0002010BD10B506
:10F6F00082B00C46694600F0D2F800281CBF02B068
:10F7000010BD019890F82C0001281EBF0C2002B0FB
:10F7100010BD019890F86000207002B0002010BD6C
:10F7200070B50D461646072100F0D2FE002804BF32
:10F73000022070BD83884FF0010CC28841880CEB19
:10F74000430C65451AD342F2107C02FB0CF240F6E2
:10F75000C41C01FB0CF1B2FBF1F1491E8CB2B4F5F3
:10F76000FA7F88BF4FF4FA74A54238BF2C46621C5A
:10F77000591CB2FBF1F25143491E8BB290F896111D
:10F78000002908BF03843380002070BD10B50C46EB
:10F79000072100F09DFE002804BF022010BD80F864
:10F7A000D740002C1EBF90F8D51000290BF0B8FAF6
:10F7B000002010BD017800291CBF417800290ED01F
:10F7C00041881B2921BF81881B29C188022906D3B2
:10F7D0001C49026840680A6548650020704712208D
:10F7E000704710B5044609F0B3FE20460BF041FA0D
:10F7F000002010BD2DE9F04116460F4604460122B7
:10F800001146384609F0A7FE0546012138460BF09F
:10F8100064FA854228BF28460123E100503189B2AD
:10F82000E631884206D901F19602401AB0FBF2F0A7
:10F83000401C83B233800020BDE8F0815C000020D2
:10F84000DE060020A006002010B504460AF0B0FA3B
:10F85000042806D00AF0ACFA052802D00BF049FCC7
:10F8600008B10C2010BD601C10F09EFD207800F047
:10F87000010005F015FD207800F0010007F0B6FD4D
:10F88000002010BD10B504460BF033FC00281CBF4F
:10F890000C2010BD204605F090FE002010BD70B574
:10F8A0000C460546062100F013FE606010B10020F2
:10F8B000207070BD0721284600F00AFE6060002815
:10F8C00004BF022070BD01202070002070BD002800
:10F8D00008BFFB2006D04068002B14BFB0F84800DA
:10F8E000B0F84A001B2924BF8842B2F5A47F04D394
:10F8F000104880189CBF002070471220704710B538
:10F9000004468C46007813466168624638B101208F
:10F9100011F0CFFB6168496A884209D906E00020EE
:10F9200011F0C7FB6168496A884201D9012010BD06
:10F93000002010BDB8F7FFFF30B5058825F400445E
:10F9400021448CB24FF4004194420AD2121B92B26D
:10F950001B339A4201D2A94307E005F40041214339
:10F9600003E0A21A92B2A9431143018030BD0844BA
:10F97000083050434A31084480B2704770B51D4684
:10F9800016460B46044629463046049AFFF7EFFF19
:10F990000646B34200D2FFDF2821204614F04BF880
:10F9A0004FF6FF70A082283EB0B265776080B0F558
:10F9B000004F00D9FFDF618805F13C00814200D291
:10F9C000FFDF60880835401B343880B220801B2858
:10F9D00000D21B2020800020A07770BD816188614B
:10F9E00070472DE9F05F0D46C188044600F12809F3
:10F9F000008921F4004620F4004800F064FB10B1B7
:10FA00000020BDE8F09F4FF0000A4FF0010BB04519
:10FA10000CD9617FA8EB0600401A0838854219DC32
:10FA200009EB06000021058041801AE06088617FB3
:10FA3000801B471A083F0DD41B2F00DAFFDFBD42A1
:10FA400001DC294600E0B9B2681A0204120C04D0A5
:10FA5000424502DD84F817A0D2E709EB06000180D9
:10FA6000428084F817B0CCE770B5044600F1280254
:10FA7000C088E37D20F400402BB110440288438805
:10FA800013448B4201D2002070BD00258A4202D36C
:10FA90000180458008E0891A0904090C418003D0DF
:10FAA000A01D00F020FB08E0637F008808331844A5
:10FAB00081B26288A01DFFF73FFFE575012070BD90
:10FAC00070B5034600F12804C588808820F40046FC
:10FAD0002644A84202D10020188270BD988935883A
:10FAE000A84206D3401B75882D1A2044ADB2C01E13
:10FAF00005E02C1AA5B25C7F20443044401D0C88E0
:10FB0000AC4200D90D809C8924B10024147009886E
:10FB1000198270BD0124F9E770B5044600F128018F
:10FB2000808820F400404518208A002826D0A0892B
:10FB300010B9A069807F2871A089218A084480B209
:10FB4000A08129886A881144814200D2FFDF288879
:10FB50006988A389421800259A420DD119B1201D48
:10FB600000F0C1FA07E0637F62880833184481B26D
:10FB7000201DFFF7E1FEA5812582012070BD2DE942
:10FB8000F041418987880026044600F12805B942E2
:10FB900019D004F10A0800BF21F40040284441882C
:10FBA00019B1404600F09FFA08E0637F00880833EF
:10FBB000184481B262884046FFF7BEFE761C618918
:10FBC000B6B2B942E8D13046BDE8F0812DE9F04146
:10FBD00004460B4627892830A68827F40041B4F84C
:10FBE0000A8001440D46B74201D10020ECE70AB17A
:10FBF000481D106023B1627F691D184613F07AFE1C
:10FC00002E88698804F1080021B18A1996B200F0A3
:10FC10006AFA06E0637F62880833991989B2FFF7B0
:10FC20008BFE474501D1208960813046CCE7818831
:10FC3000C088814201D101207047002070470189AE
:10FC40008088814201D1012070470020704770B543
:10FC50008588C38800F1280425F4004223F400417C
:10FC600014449D421AD08389058A5E1925886388C9
:10FC7000EC18A64214D313B18B4211D30EE0437F8C
:10FC800008325C192244408892B2801A80B2233331
:10FC9000984201D211B103E08A4201D1002070BD27
:10FCA000012070BD2DE9F0478846C18804460089CF
:10FCB00021F4004604F1280720F4004507EB06096B
:10FCC00000F001FA002178BBB54204D9627FA81B7D
:10FCD000801A002503E06088627F801B801A083844
:10FCE00023D4E28962B1B9F80020B9F802303BB1FF
:10FCF000E81A2177404518DBE0893844801A09E08A
:10FD0000801A217740450ADB607FE1890830304462
:10FD100039440844C01EA4F81280BDE8F087454568
:10FD200003DB01202077E7E7FFE761820020F4E7AB
:10FD30002DE9F74F044600F12805C088884620F4D5
:10FD4000004A608A05EB0A0608B1404502D200204D
:10FD5000BDE8FE8FE08978B13788B6F8029007EBEE
:10FD60000901884200D0FFDF207F4FF0000B50EAEE
:10FD7000090106D088B33BE00027A07FB946307167
:10FD8000F2E7E18959B1607F2944083050440844C2
:10FD9000B4F81F1020F8031D94F821108170E28937
:10FDA00007EB080002EB0801E1813080A6F802B001
:10FDB00002985F4650B1637F30880833184481B29F
:10FDC0006288A01DFFF7B8FDE78121E0607FE1892F
:10FDD00008305044294408442DE0FFE7E089B4F896
:10FDE0001F102844C01B20F8031D94F821108170B7
:10FDF00009EB0800E28981B202EB0800E08137805C
:10FE000071800298A0B1A01D00F06DF9A4F80EB0A9
:10FE1000A07F401CA077A07D08B1E088A08284F874
:10FE200016B000BFA4F812B084F817B001208FE715
:10FE3000E0892844C01B30F8031DA4F81F10807807
:10FE400084F82100EEE710B5818800F1280321F441
:10FE500000442344848AC288A14212D0914210D027
:10FE6000818971B9826972B11046FFF7E8FE50B915
:10FE70001089283220F40040104419790079884212
:10FE800001D1002010BD184610BD00F12803407FAD
:10FE900008300844C01E1060088808B9DB1E1360D3
:10FEA00008884988084480B270472DE9F04100F184
:10FEB0002806407F1C4608309046431808884D8825
:10FEC000069ADB1EA0B1C01C80B2904214D9801AE1
:10FED000A04200DB204687B298183A46414613F00C
:10FEE000DDFC002816D1E01B84B2B844002005E0F8
:10FEF000ED1CADB2F61EE8E7101A80B20119A94256
:10FF000006D8304422464146BDE8F04113F0C6BC55
:10FF10004FF0FF3058E62DE9F04100F12804407F12
:10FF20001E46083090464318002508884F88069AD8
:10FF3000DB1E90B1C01C80B2904212D9801AB04230
:10FF400000DB304685B299182A46404613F0D2FCB1
:10FF5000701B86B2A844002005E0FF1CBFB2E41E5F
:10FF6000EAE7101A80B28119B94206D82118324640
:10FF7000404613F0BFFCA81985B2284624E62DE9B7
:10FF8000F04100F12804407F1E4608309046431897
:10FF9000002508884F88069ADB1E90B1C01C80B2ED
:10FFA000904212D9801AB04200DB304685B29818D0
:10FFB0002A46414613F09EFC701B86B2A8440020DE
:10FFC00005E0FF1CBFB2E41EEAE7101A80B28119F7
:10FFD000B94206D820443246414613F08BFCA8199A
:10FFE00085B22846F0E5401D704710B5044600F183
:10FFF0002801C288808820F400431944904206D02A
:020000040001F9
:10000000A28922B9228A12B9A28A904201D1002083
:1000100010BD0888498831B1201D00F064F8002027
:100020002082012010BD637F62880833184481B2AA
:10003000201DFFF781FCF2E70021C1810177418299
:10004000C1758175704703881380C28942B1C28827
:1000500022F4004300F128021A440A60C089704764
:100060000020704710B50446808AA0F57F41FF3913
:1000700000D0FFDFE088A082E08900B10120A075F8
:1000800010BD4FF6FF71818200218175704710B558
:100090000446808AA0F57F41FF3900D1FFDFA07DB3
:1000A00028B9A088A18A884201D1002010BD012072
:1000B00010BD8188828A914201D1807D08B10020E3
:1000C00070470120704720F4004221F400439A4217
:1000D00007D100F4004001F40041884201D0012022
:1000E00070470020704730B5044600880D4620F464
:1000F0000040A84200D2FFDF21884FF4004088432F
:100100002843208030BD70B50C00054609D0082C6E
:1001100000D2FFDF1DB1A1B2286800F044F8201D15
:1001200070BD0DB100202860002070BD0021026864
:1001300003E093881268194489B2002AF9D100F0CB
:1001400032B870B500260D460446082900D2FFDFFC
:10015000206808B91EE0044620688188A94202D0C0
:1001600001680029F7D181880646A94201D10068BB
:100170000DE005F1080293B20022994209D3284408
:10018000491B02608180216809682160016020604C
:1001900000E00026304670BD00230B608A800268B4
:1001A0000A600160704700234360021D0181026004
:1001B0007047F0B50F460188408815460C181E465A
:1001C000AC4200D3641B3044A84200D9FFDFA01921
:1001D000A84200D9FFDF3819F0BD2DE9F04188466B
:1001E00006460188408815460C181F46AC4200D3CD
:1001F000641B3844A84200D9FFDFE019A84200D9A7
:10020000FFDF70883844708008EB0400BDE8F0819F
:100210002DE9F041054600881E461746841B884696
:10022000BC4200D33C442C8068883044B84200D99A
:10023000FFDFA019B84200D9FFDF6888304468802A
:1002400008EB0400E2E72DE9F04106881D4604466C
:10025000701980B2174688462080B84201D3C01B6F
:1002600020806088A84200D2FFDF7019B84200D910
:10027000FFDF6088401B608008EB0600C6E730B5F2
:100280000D460188CC18944200D3A41A40889842A5
:1002900000D8FFDF281930BD2DE9F041C94D0446D3
:1002A0009046A8780E46A04200D8FFDF05EB8607EF
:1002B000B86A50F8240000B1FFDFB868002816D0F3
:1002C000304600F046F90146B868FFF73AFF0500EE
:1002D0000CD0B86A082E40F8245000D3FFDFBA488B
:1002E0004246294650F82630204698472846BDE821
:1002F000F0812DE9F84305001E4602EB0600174683
:100300008946C4B200952FD000218846FF2800D925
:10031000FFDFE81C20F00300A84200D0FFDFB1455A
:1003200000D9FFDF4946DFF89C92684689F8001043
:1003300089F8017089F8024089F8034089F804407F
:1003400089F8054089F8066089F80770414600F091
:1003500009F9002142460F464B460098C01C20F088
:100360000300009012B10FE00121CEE703EB8106FC
:10037000B062002006E000BFD6F828C04CF820701C
:10038000401CC0B2A042F7D30098491C00EB840087
:10039000C9B200900829E0D3401BBDE8F88310B52E
:1003A000044603F009FC08B1102010BD2078854AEE
:1003B000618802EB800092780EE0836A53F8213066
:1003C00043B14A1C6280A180806A50F82100A0607D
:1003D000002010BD491C89B28A42EED861800520F8
:1003E00010BD70B505460C46084603F0E5FB08B1A4
:1003F000102070BD082D01D3072070BD257000208E
:10040000608070BD0EB56946FFF7EBFF00B1FFDFFE
:100410006846FFF7C4FF08B100200EBD01200EBDE5
:1004200010B50446082800D3FFDF6648005D10BD04
:100430003EB5054600246946FFF7D3FF18B1FFDF3C
:1004400001E0641CE4B26846FFF7A9FF0028F8D079
:100450002846FFF7E5FF001BC0B23EBD5949897829
:10046000814201D9C0B27047FF2070472DE9F041A9
:10047000544B062903D007291CD19D7900E00025A3
:1004800000244FF6FF7603EB810713F801C00AE062
:100490006319D7F828E09BB25EF823E0BEF1000FA5
:1004A00004D0641CA4B2A445F2D833460380184695
:1004B000B34201D100201AE7BDE8F041ECE6A0F517
:1004C0007F43FF3B01D0082901D300207047E3E6BA
:1004D000A0F57F42FF3A0BD0082909D2394A937818
:1004E000834205D902EB8101896A51F820007047E7
:1004F000002070472DE9F04104460D46A4F57F41E8
:1005000043F20200FF3902D0082D01D30720EEE6A6
:100510002C494FF000088A78A242F8D901EB8506F1
:10052000B26A52F82470002FF1D0274839462030A3
:1005300050F8252020469047B16A284641F824808B
:1005400000F007F802463946B068FFF725FE0020A4
:10055000CDE61D49403131F810004FF6FC71C01C4A
:10056000084070472DE9F843164E8846054600249A
:100570002868C01C20F0030028602046FFF7E9FF30
:10058000315D4843B8F1000F01D0002200E02A6835
:100590000146009232B100274FEA0D00FFF7B3FD8C
:1005A0001FB106E001270020F8E706EB8401009A5E
:1005B0008A602968641C0844E4B22860082CD7D3F8
:1005C000EBE60000FC060020543E020070B50E462B
:1005D0001D46114600F0D4F804462946304600F086
:1005E000D8F82044001D70BD2DE9F04190460D461D
:1005F00004004FF0000610D00027E01C20F003009C
:10060000A04200D0FFDFDDB141460020FFF77BFDB7
:100610000C3000EB850617B112E00127EDE7614FC2
:1006200004F10C00A9003C602572606000EB8500BD
:100630002060606813F0FFF941463868FFF763FDFA
:100640003046BDE8F0812DE9FF4F564C804681B021
:1006500020689A46934600B9FFDF2068027A424537
:1006600003D9416851F8280020B143F2020005B0D7
:10067000BDE8F08F5146029800F082F886B25846E5
:100680000E9900F086F885B27019001D87B22068B7
:10069000A14639460068FFF754FD04001FD067806B
:1006A00025802946201D0E9D07465A4601230095A8
:1006B000FFF764F92088314638440123029ACDF8C7
:1006C00000A0FFF75BF92088C1193846FFF786F9CB
:1006D000D9F800004168002041F82840C7E704200D
:1006E000C5E770B52F4C0546206800B9FFDF2068CC
:1006F000017AA9420ED9426852F8251051B100235F
:1007000042F825304A880068FFF746FD216800203E
:100710000A7A08E043F2020070BD4B6853F82030BB
:1007200033B9401CC0B28242F7D80868FFF7FEFC1C
:10073000002070BD70B51B4E05460024306800B91E
:10074000FFDF3068017AA94204D9406850F82500DB
:1007500000B1041D204670BD70B5124E0546002440
:10076000306800B9FFDF3068017AA94206D94068D5
:1007700050F8251011B131F8040B4418204670BD13
:1007800010B50A460121FFF7F2F8C01C20F0030063
:1007900010BD10B50A460121FFF7E9F8C01C20F092
:1007A000030010BD7000002070B5044600780E46AE
:1007B000012813D0072802D00B2813D10EE0A0681F
:1007C00061690578052003F085F9052D0AD07823A5
:1007D00000220520616903F0D3F803E00520616978
:1007E00003F078F931462046BDE8704001F016B9B3
:1007F00010B500F13902C3799478411D64F0030407
:100800002340C371DB070DD04B79547923404B71E2
:100810000B79127913400B718278C9788A4200D91A
:10082000817010BD00224A710A71F5E741780129F3
:1008300000D00C21017070472DE9F74F88B00020DF
:100840008C690D468DF80400012709781646384654
:100850004FF007094FF0110A4FF00A0B262973D207
:10086000DFE811F02600AF02F10209034F035A033B
:100870007303A103B603DF030C042F0449048404AB
:100880009504B404BF04DF04010529054C057B056C
:100890009605A405C405C605CF05030626067A06F7
:1008A000B906BE06F10613078C07B10779077E0764
:1008B00014B121781D2929D0D5F808805FEA0801F4
:1008C00042D001208DF80400686A02228DF80820C9
:1008D00006908DF809B0286A0390A8880028EFD008
:1008E00098F8001091B10F2910D27DD2DFE801F005
:1008F0007C134BDBFDFCFBFAF9F82C089EF7F600A5
:10090000022821D124B120780C2801D00027F1E35E
:100910008DF80420AAE10520696A03F0DBF8A888B5
:100920000728EED1204601F074F8022809D02046AD
:1009300001F06FF8032808D9204601F06AF807286B
:1009400003D20120207005E0B0E1002CB8D020785F
:100950000128D6D198F80400C11F0A2903D300BF8B
:1009600085F81CB02CE2A070D8F80010A163B8F88C
:100970000410A18798F8060084F83E000120287032
:100980000320207046E00728BBD1002C98D02078A7
:100990000D28B6D198F8031094F83B20C1F3C0009D
:1009A000C2F3C002104201D0062000E007208907F0
:1009B00007D198F805100142D2D198F806100142EB
:1009C000CED194F83D2098F8051020EA0202114299
:1009D000C6D194F83E2098F8061090430142BFD14A
:1009E00098F80400C11F00E0E8E10A29B8D2617F4D
:1009F000814201D9062075E3D8F800106160B8F88B
:100A00000410218198F80600A072012028700E20A1
:100A1000207003208DF80400686A069004F1390004
:100A20000290601D0390173004900BE2412890D192
:100A3000204600F0EEFF042802D1E078C00704D180
:100A4000204600F0E6FF0F289ED1A88CD5F80C8038
:100A500080B24FF04009676AFFF76CFE3A460827FC
:100A600041464B460097FFF756FA0D208DF80400DB
:100A7000686A0690606A0290002101A8FFF794FE60
:100A80002078042806D0A07F38B1012805D003289B
:100A900006D062E305202070AFE184F800A035E7BE
:100AA0001220207065E01128C1D1204600F0B1FF6E
:100AB000042802D1E078C0070FD0204600F0A9FF3B
:100AC000062805D1E078C00707D1A07F022804D00E
:100AD000204600F09EFF1128A9D107E0AAE07AE0A5
:100AE00051E130E103E1E2E0C8E01AE0102208F150
:100AF000010104F1480012F0FDFE607801280DD0DC
:100B000012202070E078C00703D0A07F88B30128AE
:100B10002FD085F800B08DF804B0C7E384F80090BA
:100B200027E0112890D1204600F073FF082804D058
:100B3000204600F06EFF132886D12869D8B1686975
:100B4000C8B104F17800102208F10101074612F043
:100B5000D1FE2078082812D014202070E078C00739
:100B60000FD0A07F022818D06178022912D0032864
:100B7000CFD10420F0E300208DF8040096E0092096
:100B8000EBE70B202870296901204870206CC1E92F
:100B900001073CE208B101286FD10B2028702969B8
:100BA00081F80190606A4860206AC1E9020723E287
:100BB000206CE2780068C2F34402521ED04000F07C
:100BC000010040F0800000E000200874E06A486105
:100BD00026E20746FEE31128D0D1204600F019FF97
:100BE0000A2802D1E078C00704D1204600F011FFA6
:100BF0001528C3D1102208F1010104F1480012F0B8
:100C000079FE20780A2810D0162020701220287033
:100C100029690920487004F1580048602030886034
:100C20001038C860206C086162E30B2020709BE2E2
:100C30002870EFE30228A1D1204600F0EAFE042844
:100C400004D3204600F0E5FE082809D3204600F032
:100C5000E0FE0E2892D3204600F0DBFE12288DD253
:100C6000A07F02288AD110208DF80400686A0690BF
:100C700098F801008DF80800F6E321E20228ABD1D4
:100C8000204600F0C6FE002810D0204600F0C1FE2D
:100C90000128F9D0204600F0BCFE0C28F4D0042036
:100CA0008DF8080098F801008DF80900D3E11128AB
:100CB000FCD1002CFAD020781728F7D16178E06AAF
:100CC000022912D05FF0000101EB4101182606EB6A
:100CD000C1011022405808F1010112F00BFE05205D
:100CE000696A00F089FE267010E60121ECE70B2806
:100CF000DCD1002CDAD020781828D7D16178E06ACE
:100D000002291CD05FF0000101EB4101102202EB2F
:100D1000C1014158B8F8010008806078E16A0228F2
:100D20000FD0002000EB4002142000EBC200095855
:100D3000404650F8032F0A604068486039E00121BE
:100D4000E2E70120EEE71128B0D1002CAED02078E8
:100D50001928ABD16078E16A022812D05FF0000058
:100D600000EB40021C2000EBC2001022085808F1E2
:100D7000010112F0BFFD0520696A00F03DFE1A2056
:100D8000BDE00120ECE7082890D1002C8ED020781F
:100D90001A288BD1E06A98F80120017862F34701A4
:100DA0000170E16AD8F8022041F8012FB8F8060076
:100DB00088800520696A00F01FFE15E385F81C9005
:100DC000F0E33078012893D11C2204F11C007168F3
:100DD00012F0D5FDE07994F83B10C00800EAD1008C
:100DE000E17860F30001E170207F002879D120785C
:100DF00003280AD0C8073FF455AE032028708DF8A9
:100E000004B0686A06904120A3E3607FA17888421D
:100E10003FF6F0AD02272771E179204621F0E0018D
:100E2000E171617A21F0F0016172A17A21F0F001A3
:100E3000A172FFF7DDFC2F708DF804B0686A069090
:100E40008DF80890FAE3307811289DD18DF8049040
:100E5000696A0691B16800208DF814000391ADF81D
:100E6000089008466168016021898180A17A8171BA
:100E700004202070F8E23078112885D18DF8049094
:100E8000686A0690301D02AB07C883E8070041205E
:100E9000ADF8080000208DF8140008460C21017000
:100EA000A88CCA4680B2F7684FF04009D4F8208079
:100EB000FFF752FC42464FF0080839464B46CDF842
:100EC0000080FFF75CF8002101A8FFF76DFCE078D7
:100ED00020F03E00801CE0702078052802D00F2012
:100EE0000DE0B7E0A07F20B1012802D0032803D095
:100EF00035E184F800A03CE684F8008006E5207027
:100F000004E530780328A0D170680168A1664068C4
:100F1000E0660520287044E23078032895D1706897
:100F20000168216740686067206C58B9A07F18B1DC
:100F3000012801D0062031E185F80090FE482064A8
:100F4000606446E385F8009043E33078022894D14A
:100F5000307900287ED1A07F02280BD00328F1D160
:100F6000607801280BD0A07994F83A1001280AD0B3
:100F7000F1480BE0B06800286DD0206411E0A17941
:100F800094F83A00F2E7B0680028F5D02064E078E1
:100F9000C00701D0012901D0E74802E0F06800282D
:100FA000EAD06064CEE78DF804B0696A0691E17812
:100FB0005846C90709D06178022903D1A17F29B118
:100FC000012903D0A17F032900D0082028706FE1F8
:100FD0003178112997D1B168296209212970E27805
:100FE0002969D2070DD081F80190206A4860606AB3
:100FF000886004F16800C860A07F02287FF4E4AD37
:10100000D6E54870206C486004F16800886004F1FF
:101010003800C860201D0861206B4861606B8861E2
:101020001BE2E1783078C90701D0062100E00A21EF
:1010300088428CD1207807281DD084F800A000BFFA
:101040008DF80490686A0690286A0390ADF808A0AD
:10105000002401E0BFE02AE28DF81440032100F8EB
:10106000011B1022716812F045FC002101A8FFF756
:101070009BFB2C624AE408202070E1E730781128BD
:10108000A8D18DF80490686A0690B068039000209B
:101090008DF814000398ADF808A0042100F8011B96
:1010A000102204F1680112F025FC002101A8FFF7CD
:1010B0007BFB2078092801D0132020E784F800B0BA
:1010C00016E0E1783078C90701D0062100E00A2156
:1010D0008842AED1102204F14800716812F0DEFBA4
:1010E00010B1042028777DE3207809283FF411AD62
:1010F0000C209DE56EE2E078C10735D0A17F012983
:1011000002D002291BD02CE00D202870296981F81B
:1011100001B06078012809D0206A4860606A886060
:1011200004F16800C860103008614FE5606A4860EB
:10113000206A886004F17800C8601038F4E7C0F3D2
:10114000440114290DD24FF0006101EBB0104FEAB9
:10115000B060E0706078012801D01020A1E4062082
:10116000CDE66078012885D00E2061E53078092829
:1011700086D185F800B00F208DF80400686A0690CB
:1011800070680290002101A8FFF70EFBE9E7E07804
:10119000C00706D0A07F01281FD10F20287004208F
:1011A000FFE015202870296902204870206C4860F3
:1011B0006078012805D004F1780088601038C86094
:1011C0004BE104F1680088601030F8E730780228BD
:1011D000CED1307908B1287702E3102028700E2094
:1011E000DFE030781328F7D185F800A029690820BE
:1011F000487070684860607801280DD004F168007C
:1012000088601030C860206B0861606B486104F131
:1012100058008861A06A20E004F1780088601038E6
:10122000F0E730780728D7D16078012819D1A17864
:10123000A06A0844C1F1100112F0DBFB12202870F3
:1012400029690920487004F15800486020308860FE
:101250001038C860206C086143E0C861E06A086229
:10126000FBE01320B8E130780828B5D1102204F152
:101270004800716812F012FB08B10B2032E72078A9
:101280000B28EED02046FFF7B3FAA078A16A0A181F
:10129000C0F11001104612F0ACFB16202870082097
:1012A0008DF80400686A069000206FE0686A069076
:1012B0008DF808A0C2E1307811288DD1B06828627D
:1012C0001420287029690920487004F158004860EA
:1012D000103088601030C860606C08616078012848
:1012E00006D004F139004861206B8861606BB4E777
:1012F000601D4861606B8861206BAEE7307808281C
:1013000091D18DF80490686A0690286A00270390AE
:10131000ADF808A08DF814700D2100F8011B102203
:10132000716812F0E7FA002101A8FFF73DFA2F6279
:101330006078012804D001E0C53F02001520DEE5F9
:101340001620287008208DF80400686A029706901D
:10135000A0788DF80C0071E150E030780B2884D132
:10136000162028706078022802D12046FFF740FA44
:10137000A07871680A18C0F11001104612F039FB0C
:1013800008208DF80400686A069070680290DFE714
:1013900030780F2891D1E079C0076FD017202870DE
:1013A00009208DF80400686A069047E1307810281B
:1013B0007DD11422311D04F11C0012F0E0FAE16A23
:1013C000208DA1F80900E16AA078C871E17901F0E7
:1013D000030100E0F4E1E26A1172E16A627A0A73E1
:1013E000E16AA07A81F82400212021E41920F3E0A9
:1013F000307811285BD1B06828621A202870052047
:10140000CFE73078032852D16078E16A022802D011
:10141000012001E0DDE0002000EB4002142000EBA1
:10142000C20273688A5819681160596851601B219B
:101430002970D5E9041205234B70636A4B60677805
:10144000E36A022F01D0012700E0002707EB4707DE
:1014500000EBC7001858C1E90202686A48620898A0
:1014600000F0F3FAFFF7B5BBD3E130780E281ED1B8
:101470006078E26A022802D0012001E06AE10020DF
:1014800000EB4001102000EBC1000223105809328C
:10149000716810F03DFC1C202870296904204870F8
:1014A000206A4860E06A09308860FE4887E678E094
:1014B00030780D2875D16178E06A022901D00121C8
:1014C00000E0002101EB4101182707EBC101A278E0
:1014D0004058716812F00EFA6078E16A022801D073
:1014E000012000E0002000EB400207EBC200B846FC
:1014F0000958A0780A18C0F11001104612F079FAC4
:101500008DF80490686A0690286A00270390ADF869
:1015100008A08DF81470062101706178E26A022932
:1015200001D0012100E0002101EB410308EBC301E0
:10153000401C5158102212F0DDF9002101A8FFF7DC
:1015400033F91D202F6228708DF804B0686A069068
:101550000B208DF8080071E03178112921D18DF828
:101560000490696A0691B16803910B21ADF80810E7
:10157000039981F800906378E26A022B01D001237D
:1015800000E0002303EB4303102707EBC303D2580B
:101590001288A1F801206278E36A022A03D00122AE
:1015A00002E09FE01EE1002202EB4207142202EB60
:1015B000C7029A58136841F8033F52684A605CE0DA
:1015C0002120287000208DF81400014601A8FFF7A3
:1015D000EBF8032722E11F2028708DF804B065E6A0
:1015E000307811287ED18DF80490686A0690B06832
:1015F000039000208DF814000398ADF808A0082788
:1016000007706178E26A022901D0012100E000211F
:1016100001EB41031C2101EBC301401C5158102276
:1016200012F068F9002101A8FFF7BEF82020287009
:101630008DF804B0686A06908DF80870314601A8EC
:10164000FFF7B2F80EE7317811294BD18DF80490ED
:10165000696A0691B16803910821ADF808100399F1
:1016600009220A70E269127852084A70E26952F857
:10167000013FC1F802309288CA8021781C299FD18D
:10168000242129708DF81400D8E7E078C00702D033
:101690004FF0060C01E04FF0070C6078022809D0EB
:1016A0004FF0000000EB040101F1090105D04FF0FB
:1016B000010004E04FF00100F4E74FF000000B7868
:1016C000204413EA0C030B7010F8092F02EA0C02F5
:1016D000027004D14FF01B0C84F800C0D2B394F810
:1016E00001C000E049E0BCF1010F00D093B990F8CF
:1016F00000C05FEACC7804D02CF0010707701827EF
:1017000006E05FEA8C7805D52CF0020707701E27EB
:101710002F70032794F801C0BCF1020F00D092B9DA
:1017200091F800C05FEACC7804D02CF001070F706C
:10173000172106E05FEA8C7805D52CF002070F70C0
:101740001921217000270078D0BBCAB3C3BB1C206D
:10175000207035E002E03078122841D12520C8E41D
:10176000207801283CD00C283AD02046FFF75EF8BC
:101770000B208DF80400686A069031E031784FF054
:101780002308112905D012203070032785F8008026
:1017900044E08DF80490696A0691B16803918DF870
:1017A000140002210398ADF8081005210170297F6B
:1017B0004170314601A8FEF7F7FF074685F8008023
:1017C000012F0DD02AE08DF80400686A06900320EE
:1017D0008DF80800287F8DF809000020287712E096
:1017E000287F80B11D202070222028708DF804B041
:1017F000686A069002208DF80800314601A8FEF7BD
:10180000D3FF07460AE00CB1FE2020709DF80400CB
:1018100020B1002101A8FEF7C7FF2BE40BB038462A
:10182000BDE8F08FF0B587B00C464E6900218DF809
:10183000041001202578034602274FF0070C85B1DC
:10184000012D54D0022D3AD1FE2030708DF8003099
:10185000606A059003208DF80400207E8DF8050055
:1018600064E02179012926D002292DD0032928D02E
:10187000042924D1B17F022921D131780D1F042DF3
:1018800004D30A3D032D01D31D2918D12189022932
:1018900015D300BF8DF80470237020899DF80410C3
:1018A000884201E0BD3F020017D20A208DF80000F7
:1018B000606A059057E070780128EBD0052007B0EA
:1018C000F0BD1D203070E5E771780229F6D131783E
:1018D0000C29F4D18DF804C0DEE71120083402F899
:1018E000040B94E80B0082E80B000320E7E715786F
:1018F000112DE4D18DF800C0656A059595680295B3
:101900008DF8101094F804E0BEF1010F13D0BEF171
:10191000020F2DD0BEF1030F1CD0BEF1040FCED1AB
:10192000ADF804700E202870207E68700021684693
:10193000FEF73AFF0CE0ADF804700B202870207E13
:10194000002100F01F0068706846FEF72DFF377019
:101950000020B4E7ADF804708DF810300520287031
:10196000207E6870277011466846FEF71DFFA6E7C7
:10197000ADF804C02B70207F6870607F00F001001C
:10198000A870A07F00F01F00E870E27F2A71C007F6
:101990001CD094F8200000F00700687194F8210032
:1019A00000F00700A87100216846FEF7FDFE2868D8
:1019B000B063A888B087A87986F83E00A06940780F
:1019C00070772879B0700D203070C1E7A971697106
:1019D000E9E700B587B005280CD101208DF800009B
:1019E0008DF80400002005918DF805000146684639
:1019F000FEF7DAFE07B000BD70B50C46054602F0F2
:101A000069F821462846BDE870407823002201F09D
:101A1000B7BF08B1007870470C20704770B50C0054
:101A200005784FF000010CD021702146F3F767FBD9
:101A300072482178405D884201D1032070BD0220A8
:101A400070BDF3F75CFB002070BD027B032A05D05C
:101A500000220A704B780B2B02D003E00420704761
:101A60000A770A62027B9300521C0273C150032062
:101A70007047F0B587B00F4605460124287B05EB7B
:101A8000800050F8046C7078411E0C290AD25B4922
:101A90003A46123101EB8000314650F8043C2846AA
:101AA000984704460CB1012C11D1287B401E10F040
:101AB000FF00287301D00324E0E70C208DF800001C
:101AC000706A0590002101966846FFF7A7FF032C76
:101AD000D4D007B02046F0BD70B515460A4604467E
:101AE00029461046FFF7C5FF064674B12078FE2848
:101AF0000BD1207E30B100202870294604F10C0063
:101B0000FFF7B7FF2046FEF791FE304670BD7047E5
:101B100070B50E460446882111F08DFF0225012E76
:101B200003D0022E04D0052070BD0120607000E0BB
:101B300065702046FEF77AFEA577002070BD28B1BB
:101B4000027E1AB10A4600F10C01C5E70120704778
:101B500010B5044686B0052001F0BCFF2078FE28B1
:101B600006D000208DF8000069462046FFF7E7FF09
:101B700006B010BD7FB50E4600218DF80C104178DF
:101B80000B2903D00C2903D0002405E0846900E070
:101B900044690CB1217E91B16D4601462846FFF79C
:101BA00054FF032809D1324629462046FFF794FF07
:101BB0009DF80C10002900D0042004B070BD04F181
:101BC0000C05EAE710B590B00C4607900B480421CD
:101BD000801E08900A488DF8191009900F926946E6
:101BE00006A8FFF7C7FF002805D11022204601995B
:101BF00011F080FE002010B010BD0000A63E0200D3
:101C0000BD3F020070B50D46040011D085B1210121
:101C1000284611F0EEFE10224E49284611F06AFEC9
:101C20004C4801210838018044804560002070BD87
:101C3000012070BD70B5474E00240546083E10E0F7
:101C40007068AA7B00EB0410817B914208D1C17BB4
:101C5000EA7B914204D10C22294611F01FFE30B1DB
:101C6000641C30888442EBDB4FF0FF3070BD2046AF
:101C700070BD70B50D46060006D02DB1FFF7DAFF36
:101C8000002803DB401C14E0102070BD314C083CE0
:101C900020886288411C914201D9042070BD61688E
:101CA000102201EB0010314611F024FE2088401C68
:101CB00020802870002070BD70B514460D0018D02B
:101CC000BCB10021A170022802D0102811D105E07A
:101CD000288870B10121A170108008E02846FFF724
:101CE000A9FF002805DB401CA070A88920800020E7
:101CF00070BD012070BD70B5054614460E000BD0B6
:101D000000203070A878012808D005D91149A1F128
:101D100008010A8890420AD9012070BD24B12878B0
:101D200020702888000A5070022008700FE064B10B
:101D30004968102201EB00112046103911F0DAFD3C
:101D4000287820732888000A6073102030700020E3
:101D500070BD00007C0000202DE9F04190460C464B
:101D600007460025FE48072F00EB881607D2DFE85C
:101D700007F00707070704040400012500E0FFDF60
:101D800006F81470002D13D0F548803000EB880160
:101D900091F82700202803D006EB4000447001E0B2
:101DA00081F8264006EB44022020507081F827403D
:101DB000BDE8F081F0B51F4614460E460546202AC0
:101DC00000D1FFDFE649E648803100EB871C0CEBD1
:101DD000440001EB8702202E07D00CEB460140782F
:101DE0004B784870184620210AE092F82530407858
:101DF00082F82500F6E701460CEB410005704078BB
:101E0000A142F8D192F82740202C03D00CEB4404D7
:101E1000637001E082F826300CEB410420236370EC
:101E200082F82710F0BD30B50D46CE4B4419002284
:101E3000181A72EB020100D2FFDFCB48854200DDA9
:101E4000FFDFC9484042854200DAFFDFC548401C39
:101E5000844207DA002C01DB204630BDC148401C1B
:101E6000201830BDBF48C043FAE710B504460168EA
:101E7000407ABE4A52F82020114450B10220084452
:101E800020F07F40F0F767FE94F90810BDE810409D
:101E9000C9E70420F3E72DE9F047B14E803696F804
:101EA0002D50DFF8BC9206EB850090F8264034E018
:101EB00009EB85174FF0070817F81400012806D022
:101EC00004282ED005282ED0062800D0FFDF01F0F0
:101ED000E5F8014607EB4400427806EB850080F800
:101EE000262090F82720A24202D1202280F8272025
:101EF000084601F0DEF82A4621460120FFF72CFFB4
:101F00009B48414600EB041002682046904796F833
:101F10002D5006EB850090F82640202CC8D1BDE856
:101F2000F087022000E003208046D0E710B58C4CFB
:101F30002021803484F8251084F8261084F8271096
:101F4000002084F8280084F82D0084F82E10411E0B
:101F5000A16044F8100B2074607420736073A07348
:101F60008449E07720750870487000217C4A103C55
:101F700002F81100491CC9B22029F9D30120F0F759
:101F8000D8FC0020F0F7D5FC012084F82200F0F7FF
:101F9000A1FF7948F0F7ADFF764CA41E207077487A
:101FA000F0F7A7FF6070BDE81040F0F74FBC10B528
:101FB000F0F771FC6F4CA41E2078F0F7B3FF607847
:101FC000F0F7B0FFBDE8104001F0A0B82020704746
:101FD0002DE9F34F624E0025803606EB810A89B069
:101FE0009AF82500202822D0691E029160490095A8
:101FF00001EB00108146D0E90112C0680391CDE9E0
:102000000420B08BADF81C00B07F8DF81E009DF849
:102010001500C8B10227554951F820400399E2192B
:10202000114421F07F41019184B102210FE0012090
:10203000F0F77FFC0020F0F77CFCF0F74AFC01F0A1
:1020400065F886F82F508AE00427E4E700218DF830
:102050001810022801D001281BD103983919014416
:102060000998081A20F07F4033280BD903208DF8F7
:1020700015000398C4F13201401A20F07F40322449
:1020800003900CE096F8240018B901F0A9F9002893
:102090004DD0322C03D214B101F02CF801E001F044
:1020A00035F8344A107820B393465278039B121BBC
:1020B00000219DF81840984601281BD0032819D00C
:1020C0005FF000008DF81E00002A04DD981A0390CE
:1020D00001208DF818009DF81C0000B10221039822
:1020E000274A20F07F40039003AB099801F01AF8CB
:1020F00010B110E00120E5E79DF81D0018B99BF82C
:102100000000032812D08DF81C50CDF80C808DF8FB
:1021100018408DF81E509DF8180058B103980123FF
:10212000C11900221846F0F757FC06E000200BB05A
:10213000BDE8F08F0120F0F7FCFB99F90C2001239A
:1021400000200199F0F748FC012086F82F008AF85A
:102150002850034820226946803011F010FC11E01D
:1021600044090020FF7F841E0020A107E83E0200F2
:10217000440700208E0000202F380100971E010028
:10218000FFFF3F000120D2E72DE9F05FDFF8408438
:10219000064608EB860090F82550202D1FD0A8F1A8
:1021A00080002C4600EB8617A0F50079DFF824B4F8
:1021B00005E0A24607EB4A004478202C0AD0F0F74D
:1021C00057FC09EB04135A4601211B1D00F0AAFF1E
:1021D0000028EED0AC4202D0334652461EE0FE4804
:1021E00008B1AFF30080F0F743FC98F82F206AB1F4
:1021F000D8F80C20411C891A0902CA1701EB126198
:102200000912002902DD0020BDE8F09F3146FFF7EA
:10221000DFFE08B10120F7E733462A4620210420DB
:10222000FFF7C8FDEFE72DE9F041E94C2569F0F72C
:102230001FFC401B0002C11700EB1160001200D40C
:10224000FFDF94F8220000B1FFDF012784F822703D
:1022500094F82E00202800D1FFDF94F82E60202073
:1022600084F82E00002584F82F5084F8205084F83C
:102270002150DA4825600078022833D0032831D075
:1022800000202077A068401C05D04FF0FF30A060F0
:102290000120F0F74EFB0020F0F74BFBF0F749FC74
:1022A000F0F741FCF0F715FB10F02AFDCC48056073
:1022B00005604FF0E0214FF40040B846C1F88002BD
:1022C000F0F7D1FC94F82D703846FFF75DFF002839
:1022D000FAD0BF48803800EB871010F816000228AB
:1022E00002D006E00120CCE73A4631460620FFF74F
:1022F00033FD84F8238004EB870090F82600202823
:1023000004D0B648801E4078F0F712FE207F0028E7
:1023100003D0F0F7FEFB2577657749E50146AC4829
:1023200010B590F82D200024803800EB821000BFFB
:1023300010F814302BB1641CE4B2202CF8D3202008
:1023400010BDA84800EB0410016021460120FFF7F2
:1023500003FD204610BD10B5012801D0032800D18F
:1023600071B39B4A92F82D30994C0022803C04EBCB
:10237000831300BF13F812400CB1082010BD521C8B
